:020000040000FA
:1000000020D700206D0A0000A54D0000590A00000D
:10001000590A0000590A0000590A0000590A000054
:10002000000000000000000000000000110B0000B4
:10003000590A000000000000590A0000590A000097
:100040005D0C00005D0C00005D0C00005D0C00000C
:100050005D0C00005D0C00005D0C00005D0C0000FC
:100060005D0C00005D0C00005D0C00005D0C0000EC
:100070005D0C00005D0C00005D0C00005D0C0000DC
:100080005D0C00005D0C00005D0C00005D0C0000CC
:100090005D0C00005D0C00005D0C00005D0C0000BC
:1000A0005D0C00005D0C00005D0C00005D0C0000AC
:1000B0005D0C00005D0C00005D0C00005D0C00009C
:1000C0005D0C00005D0C00005D0C00005D0C00008C
:1000D0005D0C00005D0C00005D0C00005D0C00007C
:1000E0005D0C00005D0C00005D0C00005D0C00006C
:1000F0005D0C00005D0C00005D0C00005D0C00005C
:100100005D0C00005D0C00005D0C00005D0C00004B
:100110005D0C00005D0C00005D0C00005D0C00003B
:100120005D0C00005D0C00005D0C00005D0C00002B
:100130005D0C00005D0C00005D0C00005D0C00001B
:100140005D0C000000000000000000000000000046
:10015000000000000000000000000000000000009F
:10016000000000000000000000000000000000008F
:10017000000000000000000000000000000000007F
:10018000000000000000000000000000000000006F
:10019000000000000000000000000000000000005F
:1001A000000000000000000000000000000000004F
:1001B000000000000000000000000000000000003F
:1001C000000000000000000000000000000000002F
:1001D000000000000000000000000000000000001F
:1001E000000000000000000000000000000000000F
:1001F00000000000000000000000000000000000FF
:10020000DEE61E284CBBCE8F025B0000EC00000037
:100210009A6A0000010000000000000000000000D9
:10022000FFFF02910000000000000000000000003D
:10023000000000000500000000000000DEE61E28AF
:10024000EAAC45B8025B000020000000031000008B
:100250000100000001000000D1500000DEE61E2871
:10026000EAAC45B8025B000030000000021000005C
:100270000000000001000000E11500008D510000A9
:10028000935100000550000074000000DEE61E28B7
:10029000EAAC45B8025B000020000000011000003D
:1002A00002000000010000009B500000DEE61E2856
:1002B000EAAC45B8025B000020000000011100001C
:1002C00003000000010000001D520000DEE61E28B1
:1002D000EAAC45B8025B00002000000000120000FC
:1002E0000000000001000000491B000053B94AB99A
:1002F000002908BF00281CBF4FF0FF314FF0FF302E
:1003000000F00CB8ADF1080C6DE904CE00F036F841
:10031000DDF804E0DDE9022304B07047704700BF58
:1003200030B44FF0000310F8014B11F8015B013AB3
:1003300084EA050443EA0403F5D1A3F101034FEA7B
:10034000D37030BC704700BF4FF0000310F8012B92
:10035000013943EA0203F9D1A3F101034FEAD37053
:10036000704700BF30B411F8014B12F8015B6C40CC
:1003700000F8014B013BF6D130BC70472DE9F04746
:1003800086468C460846089E154674461946002B3C
:1003900040F0C1808542B2FA82F245D94AB1C2F139
:1003A000200300FA02FC954094402EFA03F343EA3E
:1003B0000C0C4FEA154EA8B2230CBCFBFEF80EFB4A
:1003C00018CC08FB00F943EA0C43994528D9EB18EF
:1003D00008F1FF3704D2994502D9A8F102072B444E
:1003E000A3EB0903A4B2B3FBFEFC0EFB1C330CFB16
:1003F00000F044EA0344A04214D92C190CF1FF3355
:1004000004D2A04202D9ACF102032C44241A43EADC
:1004100007401EB1D440002334607360BDE8F0870C
:100420004746DDE76346F1E792BB431B01214FEAF4
:10043000154EAFB2200CB3FBFEFC0EFB1C330CFBC5
:1004400007F840EA0343984561D9EB180CF1FF30F7
:1004500004D2984502D9ACF102002B44A3EB080367
:10046000A4B2B3FBFEFC0EFB1C330CFB07F744EA03
:100470000344A7424DD92C190CF1FF3304D2A742F3
:1004800002D9ACF102032C44E41B43EA0040C0E76C
:10049000C2F120039540944020FA03F12EFA03F3B1
:1004A0004FEA154E9040AFB20343B1FBFEFC0EFB8A
:1004B0001C10190C0CFB07F841EA0041884522D9B1
:1004C00069180CF1FF3004D2884502D9ACF1020062
:1004D0002944A1EB08019BB2B1FBFEFC0EFB1C11F1
:1004E0000CFB07F743EA01439F420ED9EB180CF1CE
:1004F000FF3104D29F4202D9ACF102012B44DB1B35
:1005000041EA004193E76046E3E76146F7E760466A
:10051000A4E76346B8E7834206D916B90021084626
:100520007CE7C6E900E0F9E7B3FA83F78FB98342C5
:1005300001D3724508D8BEEB020460EB030301202F
:100540009C461EB9002169E73846FAE7C6E9004C27
:10055000F8E7C7F1200CBB400EFA07F522FA0CF4BD
:100560002EFA0CF1BA401C4320FA0CF3B8404FEAC3
:10057000144901431FFA84FEB3FBF9F809FB183054
:100580000B0C08FB0EFA43EA00439A4540D9E318E6
:1005900008F1FF3004D29A4502D9A8F102002344A1
:1005A000A3EB0A0389B2B3FBF9F809FB183308FB84
:1005B0000EFE41EA03418E452CD9611808F1FF3344
:1005C00004D28E4502D9A8F10203214443EA004037
:1005D000A1EB0E01A0FB02984145CE46434602D353
:1005E00006D14D4504D20138B9EB020E68EB040385
:1005F000002EA7D0B5EB0E0261EB030101FA0CFC53
:1006000022FA07F3F9404CEA0303C6E9003199E7FF
:100610004046C5E74346D9E72DE9F04307460026A3
:1006200085B0DFF83490DFF8348001AD59F8044B21
:1006300098E807003C4485E807000C22294620463C
:1006400004F0A7FF00B91CB90136052EEED1002435
:10065000204605B0BDE8F083685F0000805C0000C4
:1006600037B504461E480D4604F06FFB2CB91D48F3
:1006700003B0BDE8304004F068BBA1691A4804F03B
:1006800064FB2146A06904F0D7FD40B9174804F087
:100690005CFB204603B0BDE8304001F015BB1448B8
:1006A000616904F052FB0DF1060004F0A5FD40B1B4
:1006B000104804F04AFB104804F047FB0023ADF853
:1006C00006306069BDF80630984203D9294680B2E9
:1006D00000F0B6FF204600F0BDFE03B030BD00BF05
:1006E0008C620000AA620000C5620000ED6200009A
:1006F0001D630000336300005B63000070B54FF4BE
:100700000041002000F054FE064620B1134804F0DA
:100710001CFB002070BD01F04DF9044601F050F9BA
:1007200005462046FFF778FF04462846FFF774FF8A
:10073000054618B1626943699A4209D300212046EF
:10074000FFF78EFF01212846FFF78AFF0448DEE706
:100750000121FFF785FF31462046F5E79E63000043
:10076000CC630000014B1B68184700BF68C5002020
:1007700030B585B004460D4610220021684605F0CC
:1007800069F802238DF80230044B2A462146684658
:10079000019303F087F905B030BD00BF6507000085
:1007A000014B1860704700BF68C5002008B50448B9
:1007B00004F0CBFABDE80840024804F0C6BA00BF16
:1007C000F66300002B640000014802F063BF00BF25
:1007D0007C5F000030BFFFF7FDBF00BF154B9A6A7A
:1007E00012F0007F9A6A14BF1E201D2012F0807F35
:1007F0009A6A18BF1F2012F4801F9A6A18BF02203D
:1008000012F4002F9A6A18BF212012F4802F9A6ADE
:1008100018BF222012F4003F9A6A18BF232012F456
:10082000803F9A6A18BF24206FEA02426FEA1242A0
:100830009A62704700ED00E010B5194B0246986AC5
:100840009C6A10F4805F14BF1720162014F4006F08
:100850009C6A18BF1820A40509D5986B986A0004F3
:1008600004D51AB19A6A22F400429A6219200C4BFC
:100870009A6A12F4806F9A6A18BF1A20D2050CD4B3
:100880009B6A13F4005F18BF1C20054A936A43F467
:100890007F43936200230B7010BD1B20F5E700BF60
:1008A00000ED00E010B51C4B0246986A9C6A10F0FF
:1008B000100F14BF1120102014F0080F9C6A18BFED
:1008C0001220A40709D5586B986A000604D51AB1FE
:1008D0009A6A22F080029A6213200F4B9A6A12F0F1
:1008E000010F9A6A18BF142012F0200F9A6A18BFDD
:1008F0001520D40658BF9B6A074B9A6A920642BFDE
:100900005A6A22F400525A629A6A42F0FF029A62CC
:1009100000230B7010BD00BF00ED00E0F0B5474BA9
:1009200004465B6800258BB0C3F3080385F3118888
:10093000BFF36F8F02F07F40B0F17F4F11D102F013
:100940000C0008280DD010074CBF0C4601250022D2
:10095000033B8DF80720032B05D8DFE803F0246262
:10096000665F2C46F3E700239DF80720CAB902AE64
:1009700004F12007324620686168083403C2BC4293
:100980001646F7D1099A002D53D0C2F3080121B9B8
:100990006FEA52226FEA42220992184602A904F035
:1009A000F7F90BB0F0BD254BDA6A9107DBD4DA6AB0
:1009B000002AD8DBDA6A5200D5D55A69A16942F417
:1009C00080725A61BFF34F8FBFF36F8F5A6931F84E
:1009D000021C22F480725A61BFF34F8FBFF36F8FF6
:1009E0004DF60272914209D09A6AD2B242B1012008
:1009F0000DF10701FFF756FF0346B5E72368B3E79C
:100A00009A6A12F47F4F05D001200DF10701FFF71C
:100A100013FFF1E79B6AB3F5803FA4D3FFF7DEFE37
:100A2000EAE700200DF10701E4E700200DF10701DE
:100A3000EDE722F4FF7222F00102ADE700ED00E0E5
:100A4000044B5A6942F010025A615A6942F48062BA
:100A50005A61704700ED00E0EFF30880EFF3098181
:100A600001B57246FFF75AFF01BD00BF002080F3B9
:100A70001488BFF36F8F002080F30A8880F30B88FF
:100A800001F06EF900200E490860BFF34F8F0D484A
:100A900080F3088800F01AF8202080F311880A48B3
:100AA0004FF40061401880F30988EFF314800221AD
:100AB000084380F31488BFF36F8F00F06BF80000D9
:100AC00094ED00E020D7002020C7002072B600235C
:100AD00083F313884FF0FF300C4A03F120010133F8
:100AE000102B42F82100F8D100234FF0FF30074AC5
:100AF00003F160010133102B42F82100F8D162B6F6
:100B0000BFF34F8FBFF36F8F704700BF00E100E06E
:100B10001EF0040F0CBFEFF30880EFF3098081692A
:100B200011F8021C0229FFD001B504F037F901BD0C
:100B300040B2002807DB01234109034A00F01F00EF
:100B4000834042F82130704700E100E0054B420944
:100B500053F82220012300F01F0003FA00F0104098
:100B6000704700BF00E100E040B2002801F1010140
:100B7000ACBF00F16040064B4FEA4111C9B2ABBFB8
:100B800000F5614000F00F0080F800131954704721
:100B900014ED00E0144A08B5144B22F07F029A606D
:100BA000BFF34F8FBFF36F8FD3F8882022F470020A
:100BB000C3F88820D3F8882042F4A002C3F8882024
:100BC0004FF04042C3F83422BFF34F8FBFF36F8F13
:100BD0000023E1EE103A01F0B1FA01F0F3FA00F06F
:100BE00031F801F0B7FA00BF0000000000ED00E0AE
:100BF0001E4680B50C46074615460023E1EE103A26
:100C000083F30B88DFF824C0ACF5006E8EF30B88FD
:100C10008CF309884FF00000054988472046294693
:100C20003246B84703488047FEE700BF20D7002080
:100C3000BD4D0000CB4D00001022014B1A617047E2
:100C400000ED00E0002320210348C2180133412BAE
:100C500082F80013F9D1704700E100E008B5EFF326
:100C60000583064A103B02EBC30152F83300496882
:100C70008847BDE8084004F09CB800BF745A0000E3
:100C800008B5024B1B689847002008BD20C600200D
:100C9000034B044A1860937843F002039370704743
:100CA00020C600206CC5002008B50649064821F082
:100CB0000701C1F1005202F5802203F0ECFF002091
:100CC00008BD00BF2757012024C600200122024B87
:100CD0000020C3F8402570470090035020B1034B1B
:100CE000800143F001031847704700BFD05C00004B
:100CF000084B70B5C31A0D4607499B10044659436B
:100D00004022064804F077F82B4601462046BDE80D
:100D10007040184730C60020B76DDBB6385A000067
:100D2000402373B50B4C0093041B0B460D460A4938
:100D3000A41061430646094A094804F088F8011ED8
:100D400005DA30462B4602B0BDE87040184702B0C5
:100D500070BD00BF30C60020B76DDBB6BF4E0000CF
:100D6000385A000010B5EFF31184202383F3128862
:100D7000BFF36F8F074A136823F00201DB0711608E
:100D800002D4012004F065FB84F31188BFF36F8F58
:100D900010BD00BF80C6002070B5002201210446AE
:100DA0000520FFF7E1FE0F4801F0C0F80E4B984216
:100DB00015D101F0CBF826690C49304603F0D2FF7B
:100DC00000280BDB012535642469084904F11C0067
:100DD00003F0C8FF002801DB0020E56470BD6FF060
:100DE0000400FBE7B90E00000000AD0B845F0000BB
:100DF0000C22104B014602FB0033002030B4D3E933
:100E00000E529863EFF31180202484F31288BFF30D
:100E10006F8F1C6C04F0C00444F002041C6480F367
:100E20001188BFF36F8F1DB12B4630BC02481847A5
:100E300030BC704730C60020385A000010B4EFF3C1
:100E40001182202383F31288BFF36F8F1848016843
:100E500041F002040460C80708D482F31188BFF38C
:100E60006F8F01205DF8044B01F084B84FF05021E2
:100E7000D1F80C04D1F80C14C907EED5EFF31180AA
:100E800083F31288BFF36F8F0A490B6C03F0C00322
:100E900043F002030B6480F31188BFF36F8F82F37A
:100EA0001188BFF36F8F00205DF8044BFFF7A0BFE0
:100EB00080C6002030C6002010B1012804D0704741
:100EC000034B1B6C5B0701D1FFF792BF704700BF5C
:100ED00030C6002008B5074804F0E8FA38B10648E3
:100EE000FFF7D6FE0448FFF75BFC002008BD6FF05B
:100EF0001200FBE7605A0000FD0E00000A2838B51A
:100F00000446074D04D1AB680D2128465B6898471D
:100F1000AB6803485B68E1B29847204638BD00BF24
:100F2000605A00002DE9F04740F2FF16594FDFF8F4
:100F300068C1DFF868E100EB8101814202D1002045
:100F4000BDE8F087046814F4804FC4F3C325C4F3EC
:100F5000080340F08C80640CB34208BF4FF0FF33AD
:100F60007D5D192C00F28680DFE804F00D13191C5A
:100F70001F251C84848484366084848484848484CF
:100F8000848463787B7EC2F80C355C1C5BD10430B2
:100F9000D3E7C2F814355C1CF9D000245CE0C2F839
:100FA0000835F2E7C2F81035F5E75C1CC2F80835E1
:100FB000EDD0002404E05C1CC2F80C35E7D001241D
:100FC0005FEA531859D14FF00109DFF8CC8009FAD4
:100FD00003FAC8F80CA008E0C2F80835002DDAD1F1
:100FE0005C1CD4D000240625A146D0F800A00AF449
:100FF0000048B8F1000F1CBF4FF00009012403F0B6
:101000001F085B093FD10CEB8808D8F80032CAF3FF
:10101000412A03EA0E0343EA8A0343EA052343EA2B
:10102000090343EA4403C8F80032B0E7C2F80C35BC
:10103000D4E7C2F86035B3F1FF3F0468A7D0C4F32A
:101040000044002CBBD05C091AD10124DFF8488091
:1010500004FA03F9C8F80890A146C6E7C2F8643557
:10106000E9E7C2F86835E6E7C2F86C35E3E76FF008
:10107000150065E76FF0850062E70023DB60FFDEA7
:1010800000239B60FBE7002308F1800853F8283019
:10109000F5E700BF6464000000258450F0F8FCFF11
:1010A0002DE9F04104460D46076904F040FA4FF07F
:1010B000200890B92A4B1B787BB16426606803F046
:1010C0003CFFD0B9012004F062F9013EF6D1F4E70B
:1010D00086F31188BFF36F8FEFE7EFF31186314688
:1010E00088F31288BFF36F8F606803F026FF80B922
:1010F00086F31188BFF36F8FEFE7EFF31186314668
:1011000088F31288BFF36F8F606803F016FF002822
:10111000DED03B691D70626838691368C3F8440506
:101120000120C3F848050020C3F82001D3F820515E
:10113000C3F858015268D3F85801D20608D50820E0
:1011400062681268C2F800054FF48002C3F80423F5
:1011500001229A6081F31188BFF36F8FBDE8F0819F
:101160001DC700202DE9F7434FF0000847680569C7
:101170003C680646C4F800852860D7F80C904146C4
:10118000484601AA03F0ABFE00283CDB019BD9F8DE
:10119000002019791868FFF7C5FE002833DB6B7A49
:1011A0003169012B03D0032B2BD14FF01008AB7A00
:1011B000032B26D195F80BC0BCF1000F02D0BCF177
:1011C000010F1ED12A7A12B1022A1AD10E226B689F
:1011D0007068B3F5164F006800F0B28034D8B3F5EC
:1011E000165F00F0B0801AD8B3F5966F00F0AD80AE
:1011F0000CD8B3F5967F00F0AB80B3F5167F00F006
:10120000AA806FF0850003B0BDE8F083B3F5166FD8
:1012100000F0A480B3F5965FF3D15C4B43E0B3F5E7
:10122000E14F00F09E8008D8B3F5615F00F09B802D
:10123000B3F5964FE5D1564B35E047F6122E734580
:10124000DFD14FF400032EE0B3F5613F00F08D8055
:1012500015D8B3F5963F00F08B800AD84DF6C02E16
:10126000734500F08780B3F5614FCAD14FF46B032B
:1012700019E0B3F5E13FC4D14FF0EB7313E0B3F5E0
:10128000612F7AD009D8DFF820E1734578D0B3F523
:10129000E12FB6D14FF0E86305E0DFF810E17345C8
:1012A000AFD14FF08053C0F82435736848EA0C087A
:1012B0001B6842EA0802C3F86C250B1DD5E9010141
:1012C00083E803007B68990712D505F1180000F048
:1012D000DBFE304B984256D1287E04F10C0204F517
:1012E000907104F056F801202B7E984000F018FE13
:1012F0000823C4F800353B7A53B9C4F81031D4F848
:1013000010316B69C4F834350123C4F838352360D3
:101310007B6800209A075CBF4FF48073C4F80433E5
:101320007B68DB0644BF4FF48003C4F804332B69A9
:10133000C4F844350123C4F84805A360E36062E7BC
:101340004FF41D03AFE7144BADE74FF49E23AAE71C
:101350004FF4A033A7E74FF41C33A4E74FF41D2349
:10136000A1E70E4B9FE70E4B9DE74FF06C739AE79A
:101370000C4B98E74FF4650395E74FF0706392E7E5
:101380004FF080638FE76FF004003CE700B013007C
:1013900000A04E000000AD0B0050270000C07500FB
:1013A00000F03A0000903A0190D0030040420F0054
:1013B00040EA0103C3F30E0330B58BB940F21515B3
:1013C000094CC90BC0F3C730994201D1002030BD90
:1013D000C218D2B202F5C07244F822500133F3E7CA
:1013E0006FF01500F3E700BF00300050002230B569
:1013F000C0F80025D0F80C3585B00093D0F814352E
:10140000124C0193D0F80835114D0293D0F81035E5
:101410006846039350F8041B4B1C0CD001F01F03CB
:1014200049090DD104EB8303D3F80012294041F0A0
:101430000201C3F800120132042AEBD105B030BD1D
:101440000022803352F82330FFDE00BF0025845095
:10145000F0F8FCFF38B5044681692D4803F075FCAF
:101460002C48FFF7C3FF2C48FFF7C0FF4FF0FF32B7
:101470004FF05023C3F80823BFF36F8F72B60023D9
:10148000264903F120000133102B41F82020F8D128
:1014900000234FF0FF30214A03F160010133102B8C
:1014A00042F82100F8D14FF0E02300221A61D3F86E
:1014B000042D03F5506342F000725A605A6A22F418
:1014C000E0225A62EFF31482920707D5EFF31482F9
:1014D00022F0020282F31488BFF36F8FBFF34F8FA5
:1014E000BFF36F8FA26901219A602046A56900F0C1
:1014F0002BFB58B1002383F30B8883F30A882A68F7
:1015000082F3088883F309886B68984738BD00BF69
:1015100080640000008000500090005000E100E076
:101520000122024BC3F80025704700BF0000845021
:101530000022024BC3F80025704700BF0000845012
:1015400070B5EFF30883B3F5004F02D2094D2B7845
:101550000BB1002070BD0126074CC4F8006501F0F6
:101560002DF818B92E70C4F80005F2E76FF00D00E1
:10157000F0E700BF1CC700200000845090B5B1F117
:10158000005F83B002AF1FD2BBB16C46ADF5007DEA
:1015900002AB00934FF4007303F0C5FDA5460E4B5C
:1015A000984213D00A33984213D00C3B984208BF9C
:1015B0006FF015000437BD4690BD084B00934FF403
:1015C000004303F0B0FDEAE70023F7E76FF01500F2
:1015D000F0E76FF08500EDE70202F00020D7002071
:1015E00008B500F049FF034B984208BF6FF01500A3
:1015F00008BD00BF0002F0001FB50446074A01AB5A
:1016000007CA83E807000C221946204603F0C1FFF1
:1016100000280CBF2046002004B010BD8C5C0000E8
:1016200070B505460024054E56F8040B2844FFF714
:10163000E3FF10B90134052CF6D170BD3060000015
:1016400073B50A4606460D460146144803F07DFB75
:1016500001200DF1060103F02DFE044620B10146E4
:101660000F4803F072FB07E0BDF806303BB90D48A8
:1016700003F06BFB6FF01504204602B070BDB5FAA5
:1016800085F1490941EA4601012089B203F02BFEA8
:1016900004460028F0D001460348E2E792640000C7
:1016A000C66400000C650000356500002DE9F04FB0
:1016B000824689B010460F4615461C46D668D2F8B9
:1016C0001080FFF799FF38B914B99C4803F03DFB2F
:1016D000002009B0BDE8F08FA869504503D0002C68
:1016E000F6D19748F2E71CB9B8420BD09548EDE720
:1016F0003846FFF795FF8542EAD12A6A924B9A4213
:10170000E6D109E0FFF78CFF854201D08F48DDE785
:10171000296A8D4B994216D10DF10E0003F06CFD34
:101720000146002837D094B9894803F00EFB894858
:1017300003F00BFBADF80E40D5F81090B9F5A03FC3
:1017400034D98548C2E7854803F0FFFAC0E7002393
:10175000ADF80E30D5F81090B9F5A03FB8D8EB68C9
:101760009945B5D3AE19B3D218EB0703B0D2BD4239
:1017700024D39D4222D2013EB7421FD89E421DD2A1
:1017800018EB0A082CBF01260026EB6926D3002C93
:101790009ED173489AE76969BDF80E20914211D233
:1017A000002C95D16F4803F0D0FA91E7EB6899458A
:1017B000C7D3AE1902D218EB0703D8D3002C87D1B8
:1017C000694883E7D5F81090B9F5A03F02D8EB68D7
:1017D0009945EED2002C7FF47BAFB2E75345D6D3C8
:1017E0004345D4D23A1DA2EB0A02D3589A4504D9F4
:1017F000002C7FF46DAF5D4868E79845F8D907EB9A
:1018000009085B4B08F1050B0DF1100A93E807007E
:101810008AE807000C225146404603F0BAFE544BBA
:1018200010B9B8F1000F7AD108F10108D845EDD10F
:10183000002C7FF44DAF4F4848E7002C7FF448AFB1
:101840004D4843E700F01CF9054658B1002C7FF4E1
:101850003FAF0146494803F078FA71357FF438AF5D
:10186000474833E7474A484B002C14BF93469B46F2
:1018700000F0ACF8854204D3002C7FF429AF434834
:1018800024E75146284600F023F9102801460ED0DF
:1018900010F1160F06D11CB929463D4803F055FA40
:1018A0000135E5E7002C7FF413AF3A484CE754B913
:1018B0002946394803F049FA9DF81F209DF8101079
:1018C000364803F042FA51463B46CDF8009008F105
:1018D000700208F13000D847014690B9304FB54248
:1018E00005D114B92F4803F030FA0120F1E61CB9F4
:1018F0003146384603F029FA304600F011F9013636
:10190000EDE710F1650F05D1002CC9D1264803F091
:101910001CFAC5E7002C7FF4DBAE244814E7D8F8A6
:101920000C20AB699A4288D103F0C0FB0146002825
:1019300088D0002C7FF4CCAE1D4805E76E65000012
:101940008E650000C1650000FFFF0291EE6500009A
:101950003E6600005B630000A5660000176600009D
:101960000167000065660000D46600002D67000076
:10197000985C00005A6700008B670000DE6700007B
:10198000026800009B500000BB5000004669000048
:10199000376800006068000083680000A9680000E4
:1019A000BF680000D6680000F56800001A690000F2
:1019B000BE670000014803F044BC00BF3081FF0057
:1019C000014803F03EBC00BF3481FF00014803F032
:1019D00038BC00BF3881FF0008B50246FFF7F6FFAC
:1019E000904217D914200D4B0D4900FB023003F033
:1019F00028FC0C4B43EA026341EA0262904209D0A0
:101A0000984209D0002383F31188BFF36F8F04231A
:101A1000184602DF002008BD0120FCE73C81FF00E2
:101A20000000FA50FFFFFA502DE9F0410746FFF79A
:101A3000CDFF1423114D03FB0055284603F029FD6B
:101A4000012803D000242046BDE8F0814FF00008B3
:101A50002C1DAE1C304603F01CFD4045F2D9A01CE5
:101A600003F017FD0546204603F013FDB842EAD007
:101A7000023504EB450408F10108EBE73C81FF0067
:101A8000F8B5FFF7A3FF10281AD800244FF6FF7708
:101A90000E4DFFF79BFFA04201D80020F8BD204665
:101AA000FFF79AFF48B1A5F11006304603F0F1FCAC
:101AB000B84208D00236AE42F7D101341435E8E717
:101AC0006FF01500EAE76FF07000E7E75081FF0064
:101AD00070B504460D46FFF77FFFC8B1FFF776FFEC
:101AE000A04218D9142300220C4903FB04118818C2
:101AF00003F0A7FB0023AC1820FA03F60833202BD1
:101B000004F8016BF8D10432102AF0D1104670BDF0
:101B10006FF01500FBE76FF00D00F8E74081FF0064
:101B200010B50446FFF758FF40B11420044B054997
:101B300000FB0430BDE8104000F0C2BA10BD00BF89
:101B40003C81FF000000FFFF2DE9F04F87B0064603
:101B5000009198B303F0E3FB00270446B36BBB424C
:101B60004ED94FF00008DFF8B8A04FF000095AF83E
:101B7000043BDFF8B0B05BF8045B01931D44254BD8
:101B800093E8070003AB83E8070019460C222846B8
:101B900003F0FFFC019B00B9A5B909F10109B9F1F6
:101BA000050FE8D11C4B08F101089845DDD3009BD7
:101BB00013B10022636A1A60236A3BB3002007B0A6
:101BC000BDE8F08F2B6A154A9342EBD1AE42E9D0C3
:101BD000696B05F13C038842E4D025691A69954296
:101BE0000AD19A69A569954206D8E569954203D953
:101BF00062695D69AA4305D0DA6801301344EAE7F7
:101C00000120DCE7009A0AB1626A1360E3680137D9
:101C10001C44A3E7A45C000001000000FFFF029148
:101C2000D4690000446000002DE9F043224885B0EB
:101C300003F075FB002604461F4B204FD3F8388075
:101C4000DFF88090B04503D8002005B0BDE8F083F0
:101C5000636A97E807001D6801AB83E807000C2260
:101C60001946284603F095FC78B975B122692B69AD
:101C70009A420AD1AB69A2699A4206D8E2699A42AD
:101C800003D963696A6993430CD0256A75B10C481E
:101C900003F05BF8002383F31188BFF36F8F0423F5
:101CA000184602DFE36801361C44CBE7484603F0E0
:101CB0004CF8636A1D60F5E700020000B05C0000AC
:101CC000666900008F690000026A044B9A4203D1E2
:101CD0000349203000F0F4B9704700BFFFFF0291C4
:101CE0000000FFFF08B5EFF31083012B0C4A07D16A
:101CF000126ABFF34F8F511C4A424A41104608BD39
:101D000003F023FB00B172B6126ABFF34F8F531C6E
:101D10005A425A4103F019FB0028EFD062B6EDE7B2
:101D20000080FF0008B5EFF31083012B0B4A06D1AA
:101D3000D269BFF34F8F02F00102104608BD03F0D5
:101D400004FB00B172B6D269BFF34F8F02F00102FB
:101D500003F0FBFA0028F0D062B6EEE70080FF0047
:101D600010B503F0F2FA30B14FF050230022C3F85F
:101D70001421C3F8182103F0F7FA28B10122524BBD
:101D8000C3F8382AC3F878254FF47F02D2F83031EF
:101D9000D2F83421BFF34F8FC3F30B03092B05D1C6
:101DA000012A1EBF0122484BC3F8782503F0DCFA54
:101DB00018B10E22454BC3F8E42E03F0C6FA30B139
:101DC0000022414BC3F80C270122C3F81027002240
:101DD000D30003F57F03D3F80013BFF34F8F013116
:101DE00008D0D3F800130132D3F80433B2F5807F62
:101DF0000B60EDD1EFF31084FFF794FF00284DD076
:101E0000BFF34F8F324BD3F80024012AFBD1C3F824
:101E10000425D3F80024012AFBD1012C03D003F0C0
:101E200094FA00B172B6FFF77DFF58B1294AD36921
:101E300023F00103D361BFF34F8F254AD2F800345A
:101E4000012BFBD1FFF74EFF68B1224A136A23F042
:101E5000FF0343F020031362BFF34F8F1C4AD2F8F5
:101E60000034012BFBD1012C03D003F06EFA00B13A
:101E700062B60022164BC3F80425D3F80024012AC9
:101E8000FBD1BFF34F8F1449144BCA6802F4E062D0
:101E90001343CB60BFF34F8F00BFFDE7FFF722FF77
:101EA0000028ADD10C4BD3F88C2042F44062C3F82B
:101EB0008C20D3F8882042F47002C3F88820BFF346
:101EC0004F8FBFF36F8F10BD0040005000A0035034
:101ED000009003500080FF0000ED00E00400FA05D0
:101EE00030B50468ACB1B4FA84F30122C3F11F0326
:101EF000DBB29A4024EA0202D0E8EF5FA54204D1A7
:101F0000C0E8EC2FBCF1000FF6D1EAD102480B700B
:101F100030BD0248FCE700BF0000AD0B0200AD0B76
:101F2000014BC3F80405704700700150044B1A7947
:101F300022B9012218601A7102487047024870479E
:101F400084C600200000AD0B0C00AD0B08B5084B9B
:101F50001B6833B10520FEF7F9FD10B90520FEF727
:101F6000E7FD4FF050230122C3F8182508BD00BF3C
:101F700084C6002010B510B1012847D010BD4FF025
:101F80005023D3F81814D3F81824C90322D502F02B
:101F90000303022B05D0012B02D0002003F000FA2E
:101FA00001234FF050220220C2F8183508224FF4C6
:101FB0008273002103F1502319601C68012402F18F
:101FC00050221460164A126822B34FF05023C3F80F
:101FD0000403D3E7D3F81424D207E1D5D3F81C24A3
:101FE00002F00302013A012AD7D80D4A12681AB149
:101FF0000222C3F80423C1E7D3F80421002AFBD04E
:102000000022C3F80421D3F80431B7E700224FF4CB
:102010008073CEE71A68002AFCD019601B68ADE710
:1020200084C600204FF0502310B5D3F8002152B1E0
:102030000020C3F80001D3F800210122C3F80823CF
:10204000104B1B6898474FF05023D3F8042182B1FE
:102050000022C3F80421D3F80421D3F81824D3F8BC
:102060001824022102F00302012A03D1C3F8181533
:102070009A6010BDC3F80813024B0120BDE8104060
:102080001B68184784C6002001460148FFF728BF97
:10209000B4C500200022034BC3F88425C3F80425EF
:1020A000704700BF00900350044AD2F80834DB07A1
:1020B000FBD50160BFF35F8F704700BF00900350F6
:1020C000012208B5054BC3F88425C3F80425FFF7A2
:1020D000EBFFBDE80840FFF7DDBF00BF00900350F5
:1020E00038B5094B53F82040013053F82050A54231
:1020F00000D838BD636823B1204603F0FCF90834EA
:10210000F5E723689847FAE758600000012208B510
:10211000084B03201A70FFF7E3FFFEF747FB04208C
:10212000FFF7DEFFFEF7EAFA034A137B23F0010311
:10213000137308BD1DC700208CC6002008B50348D6
:10214000034A0021121A03F0EEF908BD20C6002050
:1021500020C7002008B50020FFF7C2FF164B03F58B
:10216000006282F3088883F30A880025E023134C79
:1021700084F82230E57725766576A57684F82050B8
:10218000636A43F4E023636284F82350FEF758FC4B
:10219000FEF752FD4FF0FF33A362E36203F085F9CF
:1021A0000120FFF79DFF0220FFF79AFF2B462A46EA
:1021B00029460348FEF71CFD20C7002000ED00E083
:1021C0000D21000008B50648064A0749121A03F017
:1021D000ACF9BDE80840054A0549064803F0A5B931
:1021E00068C500201EC60020E06900000000000055
:1021F000E069000068C5002030B10268034B044864
:102200009A4208BF0020704702487047DD55AABBBC
:102210008208F0007108F00038B50D460446B0B1F0
:10222000A0220021043003F0A1F995B1082229462B
:1022300004F1640003F0A0F9082205F1200104F183
:10224000840003F099F90020034B236038BD034854
:10225000FCE70348FAE700BFDD55AABB7108F000B0
:102260008308F0002DE9F74305460E4699461146CE
:10227000FFF7C2FF0446002840F08480002E00F0E3
:102280008580002900F08480B9F1200F40F0828021
:1022900005F14404082205F10408204603F06CF916
:1022A00005F1240708223146404603F065F906F19E
:1022B00020010822384603F05FF902A941F8049D85
:1022C0004FF4807003F04CF9002865D14FF480730F
:1022D000324A0121136093600823314A00F034FB35
:1022E0000121052308462F4A00F02EFB0823424611
:1022F00001211C2000F028FB08233A46012103207D
:1023000000F022FB224608230121022000F01CFBE2
:102310000823254A01211A2000F016FB0523234A31
:1023200001211B2000F010FB0823214A0121142069
:1023300000F00AFB08231F4A0121152000F004FBCE
:10234000082305F164020121162000F0FDFA08239C
:1023500005F184020121172000F0F6FA0823164A3D
:1023600001210B2000F0F0FA00F04AFB044601982E
:1023700000F0D8FA114B002C18BF1C46A4212846A7
:1023800003F0F6F8204603B0BDE8F0830C4CF9E703
:102390000C4CF7E70C4CF5E7084CEFE79010845035
:1023A000B06000002861000070600000146100004F
:1023B000D4600000F4600000906000008408F00029
:1023C0007608F0008008F0008108F000C2690C4B2C
:1023D0001A60826943F8042C426943F8082C0269A8
:1023E00043F80C2CC26843F8102C826843F8142C74
:1023F000426843F8182C026843F81C2C704700BF51
:102400005C1684500C4B1B68C3610C4B1B688361CA
:102410000B4B1B6843610B4B1B6803610A4B1B682A
:10242000C3600A4B1B688360094B1B684360094B00
:102430001B680360704700BF5C16845058168450B8
:1024400054168450501684504C16845048168450AC
:10245000441684504016845030B10268034B04483F
:102460009A4208BF0020704702487047DD55AABB5A
:102470000202F0000002F00038B5044668B1051D04
:102480007021284603F074F828462022044903F0FE
:102490006BF80020034B236038BD0348FCE700BF06
:1024A0003C610000DD55AABB0002F0002DE9F043BD
:1024B00085B015466F46274B04460E460FCB87E87E
:1024C0000F002DB94FF00009484605B0BDE8F08374
:1024D0002046FFF7C1FF81460028F5D1231D019357
:1024E000636AA3BB236F8BB1C3F14008A84528BF23
:1024F000A84604F1300031461844424603F034F84F
:10250000236F464443442367A5EB0805226F402A06
:1025100006D104F13001384600F0B4FB00232367F4
:1025200005F03F0835F03F0505D031462A463846CC
:1025300000F0A8FB2E44B8F1000FC3D0424631464C
:1025400004F1300003F010F8C4F87080BCE7DFF845
:102550000890B9E7BC5C00000C02F0002DE9FF41D7
:1025600004466F46134B0E460FCB87E80F002046FC
:10257000FFF772FF8046B0B9CEB1636A251D0195A1
:102580003BB90123226F636204F13001384600F049
:1025900079FB2B46043E243453F8042B12BAA34291
:1025A00046F8042FF8D1404604B0BDE8F081DFF8CA
:1025B0000880F8E7BC5C00000502F000084B1B68CF
:1025C0001B0EF02B08D1074B1A68074B9A4205D116
:1025D0000020064B186070470520704706207047A2
:1025E00028198450241A84500000E0200C1A8450CA
:1025F000002230B5134640F6FC754900023802F15E
:10260000A15404F5823490424FEA840402F101029D
:10261000CABF236025605B181E2AF0D1034A1360ED
:102620000B445360024B034A1A6030BD781084504B
:102630008410845020F80F001E4B30B51A4685B028
:10264000196800910099CC07FAD500F1A15000F566
:1026500082308000016813680193019BD807FAD586
:10266000154B164C186820231F3090FBF3F0144DC7
:102670000138002810DA00230130400153B14FF037
:102680000042A0F12001134204D1013888424FEAF0
:102690005202F8D105B030BD13680393039BDB07EA
:1026A000FAD5431823602B680293029B002BE3D1D9
:1026B0000138DEE7B4108450AC108450E41084502C
:1026C000DC108450F0B51D6885B001F01F040DB911
:1026D0001F2C28D1174D2E462F680197019FFF0709
:1026E000FAD500F1A15000F582308000006835680D
:1026F0000395039DED07FAD51F2C00EB611018BF61
:10270000C9430D4D18BF01F01F0128600B48006838
:10271000029002981CBF00FA01F111604FF0000115
:1027200008BF1060196010684300C00F136005B047
:10273000F0BD00BFB4108450E4108450DC1084500D
:102740000C4B890118603F3020F03F00403058604A
:1027500099600948D9601961596199611C3382B047
:10276000196002680192019AD207FAD5196002B085
:10277000704700BF90108450B410845038B5A0F159
:102780002003B3F5426F05462CD88F2826D800F1D8
:10279000470300F16604DB064FEA541400D001340D
:1027A00064013F34A409013411B1A1421AD30C468B
:1027B0004FF48050E300B0FBF3F0202828BF202026
:1027C00002B110600122084B21461A60FFF710FF8A
:1027D00028462146FFF7B4FF002038BD00F11F0452
:1027E0006409DDE70148F8E71C1884502221F00055
:1027F000464BF0B51D4689B01C680194019CE40766
:10280000FAD5434B002413449B001A680B181E2B67
:1028100088BFC0F11E011F320B1852095343B3F594
:10282000806F84BF4FF48061B1FBF2F1274688BF0F
:10283000091ADFF8E4E000F1A150DFF8E0C000F58C
:102840008230A14233DC2B680493049BDB07FAD56A
:10285000304B1B68296805910599CF07FAD52E4C96
:102860002E49236000231E46934203F1010040D10C
:102870001946002620F0010228488A423CD82968DF
:1028800006910699CE07FAD5254909682868079068
:102890000798C007FAD5216000210C461F488B42DB
:1028A0002DD100201D499A422CD809B0F0BD2B68CB
:1028B0000293029BDB07FAD503199B001B682E6865
:1028C0000396039EF607FAD5CEF800300023934214
:1028D00003F1010306D1164623F00103B34204D8E5
:1028E0000134AEE7CCF80070F1E7CCF800700136A7
:1028F000F4E70E600346B7E706600131BDE7046008
:102900000131CCE708600133CDE700BFB41084503B
:10291000240421147C108450D4108450D810845086
:102920007810845008B540B1202801464FF00702C6
:1029300028BF20210020FFF75BFF0022014B1A6017
:1029400008BD00BF1C188450F0B5294D85B02C4639
:102950002E680096009EF607FAD500F1A15000F50A
:10296000823080000568206801900198C707FAD579
:102970002048214F056002EB8306B24229D100278F
:102980005A1C1D4E22F001029A4227D82368029356
:10299000029BDE07FAD5194B0B449B001B681F33C3
:1029A0005B099A4213D2216803910399C907FAD5AA
:1029B00000211544056008469B1A0F4A8B4210D827
:1029C00000205A1C0C4922F001029A420CD805B092
:1029D000F0BD52F804CBC7F800C0CEE73760013332
:1029E000D2E710600131E9E708600133EDE700BF8D
:1029F000B4108450D4108450D8108450240421146E
:102A00002DE9F041814BA0B01D68986820331E4627
:102A10001A680192019AD707FAD57D4B7D4A1A6050
:102A200032680292029AD407FAD57B4A1A607B4A2E
:102A30001446116803910399C907FAD5784A1168B9
:102A4000C1F3402137680497049FFF07FAD5754FFB
:102A50001F6027680597059FFF07FAD517680029AB
:102A600000F0CF80B90540F1CC803168069106991D
:102A7000CF07FAD56C491960216807910799C907F2
:102A8000FAD51168C1F3402137680897089FFF07FE
:102A9000FAD5664F1F6027680997099FFF07FAD587
:102AA0001268002900F0AF80910540F1AC803268D7
:102AB0000A920A9AD207FAD5564A1A6032680B92DD
:102AC0000B9AD707FAD55A4A1A6031680C910C99BB
:102AD000CC07FAD55749196031680D910D99C9078E
:102AE000FAD55549196031680E910E99CF07FAD57C
:102AF0005249196031680F910F99CC07FAD55049A6
:102B00001960504B1E46196810911099C907FAD5E3
:102B10003F4C4D4B236033681193119BDB07FAD573
:102B20004A4B236033681293129BDF07FAD5484B58
:102B300023603A4B9846196813911399C907FAD53F
:102B4000324F386033681493149BDB07FAD5226048
:102B500033681593159BD807FAD53E4B236033682D
:102B60001693169BD907FAD53B4B2360336817930E
:102B7000179BDA07FAD5394B236033681893189BF3
:102B8000DB07FAD5364B236033681993199BD807B6
:102B9000FAD5344B236033681A931A9BD907FAD5B8
:102BA000314B236033681B931B9BDA07FAD52F4BFD
:102BB000236000F01DFC08BBD8F800301C931C9B60
:102BC000DB07F9D53D6033681D931D9BD907FAD506
:102BD000274B236033681E931E9BDA07FAD5254BDB
:102BE0002360D8F800301F931F9BDB07F9D50C4BEF
:102BF0001B6813F4805F204B08BF184620B0BDE867
:102C0000F0811E48FAE71E48F8E700BF9010845094
:102C10008010845000100251C01F7229B4108450DB
:102C200088108450C0CF0129C01F0E29C03F002941
:102C300040010249003184A800001649400108A162
:102C400080440888B0108450C044708880077A415E
:102C5000C0077E4100006A498006164940006E495F
:102C60000002002100822021408220218082242134
:102C700040A161A100C861510308F1000108F10001
:102C80000208F100324B2DE9F74F804692469946F3
:102C900044681A68002AFCD12E4B9B461A68002A09
:102CA000FCD14FF0FF30019100F094FC802000F047
:102CB00097FC01230720284A284DA2F59E722B601D
:102CC000C2F83C011360636A254F264E3B60A36A3D
:102CD00020463360D8F8003042F8043CD8F8083079
:102CE00098470199D9F80030002BFBD1BAF1000FB9
:102CF00020D104221C4B1A60D9F80030002BFBD1E4
:102D0000DBF800A0BAF1000FFAD1D8F80C30204659
:102D100098473B6863623368A362144BC3F800A012
:102D2000C3F844A1D9F80030002BFBD12B6003B0CD
:102D3000BDE8F08F236A4020012B04BF0B4A1360CB
:102D40000B4B1960C3F804A000F050FCD4E700BF9F
:102D500010198450201C8450001984501818845075
:102D6000CC178450D0178450C817845084168450D0
:102D7000281C8450544B10B5194698B01A6801921B
:102D8000019AD207FAD5514B514A1A600A68029249
:102D9000029AD407FAD54F4A1A600A680392039A36
:102DA000D007FAD54C4818600A680492049AD207F2
:102DB000FAD54A4A1A600A680592059AD407FAD5E4
:102DC000474A1A600A680692069AD207FAD5454A17
:102DD0001A600A680792079AD407FAD5424A1A601D
:102DE0000A680892089AD207FAD5404A1A600A6817
:102DF0000992099AD407FAD53D4A1A600A680A92DC
:102E00000A9AD207FAD53B4A1A600A680B920B9AC3
:102E1000D407FAD5384A1A600A680C920C9AD2077D
:102E2000FAD5364A1A600A680D920D9AD407FAD577
:102E3000334A1A600A680E920E9AD207FAD5314ABE
:102E40001A600A680F920F9AD407FAD52E4A1A60B0
:102E50000A681092109AD207FAD52C4A1A601A4BB7
:102E600019461C681194119CE407FAD5174B186099
:102E7000086812901298C407FAD51A600A6813926B
:102E8000139AD007FAD5124A1A600A681492149A53
:102E9000D207FAD51E4A1A600A681592159AD40705
:102EA000FAD51C4A1A600A681692169AD007FAD503
:102EB000194A1A600A681792179AD207FAD5174A60
:102EC0001A6018B010BD00BFB0108450801084503C
:102ED0000093652100043190409665900083612144
:102EE00000C3302100C3649000816190004610212E
:102EF000008111210041442100C320290C4610C843
:102F00000086312100C3602140C1282940966521F7
:102F10000013319040962529594614C8400432497F
:102F2000494B10B5194694B01A680092009AD2071E
:102F3000FAD5464B464A1A600A680192019AD407AC
:102F4000FAD5444A1A600A680292029AD007FAD562
:102F5000414818600A680392039AD207FAD53F4A9B
:102F60001A600A680492049AD407FAD53C4A1A6097
:102F70000A680592059AD207FAD53A4A1A600A6891
:102F80000692069AD407FAD5374A1A600A68079259
:102F9000079AD207FAD5354A1A600A680892089A41
:102FA000D407FAD5324A1A600A680992099AD207F8
:102FB000FAD5304A1A600A680A920A9AD407FAD5F2
:102FC0002D4A1A600A680B920B9AD207FAD52B4A3F
:102FD0001A600A680C920C9AD407FAD5284A1A602B
:102FE0000A680D920D9AD207FAD5264A1A600A6825
:102FF0000E920E9AD407FAD5234A1A600A680F92E5
:103000000F9AD207FAD5214A1A600F4B19461C684D
:103010001094109CE407FAD50C4B186008681190C6
:103020001198C407FAD51A600A681292129AD0074A
:10303000FAD5174A1A600A681392139AD207FAD57A
:10304000144A1A6014B010BDB0108450801084501F
:1030500080906521000409904096659080806121F0
:10306000802008218020649000816190004610211A
:10307000008111210041442180202029024610C8EE
:103080000086092180206021402128294096652161
:1030900040962529594614C8504B10B51C4696B089
:1030A0001A680192019AD207FAD54D4B4D4A1A601F
:1030B00022680292029AD207FAD54B4A1A604B4A0A
:1030C00042EA804022680392039AD207FAD5186038
:1030D00022680492049AD007FAD5454A1A60A2F5EC
:1030E000800242EA814122680592059AD207FAD508
:1030F000196022680692069AD007FAD53D4A1A60EE
:1031000022680792079AD107FAD53B4A1A602268CB
:103110000892089AD207FAD5384A1A6022680992AA
:10312000099AD007FAD5364A1A6022680A920A9A92
:10313000D107FAD5334A1A6022680B920B9AD2074C
:10314000FAD5314A1A6022680C920C9AD007FAD547
:103150002E4A1A6022680D920D9AD107FAD52C4A90
:103160001A6022680E920E9AD207FAD5294A1A607E
:1031700022680F920F9AD007FAD5274A1A60216861
:1031800010911099C907FAD51A60144B1A4619689C
:1031900011911199C807FAD5114B2049196011688E
:1031A00012911299C907FAD51D4919601168139136
:1031B0001399CC07FAD50B49196011681491149929
:1031C000C807FAD517491960116815911599C907EB
:1031D000FAD5154A1A6016B010BD00BFB010845061
:1031E000801084504004419000862929D81001C8DD
:1031F000401441904014212940146521003440902E
:1032000000310C90C0400C90C030202940960D90A9
:1032100000416090031645C80086112100416021DD
:10322000594644C84014459040142D90264870B526
:10323000054688B004680094009CE607FAD5234C44
:1032400023480460234C44EA83432C680194019C86
:10325000E407FAD50360930143EA824242F0104446
:1032600044F4C0442B680293029BDE07FAD5046045
:103270002B680393039BDB07FAD5174B03608B0185
:1032800043EA814141F0104343F4C0432E68049661
:10329000049EF607FAD503602B680593059BDE07AD
:1032A000FAD5046041F058412B680693069BDC0771
:1032B000FAD5016042F058422B680793079BDB0761
:1032C000FAD5026008B070BDB0108450C021022948
:1032D000801084508071009880611890354B8EB0BA
:1032E00019461A680092009AD207FAD5324B334A2F
:1032F0001A600A680192019AD007FAD5304A1A601A
:103300000A680292029AD207FAD52E4A1A600A680F
:103310000392039AD007FAD52B4A1A600A680492DE
:10332000049AD207FAD5294A1A600A680592059AC2
:10333000D007FAD5264A1A600A680692069AD2077A
:10334000FAD5244A1A600A680792079AD007FAD574
:10335000214A1A600A680892089AD207FAD51F4AC9
:103360001A600A680992099AD007FAD51C4A1A60AD
:103370000A680A920A9AD207FAD51A4A1A600868A5
:103380000B900B98C007FAD51A600A680C920C9A39
:10339000D007FAD5144A1A600A680D920D9AD2071E
:1033A000FAD5124A0E211A6000200D230F220EB00A
:1033B000FFF73CBFB0108450801084508043012937
:1033C00040633921807001298020542100D134903C
:1033D000C0403490C0302029C0530D900041389037
:1033E000832308C880E3102100413821CF4308C857
:1033F00001232DE9F04192B0CDE90333624B1D4624
:103400001A680592059AD207FAD5604B604C236082
:10341000604B19461A680692069AD707FAD55E4B92
:103420001A68D60400F1A8802A680792079AD00784
:10343000FAD55A4A22600A680892089AD207FAD541
:103440001E68C6F30036002E40F098801220FFF769
:10345000F3F807461320FFF7EFF887428CBF1220DE
:103460001320FFF7E9F8471EFFF738FF03AB01AA67
:1034700039461220FFF726F904AB804602AA3946E6
:103480001320FFF71FF900EB4800022832D0032871
:103490003ED0012874D12B680993099BDB07FAD52C
:1034A0003F4B23602B680A930A9BD807FAD53D4B04
:1034B00023602B680F930F9BD907FAD53A4B2360F3
:1034C0002B681093109BDA07FAD5384B23602B68D2
:1034D0001193119BDB07FAD5354B2360013F25D5AE
:1034E0001023192218210020FFF7A0FE304612B049
:1034F000BDE8F0812B680B930B9BD907FAD52D4BB8
:1035000023602B680C930C9BDA07FAD52A4BCFE784
:103510002B680D930D9BDB07FAD5284B23602B6896
:103520000E930E9BD807FAD5254BC1E703AB01AA32
:1035300039461220FFF7C6F804AB044602AA394602
:103540001320FFF7BFF810EB440402D1FFF712FC81
:10355000C4E7FFF7E5FC022C08D0032C09D0012CAE
:1035600010D117211620FFF797FDB7E7152114207A
:10357000F9E70F210E20F6E7124EB7E7124EB5E736
:10358000124EB3E7124EB1E7B010845000084A5112
:1035900080108450B41084508810845000084E511C
:1035A00000065A4940065E4900044241001442495F
:1035B00040042E49000652494006564900063A4941
:1035C00040063E490608F1000708F1000408F10032
:1035D0000508F100014B1860704700BF081A8450BD
:1035E000014B1860704700BF041A8450034A1368E7
:1035F0001842FCD0024A106018467047001A8450E6
:10360000081A845010B50A4C23681BB101232360AB
:10361000002010BD00F046F80028F7D00138062839
:1036200003D8044B53F8200010BD034810BD00BF61
:1036300000C700205C610000FE8FFFFFBFF34F8FCB
:103640000549064BCA6802F4E0621343CB60BFF33E
:103650004F8F00BFFDE700BF00ED00E00400FA055A
:1036600030B44FF0FE320025074B084C084949683A
:10367000C3F80024C3F80424C3F80824C3F80C24B6
:10368000C4F8005530BC0847001084500000845036
:10369000B8C50020024BD0E90012C3E90012704700
:1036A000B8C5002038B500F02FF820B1032400F091
:1036B00063F8204638BD00F031F898B900F0ACF856
:1036C00098B90F4DD5F828391B0EF02B08D1D5F835
:1036D000242A0C4B9A420AD0072400F017F8E6E798
:1036E0000624FAE70424204638BD0024F5E701202B
:1036F00000F092F804460028F7D1C5F80C0AD8E784
:10370000001084500000E020002070470020704727
:10371000014BC3F8040A70470010845010B51148DB
:1037200000F048F800B110BD0F4800F043F8002841
:10373000F9D10E4C204600F03DF80028F3D10C4B97
:103740000C481C6000F036F801460028EBD100F070
:103750002DF8044608B1204610BD00F03FF8204681
:10376000FAE700BFD0C50020CCC50020C8C50020A6
:10377000C0C50020C4C5002008B5084800F024F8E2
:10378000074800F021F8074800F01EF8064800F04E
:103790001BF8BDE8084000F00BB800BFD0C5002002
:1037A000CCC50020C8C50020C4C50020002070473B
:1037B000704700BF08B5034B02681B681068984744
:1037C000002008BDE8C5002008B5034B02685B680F
:1037D00010689847002008BDE8C5002070B5094C66
:1037E000094D2069AB68984718B1084B08485B68D9
:1037F00098470021074AEB6811602069BDE87040D6
:10380000184700BFD4C50020E8C50020B8C5002077
:103810007861000004C70020F8B51A4D1A4E04461E
:10382000B26828699047E8B9184F3B684CB1A3B11A
:10383000012B19D0013B3B602869F36898470020B1
:10384000F8BD43B90121124AC2F800151149D1F857
:103850001029002AFBD101333B60F368286998479F
:103860000020F8BD0C48F8BD0A4AD2F81039002BE8
:10387000FBD1074A6FF07E40C2F80035FFF748FFE2
:103880003B68D7E7D4C50020E8C5002004C7002066
:103890000000845000108450E98FFFFF10B50446EB
:1038A00050B1636813F0685F05D0064A934202D0B6
:1038B00000236260236010BD034B04485B68984797
:1038C000EFE700BF2C5F5CA9B8C50020986100003D
:1038D000C8B143680D4A934213D013F0685F0ED00D
:1038E000012350E8002F194640E8001C9CF0000F0F
:1038F000F7D1012AF5D0BFF35F8F0020704704484D
:103900007047044870476FF4E04070472C5F5CA933
:10391000E98FFFFFEA8FFFFF034680B14268094944
:103920008A420AD012F0685F05D0BFF35F8F002291
:1039300010461A60704704487047044870476FF497
:10394000E04070472C5F5CA9E98FFFFFEA8FFFFF23
:1039500010B5044620B10023034A2360626010BD05
:103960000248FFF77DFEF6E73A00003AC06100002A
:103970002DE9F04101260746B24201DCBDE8F081A5
:103980003B461F4613F8014B002CF7D0252CF8D1ED
:103990001C780237252CF3D00023DFF804819C46E5
:1039A0001D461F2D18D8A4F1200EBEF1100F09D905
:1039B000A4F1300EBEF1090F1ED80A24202504FB05
:1039C00003E304E028FA0EFE1EF0010F06D017F8FC
:1039D000014B002CE5D128E07F2D1CD8A4F1300E3E
:1039E000BEF1090FE9D9242C10D1BCF1000F46D04B
:1039F000B34246D00023EAE724F0040EBEF12A0FBA
:103A0000F8D06C2C09D145F08005E0E724F0040ED5
:103A1000BEF12A0FEED06C2C22D06C2C1BD8682C57
:103A200023D06A2C28D04C2C26D0BCF1000FA5D076
:103A3000B445A1D144F020070B68A7F1650CBCF197
:103A4000020F01D9612F1ED1073323F0070308337A
:103A500001360B608FE7742CB9D07A2CB7D0E4E72D
:103A60002C0648BF45F40075CDE7EC0548BF45F48A
:103A7000007545F48075AAE745F42075A7E79C46D4
:103A8000B8E76324D6E7692C02D007D8632C03D0AB
:103A90002F0601D5AC05D7D40433D9E7732CF6E74C
:103AA000892801002DE9F04F436893B080460193C7
:103AB00083789807CDE9061216D50B4600250B92A0
:103AC0001F789FB1252F15D0013305934146384605
:103AD000019B01359847002880F2458498F8023010
:103AE00043F0040388F802304FF0FF35284613B046
:103AF000BDE8F08F5F789A1C252F0592E6D0002450
:103B00002646A246A346BBF11F0F32D8A7F12003D9
:103B1000102B0AD8DFE803F02409092A0909091B38
:103B200009090922092709091900A7F13003092BFE
:103B30002DD92A2F39D154B90B9B1BF0400F53F8C4
:103B4000042B0B9329D0164601E04BF0010B059B8B
:103B500013F8017B0593002FD5D15BE04BF0020BEE
:103B60004BF0040BF3E74BF0080BF0E74BF0100BB6
:103B7000EDE7BBF17F0F3FD8A7F13003092BD8D871
:103B80001BF0400F03D00A2202FB0636DFE70A22B1
:103B900002FB0A3A4BF0200BD9E7B2F1000AF9DA3E
:103BA000CAF1000A4BF0280BD1E72E2F05D11BF0EC
:103BB000400F9BD14BF0400BC9E7242F1CD1002CA8
:103BC00000F03F81079B1BF0400F0B930AD1524638
:103BD0000BA90698FFF7CCFE0B9B1A1DD3F800A08B
:103BE0000B92B4E732460BA90698FFF7C1FE0B9B78
:103BF0001A1D1E680B92AAE76C2F00F00F8100F2CD
:103C00000681682F00F012816A2F00F017814C2F77
:103C100000F0148134B1079B22460BA906980B9340
:103C2000FFF7A6FE002E47F02003B8BF2BF0400B95
:103C30000293A3F16503BCBF00261FFA8BFB022B86
:103C400040F20481029B612B40F07282FF431BF023
:103C5000400F0CA84BF4C05407F0200314BF3146AA
:103C60004FF0FF31A346049301270B9B073323F04A
:103C7000070303F1080293ED000B0B92049A01F085
:103C8000F1FD431C0646DDF83090DBB20393702350
:103C9000029309F10903122B0CD909F16303C62B16
:103CA00040F20D8109F2E73340F2CE72934294BFA5
:103CB000032704279DF8342002F00C0312F00102C0
:103CC00040F018811BF0020F40F011811BF004043A
:103CD00000F0F780002B40F0108120231BF4405FA0
:103CE00022D1039A002E02F1480208BF01266A443D
:103CF000133A039921B112F8011D302900F03281E5
:103D00001BF0100F039A18BF324619F1040FC0F2CE
:103D10002E81B14580F22B814A454BF4005B40F384
:103D2000288109F10106961B1BF40052089200F04D
:103D3000228129EAE974013403B10134002E00F034
:103D40002181721C1444A245CCBFAAEB04040024B8
:103D50001BF0090F04D12C44A54240F01881002427
:103D60003BB118464146019B013598470028FFF6B4
:103D7000B5AE1BF4006F12D041463020019B98472E
:103D80000028FFF6ABAE049B41460235C3F1780034
:103D9000019B00F0F80098470028FFF69FAE1BF04B
:103DA000080F05D12C44AC4240F0FD80254600248C
:103DB000089B002B00F0268129EAE97A7642A9EBDC
:103DC0000A02039B0AF1FF3A6F1C0292934289BFD9
:103DD0000CAB3020D3185879564500F3ED8041469E
:103DE000019B9847029A002802F10102FFF676AE85
:103DF000BAF1FF3F09D141462E20019B029298471C
:103E00000028FFF66BAEAF1C029A3D46D9E7742F2F
:103E10003FF49DAE7A2F3FF49AAEFBE61BF0800F85
:103E200018BF4BF4007B4BF0800B90E61BF4807FB7
:103E300018BF4BF4007B4BF4807B88E64BF4207B6F
:103E400085E626465446B346B24680E6FF431BF05D
:103E5000400F07F0200308BF062604930B9B07338F
:103E600023F0070303F1080293ED000B029B0B9272
:103E7000652B12D1711C00224BF4805BC9B2134632
:103E800011290CA84FF0020728BF112100F008FBF0
:103E9000DDF83090C3B20393FBE6029B662B05D19D
:103EA0004BF4005B334601221121E9E7F1B2002215
:103EB000652001291346029038BF0121E0E702275F
:103EC000F8E6002B3FF40AAFBAF1030F39DC9DF896
:103ED0003430A44E13F0080FA34B08BF1E46B14662
:103EE0004F4619F8010BA0BBAE1B374485E023BB3E
:103EF0002B23F3E61BBB2D23F0E62022BAF1040F9F
:103F000012DD1BF0080FAAF104040ED12C44414627
:103F10002020019B0135029298470028FFF6DEAD74
:103F2000A542029AF3D192B1002441461046019B6A
:103F3000013598470028CADAD0E52B22DEE72D228A
:103F4000DCE71BF0080FAAF10304C0D1DEE714463A
:103F5000BDE7049B4146C01A019BC0B298470028A8
:103F6000BEDABBE503990139C9B20391C1E6561E19
:103F7000DAE60026D8E61BF4006F0CBF0324052404
:103F80003C44D9E61BF0100F18BF0134DBE609935F
:103F90004146019B20209847002805F10105099B17
:103FA000BFF6DAAE9AE541463020019B01359847CD
:103FB0000028BFF6F8AE91E5D1450AD19DF835301D
:103FC000352B1DD805D19DF8343013F0100F08BFE4
:103FD00031204146019B98470028FFF67FAD1BF03A
:103FE000100F0AD0BAF1FF3F07D1AF1C41462E2077
:103FF000019B98470028FFF671AD3D463C4436E2F0
:104000003120E6E79DF83500414631281EBF9DF876
:10401000343023F010038DF83430019B984700288A
:10402000FFF65CAD002E68DD41462E20019B9847CF
:104030000028FFF653AD4FF0010A039B4146D346DB
:104040009A45B7BF0CAB302053445879019B984731
:104050000028FFF643AD0AF1010A5645EDDA0235B4
:104060005D44029B4146049A981A019BC0B298474E
:104070000028FFF633ADB9F1000F04DB4AD19DF8FB
:104080003430DB0646D5C9F100092D204146019B9D
:1040900098470028FFF622AD042F3DD14FF47A77E0
:1040A0004146019B033599FBF7F606F13000C0B29B
:1040B00098470028FFF612AD07FB16996427414682
:1040C000019B013599FBF7F606F13000C0B2984725
:1040D0000028FFF603AD07FB16990A274146019B0E
:1040E000013599FBF7F606F13000C0B29847002879
:1040F000FFF6F4AC07FB169914E01BF0100F01D18A
:104100000135AEE741462E20019B02359847002835
:10411000A7DAE3E42B20B9E7032F05F10205CDD0A0
:10412000012FDAD109F130006F1C4146C0B25FE7C0
:10413000A7F16303122B00F2FF80DFE813F01700F2
:104140005700FD00FD00FD00FD005700FD00FD00D3
:10415000FD00FD00FD001701F800FD00FD002C0032
:10416000FD00B900C6690000C26900000B9B012474
:104170000CAF1A1D1B680B928DF830301BF0080F26
:104180002AD007EB04093E464E4527D1EF1B3744A2
:10419000AAEB040431E70B9B1A1D0B921F68AA4B74
:1041A000002F08BF1F461BF0400F384614BF314692
:1041B0004FF0FF3101F0FDF90446DFE741462020D2
:1041C000019B98470028FFF689AC013EB442F5D325
:1041D0005544B246AD1BD4E75646F7E7414616F8BC
:1041E000010B019B98470028CEDA77E41BF0800F83
:1041F0000B9B35D01BF4007F2DD0073323F0070332
:1042000003F10802D3E900010B922BF010090029F9
:104210001FFA89F936DA404249F4806961EB4101BD
:104220000DF1300B0A235A4601F0CFF919F0400F77
:10423000A0EB0B0B65D029F001025E4592B240F372
:10424000B280002F00F0A98019F010033446914687
:1042500026D002345CE01A1D18680B92C117D4E70F
:104260001A1D1BF4807F19680B9201D10846F5E7EF
:104270001BF4007F19BF48B241F3C01108B241F3EB
:10428000C031C2E750EA0103CAD11BF0400FC7D0CA
:10429000002EC5D12BF0110B34461FFA8BF9B34613
:1042A00040F2064319EA03031CBF013400232FE048
:1042B0002BF0100B0A231FFA8BFB1BF080040B9AC8
:1042C00057D01BF4007115BF0732101D22F00702F2
:1042D0000B900FBF106802F108010B91D2E90001A9
:1042E00050EA010252D12BF016091BF0400F1FFAC1
:1042F00089F94FD0002E4DD12BF0170B1FFA8BF9F7
:10430000B34619F0100352D0002F4ED10BF1010427
:1043100019F0080F5ED119F0010F06D0A2456DDD2E
:10432000AAEB040404EB0B06544622464DE04BF086
:10433000100B10237827C0E7029B782B04D1C7F11C
:10434000780343F01003B8E741462520019B9847C6
:104350000028FFF6C3AB41463846019B984700282A
:10436000FFF6BCAB0235059BFFF7AABB082300276D
:10437000A3E7111D10680B911BF48071B0D01BF4E2
:1043800000711ABFC0B2214680B2A9E72BF0060B1C
:104390001FFA8BF90DF1300B45E729F0110934466E
:1043A0001FFA89F97CE79146ABE75C4651E75C462A
:1043B00076E7CDE9022341462020019B984700285B
:1043C000FFF68CAB029A039B01329245F1DC2C1B69
:1043D000A5181446EBB141463020019B98470028B0
:1043E000FFF67CAB67B901352F462E44F31B5B45C6
:1043F00021DC5D460CAE4DBB5F44C9E65E4694E7EA
:10440000023541463846019B98470028ECDAFFF711
:1044100065BB40F2064319EA030FE5D019F0020F1D
:1044200005F10105414614BF2B20202019F4806FAF
:1044300018BF2D20E7E741463020019B0137984700
:104440000028D3DAFFF74ABBCA690000013D4146A4
:10445000019B705D98470028CDDAFFF73FBB4146CE
:104460002020019B013598470028FFF637AB631BDE
:10447000002BF4DC77E700BF1FB502AB074A0093BF
:104480004FF0CC3301F085F9DDE90201C00840EAC4
:104490004170C90805B05DF804FB00BFCDCCCCCCA1
:1044A0002DE9F04F9DB055EC104BCDE90B122A468B
:1044B000290D0D93C5F31303D20FC5F30A550790C9
:1044C0008DED050A0A9275B922461A431BD1302395
:1044D0000126056043710A9B43F0020303713046D5
:1044E0001DB0BDE8F08F40F2FF7295424DD1059AA4
:1044F000002613430A9B079A14BF43F0080343F0B6
:1045000004031371EBE7059A4FEA83089A46B14D0D
:1045100002F001020992059A48EA92789700012276
:104520001646C5F1000B0892584600F017FAB5F18F
:10453000FF3FACBF8146A0F10109ABEB090B09EBD2
:1045400005035846069300F00FFA18A9A0F17D055F
:10455000584600F029FA14AB089AA9EB0505019317
:1045600012AB02925146009318AA2B46059801F00F
:1045700053F8B9F1010F04460D4600F2D880099BAB
:10458000002B40F0CB8001276FE0059A43F4801A9E
:10459000A5F2354502F001024FEA8A080992059A10
:1045A000134348EA92784FEA82074BD140F2FE73F8
:1045B00019420CBF01260026002D3246B1DB2846E9
:1045C00000F0C6F90346032DC8BF013B1846069309
:1045D00000F0CAF9069B7C3018A95D1B05441846FB
:1045E00000F054FA14AB18AA0598019312AB514687
:1045F000029600932B4601F00FF8069B04460D46E9
:10460000152B00F2888016AB734A3846414600935A
:104610004FF0CC3301F0BDF8169B179A9B0843EA84
:10462000827303EB8303BB42DDE9129A0CD1384657
:10463000414600F0A1F9069B83428CBF0027012769
:10464000002612E00126B7E7099B002B53D1013F5A
:1046500048F1FF31B81B61F1000100F08DF9069BB4
:10466000099F83428CBF002601260C9B002B40F043
:104670009280DDF82CB04FF000084FF00A0ACDF818
:104680002080CDF81480DDE91201FFF7F5FE149BC0
:10469000CDE90E01184615991093FFF7EDFE0E9B1C
:1046A00081460F9A98420B461191934180F08D807C
:1046B00020462946FFF7E0FE0AFB09F3109AB8F1FD
:1046C000000F14BF002707F001070AFB10480D4632
:1046D000934214BF002606F001060E9B5FFA88F88D
:1046E000044612930F9BCDE91339119B1593089B38
:1046F00001330893C7E7B81C48F1000100F03CF90A
:10470000069B83428CBF00200120B9EB00006AF1B8
:104710000002CDE9120200273E46A6E7129B0127C0
:10472000139A013B42F1FF32CDE9123288E7B9F129
:104730003E0FF0D84FF0FF33A9F12000C9F120015E
:1047400003FA09F203FA00F023FA01F103FA09F37C
:10475000024327EA03070A4328EA020857EA080740
:104760000CBF012700276BE700FB02FC0133A1FB14
:10477000001262448C4275EB020CF5D2069A134487
:104780000D9A13440B9A012BB8BF01239A42A8BF7C
:104790001A4693466FE70A21002201230846E9E7FB
:1047A0000AFB03F00131A2FB0A230344944275EB98
:1047B0000300F5D2594511DDBBF1000F02D154EAD7
:1047C00005030BD00123059372E70A220023012180
:1047D000ECE700BFCCFBFFFFCDCCCCCC7EB34FF0E1
:1047E0000A0A149B159918460F93FFF745FE0F9B75
:1047F0000AFB00F281460E919A4220D1B8F1000FD7
:1048000014BF002707F00107DDE91201FFF734FEAE
:1048100010900F9120462946FFF72EFE0F9B0AFBB2
:104820001048109A04460D465FFA88F81292CDE9B6
:1048300013390E9B1593089B01330893D1E7069B10
:10484000089A13449946002F5BD0B8F1050F58D150
:1048500014F001034BD1059A32B9DDE914239D42CE
:1048600008BF944260D0059B18194FF00A044FF01E
:1048700000024FF0010645F100012546A04271EB10
:10488000020754D2EBB1B3451BDA0C9B63B106EBC4
:1048900009030D9A1A4422EAE2730B9A9A42A8BFBE
:1048A0001A46964293460CDD053009F1010906F1DE
:1048B000FF364FF00A024FF0000341F10001FBF711
:1048C00015FD5E450FFA89F9079BA8BF5E4636B213
:1048D000B14406F1050809F1FF3798444FF000098B
:1048E000B1452BDB079B0A9A1F601A71F7E5059B00
:1048F0002BB9DDE914239D4208BF944209D001235E
:10490000B2E7059B53B9DDE914239D4208BF9442E9
:1049100004D1099B002BF2D1002EF0D0B8F1040F86
:1049200094BF002301239FE74FF00408F1E705FB44
:1049300002F70136A4FB05423A449FE70A2200230E
:10494000FBF7D4FC303209F1010908F8012DC7E763
:10495000014B5843800C704741340100014B5843D0
:10496000000D7047FB2E0B00024B5843C00C01306A
:10497000704700BF4F93120070B50346094A0020EC
:104980004FF0CC364FF0333506FB03F402FB014405
:10499000A3FB023121449D4275EB010401D3013098
:1049A000F2E770BDCDCCCCCC1A232DE9F04FB0FB93
:1049B000F3FA334E03FB1A0389B004460D4606EBA7
:1049C0000A1653B9D6E90023C1E90023D6E902014A
:1049D000C5E9020109B0BDE8F08F2A4A02EBC30322
:1049E000D3E9008904AB404649460093D6E9022347
:1049F00000F0CFFE06AB83460F4640464946009383
:104A0000D6E9002300F0C5FE00238146DDE90662F9
:104A100016EB0B0652EB070828BF012333B1049BAA
:104A2000059A013342F10002CDE904322046039198
:104A3000FFF79AFF07461A2000FB0AF0FFF794FFE2
:104A40003F1A3246434648460399009700F0BCFEA1
:104A50000D4A4FEA141C640004F01E0352F82C4067
:104A6000DC4004F003042418304641F10001DDE984
:104A70000423C5E900414146009700F0A5FEA7E7E1
:104A8000A85D0000D85C0000E46100002DE9F04F53
:104A90001A2700F11905DFF8E8A089B004460E4690
:104AA000B5FBF7F56F434FEA051B0AEB05153A1AFC
:104AB0000AD1D5E90023C1E90023D5E90201C6E9FD
:104AC000020109B0BDE8F08F2B4B03EBC203D3E921
:104AD000008904AB404649460093D5E9022300F023
:104AE00058FE5AF80B206B68013ACDE9020106A97D
:104AF00063F1000340460091494600F04AFE8A46B1
:104B0000029900238146DDE906526D18039952EBA4
:104B1000010828BF012333B1049B059A013342F1F8
:104B20000002CDE904323846FFF71EFF0746204653
:104B3000FFF71AFF3F1A2A46434648465146009758
:104B400000F042FE0D4A4FEA141C640004F01E03FC
:104B500052F82C40DC4004F00304013424182846A9
:104B600041F10001DDE90423C6E900414146009717
:104B700000F02AFEA3E700BFD85C00003862000006
:104B8000785E00007047836800EBC101B3F5004F09
:104B90002CBF51F8220031F81200704700EBC10120
:104BA0008068B0F5004F2CBF41F8223021F8123058
:104BB0007047012208B5FFF7E6FFD04008BD8368C3
:104BC00000EBC101B3F5004F08D34B681AB143F0B5
:104BD00001034B60704723F00103FAE74B881AB1D9
:104BE00043F001034B80704723F00103FAE75300C1
:104BF0000122FFF7D3BFB0F5004F34BF04230823D1
:104C0000481C0833A0EBD300B0FA80F0C0F11F00BD
:104C100070472DE9F0410D4686680446FFF7C9FF4D
:104C2000B6F5004F014601D3012832D03046FFF7D8
:104C3000E2FF04EB80010E6996B90122E36882402D
:104C40001343E36002220D612B4629462046FFF7FD
:104C5000A5FF032229462046BDE8F041FFF79EBF8D
:104C6000022231462046FFF78EFF074603462946BB
:104C70002046FFF793FF0322334629462046FFF7DD
:104C80008DFF39462B462046FFF788FF022231462A
:104C9000E1E7BDE8F081B2F5802F2CBF08230423A3
:104CA0002DE9F0410026D21A8C18CD1D25F00705FC
:104CB00024F00704641BE408056021462046AC602C
:104CC000EE60FFF798FF421D9200013002F10707E6
:104CD0004FEAD7073146A2F1100205F11000B8BF24
:104CE000324600F0B7FD3A4631462846FFF77FFFCF
:104CF0003346324631462846FFF750FFA4EB0708FB
:104D0000284631460122FFF75AFF42463946FFF74F
:104D10006EFF3B46324639462846FFF73FFF2146A5
:104D20002846FFF764FF4346324621462846FFF7F0
:104D300035FF214628460122FFF741FF3946BDE8ED
:104D4000F041FFF766BF002070470FB407B504A914
:104D500051F8040B0191FBF70BFD03B05DF804EB78
:104D600004B0704738B50C46054658B151B10B68D0
:104D700043B14B6833B11C22002100F06BFD0020D1
:104D80002C6138BD6FF01500FBE77047FEE77047F8
:104D9000012801D1EFF3058300F09EBB01460068B6
:104DA000FFF7F6BF08B5FBF715FDBDE8084000F0BA
:104DB00000B8704700210120FFF7EABF61B662B674
:104DC00080F31188BFF36F8F7047EFF311802023BA
:104DD00083F31288BFF36F8F704708B5FBF750FF5E
:104DE000002008BD0C220369C9B201FB0233186C14
:104DF00000F00700704770B5C9B20369EFF3118581
:104E0000202484F31288BFF36F8F0C2606FB013435
:104E1000246C14F0C00408D0A24206D085F3118897
:104E2000BFF36F8F4FF0FF3070BD012206FB0133DF
:104E30001A6485F31188BFF36F8F436803EBC103D6
:104E40005B6898470020EFE78022FFF7D4BFF8B5F2
:104E5000069F0469C9B2EFF31186202585F31288F5
:104E6000BFF36F8F0C2505FB0144256C05F0070C83
:104E7000BCF1010F0CD1276486F31188BFF36F8F4B
:104E8000C4E90E23436853F8313098470020F8BD39
:104E900005F0C005AF4286F31188BFF36F8F0CBFDA
:104EA0006FF077004FF0FF30F1E713B580240094E6
:104EB000FFF7CDFF02B010BD6FF08500704710B452
:104EC0001C240069CBB203FB040000215DF8044BF5
:104ED00010470020FDF74EB8002000F0BABA30B5F8
:104EE00043681360057A446804EBC504A34202D307
:104EF0006FF0010030BD5C798C4201D00833F0E7DF
:104F00000020F7E743681B68D3F88004C3F88004E7
:104F10007047436802691B68D3F8100150B1002044
:104F2000526912780A70C3F81001D3F810210122D7
:104F30001A6070474FF0FF30704702680346D2F89E
:104F4000580140B95B689B0706D4D2F820010038AD
:104F500018BF012070470120704742681368D3F8DA
:104F60000413C90517D5D3F82011A1B1EFF31181AE
:104F7000202080F31288BFF36F8FD3F8200130B167
:104F80000020C3F82001D3F820010120D86081F36C
:104F90001188BFF36F8F5268D20614D5EFF31182D8
:104FA000202181F31288BFF36F8FD3F8581111B10C
:104FB0000021C3F800154FF48001C3F8081382F3F1
:104FC0001188BFF36F8F704710B50446002201218E
:104FD0000920FBF7C9FD0920FBF7AAFD2046BDE823
:104FE0001040FCF7BFB810B504460022012108208C
:104FF000FBF7BAFD0820FBF79BFD2046BDE81040FB
:10500000FCF7B0B830B589B0154601230A46014611
:10501000684600F0DAF8044640B92022694628467E
:10502000FBF77EF9002808BF6FF06404204609B042
:1050300030BD2DE9F04190B09DF85C600446884693
:1050400015461F4601463346402208A800F0BDF829
:1050500038B91022404608A9FBF762F920B96FF071
:10506000640010B0BDE8F081334639466846169AB0
:1050700000F0ABF80028F4D12022334669460DEB4E
:10508000020000F0A2F80028EBD120212B46224696
:105090000DEB010000F01CF8E3E713B501240194C7
:1050A000049C0094FFF7C5FF02B010BD08B500F0E6
:1050B0000DF808B900F068F808BD13B50024019494
:1050C000049C0094FFF7B5FF02B010BDFCF738BA9E
:1050D000F0B5144606460F461D46ADB0FCF720FA63
:1050E000334621462A46009703A800F026FA0446D4
:1050F000FCF71EFAA4F57003A3F676030E2B0DD869
:10510000DFE803F0080C0C0C0C0C0C0C0C0C080861
:105110000C080E006FF015002DB0F0BD2046FBE727
:105120006FF06500F8E72DE9F84F15469A42904672
:1051300081468A461E4628BF9846AB46FCF7F0F9E2
:105140000027AF4205D30024FCF7F2F92046BDE862
:10515000F88F0A9B0AEB07013BB108F103021846DE
:1051600022F0030200F05CFB0A9942464846FDF734
:105170009DF904460028E7D1ABEB080B5E45B0462D
:10518000374428BFD846DCE7FCF7DAB90123FCF73F
:10519000F5B938B504460D46FCF7C2F92946204654
:1051A000FDF7DCF90446FCF7C3F9A4F57003A3F599
:1051B0000073052B04D8252222FA03F3DB0701D460
:1051C000204638BD6FF01500FBE7F0B59FB00446F0
:1051D00001A80D4616461F46FCF702FA50B93B4699
:1051E0003246294601A8FCF7C9F918B9214601A899
:1051F000FFF7CFFF1FB0F0BD13B5044658B1012033
:105200000DF1060100F06CF818B9BDF806305B0826
:10521000238002B010BD6FF01500FAE770B50546A7
:1052200008460C46FCF7FCF92146024601232846B5
:10523000BDE87040FCF73ABA0A4600230146FCF785
:1052400035BAEFF31083012B03D10068BFF34F8F02
:10525000704772B60068BFF34F8F62B670472DE992
:10526000F8430D461646FCF7DFFB0446F8B1F5B1EE
:10527000023000F00EF900278146B8460434B945E3
:1052800007D8002406B134600020A5F80080BDE8EE
:10529000F883204600F0FDF8C3439BB2A21C002B0C
:1052A000F0D0984538BF984614460137E7E76FF0CD
:1052B0001500ECE710B50C46FCF7B6FB58B154B13D
:1052C000023000F0E6F84FF6FF72904203464FF0CE
:1052D000000003D120806FF0150010BD2380FCE793
:1052E0000022FFF7BCBF37B50D4601AA0DF1020140
:1052F000FFF7B5FF044648B9BDF80230AB4208D20B
:10530000019848B1E94389B200F0B3F8204603B0F0
:1053100030BD6FF01504F9E76FF00B04F6E70346B4
:105320005A6B00233C309A4200D17047C168013368
:105330000844F8E7FEF766B908B5FBF745FAFFF74A
:1053400026FDBDE80840FEF75DB94FF47F03D3F8B2
:105350003001D3F83431BFF34F8FC0F30B00A0F10D
:1053600009035842584170474FF47F02D2F8303158
:10537000D2F83401BFF34F8FC3F30B03092B03D1D2
:10538000431E58425841704700207047004700F0C4
:1053900088B840F00040C1F88000C2F88000704733
:1053A000F7B5044618B1012824D003B0F0BD4FF082
:1053B00050230222C3F8082301220646DA60C3F80C
:1053C0000401D3F80431012342F210754FF0502745
:1053D0008DF80730DCB1012CE7D1D7F80C3403F499
:1053E00080338EBB002BE0D00120FFF7D0FF013DC2
:1053F000F3D1DAE74FF050230022C3F808035860D6
:10540000C3F80021D3F800310DF10706DBE7D7F828
:10541000183403F480333EB9002BC6D00120FFF7C7
:10542000B6FF013DF3D1C0E7D7F8182402F003021C
:105430003270002BB9D09DF807000128B5D1FFF7D5
:10544000A6FF013DC6D1B0E7D7F80C2402F0010257
:10545000EEE7FFF7A5BF4FF0FF3307B500F00300FD
:10546000019301AB184400F0CEF9019803B05DF848
:1054700004FB13B50222ADF806100DF10601044637
:10548000FFF7E9FF014624F00300FCF719FE02B024
:1054900010BD20F003031B6882070CBF98B2180CE4
:1054A000704708B1FBF71ABC7047704740B1C3683A
:1054B000587810F001001EBF1878B0FA80F040094B
:1054C0007047EFF31183202383F31288BFF36F8FAC
:1054D000FEE708B5FFF7F5FF10B5EFF311842023C1
:1054E00083F31288BFF36F8FFFF7F3FF84F3118804
:1054F000BFF36F8F10BD10B5D0E9003433B9002071
:10550000E268537843F00103537010BD204698477A
:105510000028F4D00028B8BF4042FF28A8BFFF20D1
:10552000E3681870ECE700F095B900F06CB9EFF3A0
:105530000580003818BF012070472DE9F041069F13
:10554000044615461E46FCF767FE38B93B46324610
:1055500029462046BDE8F041FCF784BEBDE8F08155
:105560000A460021FDF70AB900F04DB900F072B902
:105570000A46002100F06EB901EB820204388A422B
:1055800001D10020704752F8043D1BBA40F8043F97
:10559000F5E70139024410B5904201D1002005E041
:1055A000037811F8014FA34201D0181B10BD013040
:1055B000F2E70246014410B58A42134603D01C7834
:1055C0000132002CF8D1181A10BD2DE9F047C3F1B3
:1055D00037090746884603F01F055FFA89F9164622
:1055E0004FF0000A384641462A465346FAF77EFEF7
:1055F0004346D4B23A4688460746092C84BF4C44F9
:10560000E4B2AA4204F1300473EB0A0306F8014B3A
:10561000E8D23046BDE8F0872DE9F04F061889B092
:105620009946154641EB010404AB3046DDF84CB019
:1056300021460093A9F1410AD2E9002300F0A9F81C
:1056400006AB07468846304621460093D5E902233B
:1056500000F09FF80022DDE90463841951EB030692
:10566000069B28BF0122D5E90001D218079B43F110
:105670000003381848EB0101B84271EB0801E968F2
:10568000039138BF0120A96828BF0020CDF800A0F1
:1056900014EB010C039946EB010110EB0C0041F1F6
:1056A0000001A04271EB060C34BF4FF0010C4FF02B
:1056B000000CCDE906231CEB020243F1000300F0CD
:1056C00083F8129BC3E90001149B012BDDE906233B
:1056D00029D1D5E90201D5E900C5201ACDF800A0ED
:1056E00066EB0101674578EB050534BF0125002510
:1056F000401B61F10001844276EB010534BF0125B6
:105700000025521B63F1000300F05EF8DDE906237B
:10571000CBE9000120463146CDF800A000F054F856
:1057200009B0BDE8F08F17EB070E48EB080C201905
:1057300046EB0601BE457CEB080834BF0127002775
:10574000C71941F10008D5E9000186457CEB010C41
:1057500034BF01200020D5E90215381A68F1000C89
:10576000401A6CEB050192185B41A74278EB0605E5
:1057700034BF01250025521943F10003874278EB1D
:10578000010834BF01250025521BA9F140050095F1
:10579000B8E7F0B50F460446A0FB0201059EA7FB43
:1057A00002524919A3FB0445A7FB037342F100020F
:1057B000611845F10004D21943F10003121943F1B5
:1057C0000003C6E90023F0BDF0B5059CC4F1400715
:1057D000C4F12006A4F12005E04002FA06F6BB4021
:1057E00022FA05F5BA403343C4F120062B4301FAEF
:1057F00006F6A4F12005304321FA05F5E1402843DF
:1058000019431043F0BD0A44431E914200D1704732
:1058100010B511F8014B914203F8014FF9D110BDB9
:10582000884210B501EB020402D98442234607D80E
:10583000431EA14208D011F8012B03F8012FF8E70D
:10584000024401468A4200D110BD13F8014D02F80E
:10585000014DF7E702440346934200D1704703F835
:10586000011BF9E72DE9F04F55EC104BA446C5F3A9
:105870000A540346084644EA0C072946C5F31305B3
:105880003026E14657EA0508AE465E7174D1002421
:10589000A1421C716EDA0121A04219714FF000047F
:1058A0001ADA204603F112060D25C2F157024FF015
:1058B000300C07F00F013F0947EA0E774FEA2E1E22
:1058C000002940F08780A84201DB86F800C0013D36
:1058D00006F1FF36EDD176E00C2868DCC0F10D0151
:1058E0000126890001F1FF3EA1F12108C1F1210744
:1058F00006FA08F826FA07F706FA0EF648EA070845
:1059000016EB060A48EB080BDAF100076BEB4B0EBF
:105910001AF1FF3A4BF1FF3B0AEA0C0A0BEA050BBE
:10592000564578EB0B0B11DBC1F1200BB1F1200ACE
:105930002CFA01F105FA0BFB58BF45FA0AFA41EAC5
:105940000B0158BF41EA0A01C90724D51CEB060C1C
:1059500045EB0805E146B5F5801F1CDB5979B4F528
:10596000806F01F10101597127D007EA0C070EEA97
:10597000050E97E7002891E75CB13126C90F002892
:10598000A4F2FF345E7119710FDB0C28A6DD0D2027
:1059900005E00124F2E707EA09090EEA0505B4F576
:1059A000806F06D04F46AE467CE70020F7E70D201B
:1059B00078E759EA05051A7908D01A794FF4806416
:1059C00042F008021A711C60BDE8F08F42F0040238
:1059D0001A71F8E70929D4BF30318918A84231700B
:1059E000B8BF284673E7000094A9FF7F01000000BC
:1059F000CD0C000000000000990D0000385A000096
:105A00003553000000000000E74F0000605A00001E
:105A1000C94F00004C5A0000D50E000000000000E5
:105A2000A90C000000000000395300000000000035
:105A3000291C00000000000059640000905F000075
:105A4000A05F000018C6002030C600206C64000073
:105A5000BC5F0000246000001AC600207CC5002046
:105A600076640000F05F0000246000001CC6002087
:105A700098C5002000000000B54D000000000000A7
:105A8000B54D000000000000B54D00000000000012
:105A9000B54D000000000000B54D000025200000BD
:105AA0008D53000000000000B54D00000000000014
:105AB000B54D0000605A00005B4F00004C5A0000DA
:105AC0005B4F000000000000B54D0000000000002A
:105AD000B54D000000000000B54D000000000000C2
:105AE000B54D000000000000B54D000000000000B2
:105AF000B54D000000000000B54D000000000000A2
:105B0000B54D000000000000B54D00000000000091
:105B1000B54D000000000000B54D00000000000081
:105B2000B54D000000000000B54D00000000000071
:105B3000B54D000000000000B54D00000000000061
:105B4000B54D000000000000B54D00000000000051
:105B5000B54D000000000000B54D00000000000041
:105B6000B54D000000000000B54D00000000000031
:105B7000B54D000000000000B54D00000000000021
:105B8000B54D000000000000B54D00000000000011
:105B9000B54D000000000000B54D00000000000001
:105BA000B54D000000000000B54D000000000000F1
:105BB000B54D000000000000B54D000000000000E1
:105BC000B54D000000000000B54D000000000000D1
:105BD000B54D000000000000B54D000000000000C1
:105BE000B54D000000000000B54D000000000000B1
:105BF000B54D000000000000B54D000000000000A1
:105C0000B54D000000000000B54D00000000000090
:105C1000B54D000000000000B54D00000000000080
:105C2000B54D000000000000B54D00000000000070
:105C3000B54D000000000000B54D00000000000060
:105C4000B54D000000000000B54D00000000000050
:105C5000B54D000000000000B54D00000000000040
:105C6000B54D000000000000B54D00000000000030
:105C7000B54D000000000000B54D0000FFFFFFFF24
:105C8000DEE61E284CBBCE8F025B0000DEE61E283F
:105C90004CBBCE8F025B0000DEE61E28838451865B
:105CA000025B0100DEE61E284CBBCE8F025B0000CB
:105CB000DEE61E28EAAC45B8025B000002000000E8
:105CC00000000000CD2300000524000000000000BB
:105CD0000338FDD8704700000100000000000000FC
:105CE0000500000000000000190000000000000096
:105CF0007D000000000000007102000000000000B4
:105D0000350C000000000000093D0000000000000C
:105D10002D31010000000000E1F505000000000049
:105D200065CD1D0000000000F90295000000000094
:105D3000DD0EE90200000000514A8D0E0000000057
:105D40009573C24800000000E941CC6B01000000DF
:105D50008D49FD1A07000000C16FF2862300000084
:105D6000C52EBCA2B1000000D9E9AC2D780300001B
:105D70003D9160E45811000031D6E275BC56000038
:105D8000F52E6E4DAEB10100C9EA26836778080092
:105D9000ED95C28F055A2A00A1EDCCCE1BC2D300CF
:105DA00025A4000A8BCA22040000000000000000A5
:105DB00000000000000000100000000000000000D3
:105DC000B9340332B7F4AD1410DB1AB30892540E91
:105DD0000D307D951447BA1A66088F4D26ADC66DF5
:105DE000F598BF85E2B74511CA96853D92BD1DEB7A
:105DF000FCA11860DCEF52163C92AE220BB8C1B485
:105E0000839D2D5B0562DA1C304C7E8F4E8BB25B1E
:105E100016F4529F8B56A512FBD4827643ED8AF07E
:105E20008FE7F9311565191850F19BD94A13EEB473
:105E3000284CF0A686C1251F035FC270CB9E491671
:105E4000E642889C44EB2014B0650836AD6EA5850B
:105E500085F0CA14E2FD031A0B899979D5B13D0981
:105E6000D8DA973A35EBCF10AC363F5E73BB38CFFC
:105E70003E6752FA44AFBA1501000000000000006E
:105E80000000000000000020345065C05FC9A65229
:105E9000BB13CBAEC440C21806C8DF7100D5A87CC6
:105EA000F56F0FDA58FC27136E4756357D242065B1
:105EB00002C7E768E48CA41DE9E60268D7CD396122
:105EC0007977FCC2405BEF16798CDE43FFA751F96E
:105ED00091F3B278F5BDBE11E857E9D6E8BEE87B8C
:105EE000B054AC8F848D751BEA23A499E9F9D38B48
:105EF000B7A3714061DA3E15CEE33ECB73F9480893
:105F00008C97B427D51B7010A2BFEFB9EB85321563
:105F10004DB44DB49BBB6F1996B6076CF8E7EEAD68
:105F200036D9B4F59135AE13222218AF4E6A684DBA
:105F300091DAAA3D4F40741E9FBD9EE006A1C09815
:105F400057C2A7FDA40E90170E7D497173E3208FF1
:105F5000B220D87605143B12853D7434811343B0CA
:105F6000AD297A5F27F4351C000000000002000014
:105F70000004000000080000001000000000000005
:105F80008D4D0000210D0000F10C0000000000000C
:105F90003D0E0000650D0000D34E0000D94E0000FC
:105FA000B94E0000494E0000AB4E0000000000005A
:105FB000E54D0000000000000000000000900050CF
:105FC0000200000000000000CC5F000000900050C4
:105FD000D85F000001000000E05F00000400000046
:105FE000010000000E000400000602000F0606007B
:105FF000008000500200000000000000006000006F
:10600000008000500C6000000100000014600000DF
:10601000040000001D0000001B0004001C0602001C
:106020001A060600134F0000A1100000054F0000E3
:106030000000000000020000000400000008000052
:10604000001000000000000000020000000400003A
:106050000008000000100000F0590000F059000096
:10606000205A0000205A0000385A0000385A000018
:10607000FFFFFFFFFFFFFFFFFFFFFFFF000000002C
:10608000000000000000000001000000FFFFFFFF13
:10609000FCFFFFFFFFFFFFFFFFFFFFFF000000000F
:1060A000000000000000000001000000FFFFFFFFF3
:1060B000512563FCC2CAB9F3849E17A7ADFAE6BCAA
:1060C000FFFFFFFFFFFFFFFF00000000FFFFFFFFDC
:1060D0000000000096C298D84539A1F4A033EB2DFA
:1060E000817D0377F240A463E5E6BCF847422CE1EA
:1060F000F2D1176BF551BF376840B6CBCE5E316B2E
:106100005733CE2B169E0F7C4AEBE78E9B7F1AFEF1
:10611000E242E34FFFFFFFFF7F000000800000002E
:106120000000000000000000FFFFFFFF7F000000F4
:1061300080000000000000000000000067E6096A1F
:1061400085AE67BB72F36E3C3AF54FA57F520E5198
:106150008C68059BABD9831F19CDE05BFF8FFFFFD8
:10616000FF8FFFFFFE8FFFFFFE8FFFFFFD8FFFFF03
:10617000FC8FFFFFFC8FFFFF436F756C64206E6F19
:1061800074206C6F636B20706F776572207361761B
:1061900065206D75746578006D757465785F6672DD
:1061A00065652063616C6C65642077697468204E56
:1061B000554C4C20706172616D6574657200000011
:1061C00043616E277420696E697469616C697A65D0
:1061D000206D757465782C20776173204E554C4C7A
:1061E0000D0A000000000000000000000000000098
:1061F000000000000000004095596959555554555C
:1062000015555556040515411054554045515544F2
:106210004045504450555545004000404004449688
:106220006555565545404554514115405591555574
:106230005555405105010000544554544555050439
:106240000010041014044000000001405555154191
:1062500054040000440001000000004041000044DC
:106260005044455054005555545565510040004028
:10627000010000010005010011545151545555050C
:106280000000000000000000000000004174746580
:106290006D7074696E6720746F20626F6F74207305
:1062A0006C6F742025642E0D0A004E6F2066775F98
:1062B000696E666F2073747275637420666F756E95
:1062C000642E0D0A00417474656D7074696E6720E8
:1062D000746F20626F6F742066726F6D20616464EA
:1062E0007265737320307825782E0A0D0046616937
:1062F0006C656420746F2076616C69646174652CD0
:10630000207065726D616E656E746C7920696E7651
:10631000616C69646174696E67210A0D0046697277
:106320006D776172652076657273696F6E20256482
:106330000D0A004661696C656420746F20726561A6
:106340006420746865206D6F6E6F746F6E69632072
:10635000636F756E746572210A0D00576520617355
:1063600073756D6520746869732069732064756541
:1063700020746F20746865206669726D776172653C
:106380002076657273696F6E206E6F742062656926
:106390006E6720656E61626C65642E0A0D00466151
:1063A000696C656420746F2070726F74656374200B
:1063B000423020666C6173682C2063616E63656C8B
:1063C00020737461727475702E0A0D004E6F206216
:1063D0006F6F7461626C6520696D61676520666FBF
:1063E000756E642E2041626F7274696E6720626FF1
:1063F0006F742E0A0D002A2A2A20426F6F74696E6C
:1064000067206E524620436F6E6E6563742053445E
:106410004B2076322E372E302D35636238353537A6
:106420003063613433202A2A2A0A002A2A2A205576
:1064300073696E67205A6570687972204F532076B1
:10644000332E362E39392D31303062656663373060
:10645000633734202A2A2A0A00636C6F636B403545
:1064600030303000000102030405060775617274C4
:10647000403930303000756172744038303030004F
:10648000426F6F74696E67202830782578292E0D49
:106490000A0053657474696E67206D6F6E6F746F58
:1064A0006E696320636F756E7465722028766572FD
:1064B00073696F6E3A2025642C20736C6F743A20D8
:1064C0002564290D0A004661696C65642064757253
:1064D000696E672072656164696E67206F662074FB
:1064E0006865206E756D626572206F6620746865E0
:1064F00020636F756E74657220736C6F74732C20DB
:106500006572726F723A2025640D0A004D6F6E6FCE
:10651000746F6E69632076657273696F6E20636F46
:10652000756E7465722069732064697361626C654D
:10653000642E0D0A004661696C6564206475726999
:106540006E672073657474696E6720746865206D6A
:106550006F6E6F746F6E696320636F756E746572B2
:106560002C206572726F723A2025640D0A00496E04
:1065700076616C6964206669726D77617265206905
:106580006E666F20666F726D61742E0A0D0054681E
:1065900065206669726D7761726520646F65736EE0
:1065A00027742062656C6F6E672061742064657368
:1065B00074696E6174696F6E20616464722E0A0D75
:1065C0000073726320616E6420647374206D757350
:1065D0007420626520657175616C20666F72206C35
:1065E0006F63616C2063616C6C732E0A0D004669E9
:1065F000726D7761726520696E666F20646F657376
:106600006E277420706F696E7420746F20697473C4
:10661000656C662E0A0D00466972776D61726520A1
:10662000686173206265656E20696E76616C69646D
:10663000617465643A20307825782E0A0D00436134
:106640006E6E6F742072656164207468652066697F
:10665000726D776172652076657273696F6E2E2038
:1066600025640A0D004669726D7761726520766552
:106670007273696F6E202825752920697320736DE8
:10668000616C6C6572207468616E206D6F6E6F74E2
:106690006F6E696320636F756E746572202825754F
:1066A000292E0A0D00496E76616C69642073697A3F
:1066B00065206F7220746F74616C5F73697A6520F6
:1066C000696E206669726D7761726520696E666FAA
:1066D0002E0A0D004669726D7761726520696E66DB
:1066E0006F206973206E6F742077697468696E20FB
:1066F0007369676E656420726567696F6E2E0A0D37
:1067000000426F6F742061646472657373206973F3
:10671000206E6F742077697468696E207369676E84
:10672000656420726567696F6E2E0A0D005265738D
:1067300065742068616E646C6572206973206E6F89
:10674000742077697468696E207369676E65642068
:10675000726567696F6E2E0A0D00436F756C642059
:106760006E6F742066696E642076616C6964206661
:1067700069726D776172652076616C6964617469B4
:106780006F6E20696E666F2E0A0D0056616C69642B
:106790006174696F6E20696E666F20646F65736ED9
:1067A00027742062656C6F6E6720746F207468694F
:1067B00073206669726D776172652E0A0D00626CD6
:1067C0005F63727970746F5F696E697428292072D3
:1067D000657475726E65642025642E0A0D007665F9
:1067E000726966795F7075626C69635F6B657973F6
:1067F00028292072657475726E65642025642E0ADE
:106800000D0041207075626C6963206B65792063AF
:106810006F6E7461696E73203078464646462C2050
:10682000776869636820697320756E737570706F1F
:10683000727465640A0D004B6579202564206861D7
:1068400073206265656E20696E76616C696461743F
:1068500065642C20747279206E6578742E0A0D00A0
:106860007075626C69635F6B65795F646174615FA9
:1068700072656164206661696C65643A2025642EE6
:106880000A0D00566572696679696E6720736967DB
:106890006E617475726520616761696E7374206BD7
:1068A00065792025642E0A0D00486173683A20300E
:1068B00078253032782E2E2E253032780D0A004978
:1068C0006E76616C69646174696E67206B657920AE
:1068D00025642E0A0D004669726D7761726520731A
:1068E00069676E617475726520766572696669653F
:1068F000642E0A0D005075626C6963206B65792007
:106900006469646E2774206D617463682C207472EE
:1069100079206E6578742E0A0D004669726D776174
:1069200072652076616C69646174696F6E2066615E
:10693000696C65642077697468206572726F722073
:1069400025642E0A0D004661696C656420746F2011
:1069500076616C6964617465207369676E617475D2
:1069600072652E0A0D004552524F523A2043616E15
:106970006E6F742066756C66696C6C204558545F48
:1069800041504920726571756573742E0D0A005768
:1069900041524E494E473A204F7074696F6E616C98
:1069A000204558545F415049207265717565737474
:1069B000206E6F742066756C66696C6C65642E0D54
:1069C0000A00696E66006E616E00286E756C6C2937
:1069D0000000000000000000FFFFFFFFFF000000BC
:1069E000474D000000000000DB4D000000000000EB
:1069F000000000000000000000C2010000010300D0
:106A00000000000019C7002018C700200000000087
:106A10000000000000C201000001030000000000AF
:106A20001BC700201AC7002000000000FFFF000065
:106A3000000000003D360000C8C50020E4C500206D
:106A4000DCC50020D8C50020D4C5002010C6002019
:106A500008C6002000C6002000000000F8C5002085
:106A6000513900009D380000D1380000193900006C
:106A700008C700203A00003A0CC700203A00003A4C
:106A800010C700203A00003A14C700203A00003A2C
:0A6A900000000000000015E015E012
:10820000F842002081AA000039F200006DAA0000A7
:108210006DAA00006DAA00006DAA00006DAA000002
:1082200000000000000000000000000019AC000089
:108230006DAA000000000000D9AB00006DAA00008C
:1082400095AD000095AD000095AD000095AD000026
:1082500095AD000095AD000095AD000095AD000016
:1082600095AD000095AD000095AD000095AD000006
:1082700095AD000095AD000095AD000095AD0000F6
:1082800095AD000095AD000095AD000095AD0000E6
:1082900095AD000095AD000095AD000095AD0000D6
:1082A00095AD000095AD000095AD000095AD0000C6
:1082B00095AD000095AD000095AD000095AD0000B6
:1082C00095AD000095AD000095AD000095AD0000A6
:1082D00095AD000095AD000095AD000095AD000096
:1082E00095AD000095AD000095AD000095AD000086
:1082F00095AD000095AD000095AD000095AD000076
:1083000095AD000095AD000095AD000095AD000065
:1083100095AD000095AD000095AD000095AD000055
:1083200095AD000095AD000095AD000095AD000045
:1083300095AD000095AD000095AD000095AD000035
:1083400095AD0000000000000000000000000000EB
:10835000000000000000000000000000000000001D
:10836000000000000000000000000000000000000D
:1083700000000000000000000000000000000000FD
:1083800000000000000000000000000000000000ED
:1083900000000000000000000000000000000000DD
:1083A00000000000000000000000000000000000CD
:1083B00000000000000000000000000000000000BD
:1083C00000000000000000000000000000000000AD
:1083D000000000000000000000000000000000009D
:1083E000000000000000000000000000000000008D
:1083F000000000000000000000000000000000007D
:10840000DEE61E284CBBCE8F025B00008C00000015
:108410005C96000001000000008200000082000065
:10842000FFFF0291000000000000000000000000BB
:10843000000000000000000002000000DEE61E2830
:10844000EAAC45B8025B0000280000000310000001
:108450000100000001000000FF000000010000001A
:10846000F8420020DEE61E28EAAC45B8025B0000B8
:1084700028000000021000000000000001000000C1
:10848000FF00000001000000FC42002053B94AB97F
:10849000002908BF00281CBF4FF0FF314FF0FF300C
:1084A00000F00CB8ADF1080C6DE904CE00F008F84E
:1084B000DDF804E0DDE9022304B07047704700BF37
:1084C0002DE9F04786468C460846089E15467446B8
:1084D0001946002B40F0C1808542B2FA82F245D99C
:1084E0004AB1C2F1200300FA02FC954094402EFAF2
:1084F00003F343EA0C0C4FEA154EA8B2230CBCFB65
:10850000FEF80EFB18CC08FB00F943EA0C43994532
:1085100028D9EB1808F1FF3704D2994502D9A8F100
:1085200002072B44A3EB0903A4B2B3FBFEFC0EFB32
:108530001C330CFB00F044EA0344A04214D92C196C
:108540000CF1FF3304D2A04202D9ACF102032C4457
:10855000241A43EA07401EB1D440002334607360FC
:10856000BDE8F0874746DDE76346F1E792BB431B72
:1085700001214FEA154EAFB2200CB3FBFEFC0EFBFF
:108580001C330CFB07F840EA0343984561D9EB180C
:108590000CF1FF3004D2984502D9ACF102002B4413
:1085A000A3EB0803A4B2B3FBFEFC0EFB1C330CFBD5
:1085B00007F744EA0344A7424DD92C190CF1FF33C5
:1085C00004D2A74202D9ACF102032C44E41B43EAD3
:1085D0000040C0E7C2F120039540944020FA03F127
:1085E0002EFA03F34FEA154E9040AFB20343B1FBAE
:1085F000FEFC0EFB1C10190C0CFB07F841EA0041B5
:10860000884522D969180CF1FF3004D2884502D977
:10861000ACF102002944A1EB08019BB2B1FBFEFCC6
:108620000EFB1C110CFB07F743EA01439F420ED9D6
:10863000EB180CF1FF3104D29F4202D9ACF10201D8
:108640002B44DB1B41EA004193E76046E3E76146C8
:10865000F7E76046A4E76346B8E7834206D916B950
:10866000002108467CE7C6E900E0F9E7B3FA83F7A2
:108670008FB9834201D3724508D8BEEB020460EB88
:10868000030301209C461EB9002169E73846FAE73A
:10869000C6E9004CF8E7C7F1200CBB400EFA07F51D
:1086A00022FA0CF42EFA0CF1BA401C4320FA0CF317
:1086B000B8404FEA144901431FFA84FEB3FBF9F8AE
:1086C00009FB18300B0C08FB0EFA43EA00439A45ED
:1086D00040D9E31808F1FF3004D29A4502D9A8F135
:1086E00002002344A3EB0A0389B2B3FBF9F809FBA8
:1086F000183308FB0EFE41EA03418E452CD9611860
:1087000008F1FF3304D28E4502D9A8F102032144B7
:1087100043EA0040A1EB0E01A0FB02984145CE4682
:10872000434602D306D14D4504D20138B9EB020EBF
:1087300068EB0403002EA7D0B5EB0E0261EB03013A
:1087400001FA0CFC22FA07F3F9404CEA0303C6E9EC
:10875000003199E74046C5E74346D9E7F0B5354BC8
:10876000354A4921C3F800263448C3F8042685B0A9
:10877000C3F80826C3F80C26C3F81026C3F814263D
:10878000C3F81826C3F81C2606F0CCFC06F0F2F855
:1087900000F084FA054601A800F08EFF0446284642
:1087A00000F08CFA264B1B68A34205D045212548D2
:1087B00006F0B8FC06F0E0F9039A4921224806F0D9
:1087C000B1FC4921214806F0ADFC4FF440314FF493
:1087D000004003F0B7FD044620B145211C4806F0D7
:1087E000A1FCFEE769469DF8080000F035F8009B03
:1087F000039D1D44019B1E8903F08CFDAF1901F000
:10880000E9FA01F0B9FA01F0D3FA84F30B8884F3A2
:108810000A88AB5983F3088884F31488BFF36F8FF9
:10882000BFF36F8F7B68984745210A4806F07AFCB2
:10883000FEE700BF008001503546526E280F010050
:1088400008000020410F0100640F0100930F010098
:10885000B80F0100EB0F0100024608B538B105481A
:108860000023452106F05EFC6FF0150008BD08608E
:10887000FCE700BF0E10010021B1012908D06FF004
:108880001500704748B10128054818BFFF20704700
:10889000022834BF0220FF2070470D20704700BF20
:1088A000080000002DE9F04FDFF8F8A1FDB03CA86A
:1088B000DDE9888916461C468A9FDAF8005003F0E5
:1088C0005FFDB8F1000F07D0B9F1000F04DD4A4693
:1088D00041463CA803F062FD4FF0000833897289DD
:1088E000D6F80CB013449B44C3453AD80CA93CA815
:1088F00003F05AFD27B1202238460CA906F0E5FC0A
:1089000000232246009331464FF6FF7306A806F077
:1089100032F8804610BB20460B9E00F0A9F9864233
:108920001CD84FF0FF37DFF880910DF1120304AA35
:1089300005A906A806F06DF800280FDB40F0A88016
:10894000059906A806F0B1F810BB4FF6FF71BDF807
:108950001200564A32F8023B8B4217D1DAF8005027
:108960009AE0879BABEB0809994528BF9946414699
:108970004B462046869A06F0E3FB0028EED14A4695
:1089800086993CA803F00AFDC844ADE79842E1D1BE
:10899000BDF81230102B1ED1BDF81060202EDDD195
:1089A0003346204605991CAA06F0CAFB0028D5D1FB
:1089B00000F074F9324680461CA90CA800F0FEF8BD
:1089C0000646404600F07AF9394B1B68B342C5D1E0
:1089D0004FF00108A9E7012B32D1BDF81030202B50
:1089E000BCD8204605991CAA06F0AAFB0746002819
:1089F000B4D19DF810B0BBF1200F02D94FF0FF3772
:108A000093E7D9F800302B4E0393039B9F42F5DA8E
:108A10003CA803F0B5FC72683CA8126856F8081B25
:108A200003F0BCFC14A93CA803F0BEFC5A461CA9E8
:108A300014A806F03AFC00283FF477AF0137E4E7CA
:108A4000222B7FF472AF7B1C3FF46FAFD9F800305C
:108A5000BB42D3DDBDF81030802B3FF67FAF204600
:108A600005991CAA06F06CFB00287FF477AF00F094
:108A700015F9FFB206462021BDF810301CAA009758
:108A80000CA800F019F80546304600F017F9B5E7D4
:108A9000B8F1000F3FF462AF00F008F928467DB04E
:108AA000BDE8F08F04000020780A0100FC0E0100F0
:108AB000080000207C0A01002DE9F04796B0164618
:108AC0001D469DF87820384B074653F8321003EBCB
:108AD000C2035B6801911868DFF8D080014430233D
:108AE00002AA01A8D8F8009006F0B9F9002851D1DF
:108AF000DDE901431C44214606AB03AA01A806F0A8
:108B0000D6F9002846D1049A072A43D12849059866
:108B100006F0CBFB00283DD1079A082A3AD1254917
:108B2000089806F0C2FBA8BB214602AA01A806F0DD
:108B3000AAF978BBDDE901A30AEB0302944229D12B
:108B4000412B27D135443023294603AA02A8029697
:108B500006F085F9E0B9DDE9023213449D4217D3EE
:108B60002A4602A906A805F0AEFF88B92A4602A93E
:108B70000EA805F0A8FF58B99AF80030042B07D1C9
:108B80002021384606AB0AF1010203F013FC38B18C
:108B9000D8F8009000F08AF8484616B0BDE8F08793
:108BA000054BD3F80090F5E77C0A01000400002093
:108BB0003D100100341001000800002070B5094B81
:108BC00004461D680023934205D1074B1D6800F041
:108BD0006DF8284670BDE65CC85C8642F7D101336B
:108BE000F1E700BF04000020080000200B7868B106
:108BF000012806D0FF2B14BF4FF0FF304FF4407018
:108C00007047054A934203D0022BF4E70D2BFAE795
:108C10004FF44070704700BF080000001FB50C46BD
:108C2000A8B1012815D11048C0B2214601F080FC3E
:108C300050B92068102381686A46103906F080FA1E
:108C400048B1206806F07BFA4FF0FF300AE00D20B3
:108C5000EBE7FF20E9E710226846044906F025FB10
:108C60000028EED104B010BD08000000180F01006C
:108C700013B5044605F058FF6A460146204605F044
:108C800060FE30B10448452106F04CFA002002B0E5
:108C900010BD0098FBE700BF45100100024B1868AB
:108CA000421C1A60704700BFD0030020024A1368BC
:108CB000013B1360704700BFD0030020034B1B68CB
:108CC000834201D005F058BF704700BFD003002099
:108CD00003464FF4807213B5084693F8B81001921A
:108CE000C1B1012903D0FF2804D0012010E0104AAF
:108CF000904211D1582404FB013204FB0133526A23
:108D000003F1280401A901F03BFC08B9019B236091
:108D100002B010BD0D28ECE70228E6D1582404FB70
:108D2000013204FB0133126D03F15404EAE700BF82
:108D30000800000038B590F8B8300446F3B1012BB4
:108D400006D0FF21FFF7C4FFD0B10125284638BD6A
:108D50000D49FFF7BDFF0028F7D102212046FFF79C
:108D6000B7FF054670B9582294F8B83002FB0343A8
:108D7000186A06F023FAC4F8B400E7E70D21E8E723
:108D8000FF21EBE70925E1E7080000002DE9F04F9E
:108D90004A4B8DB0044690F8B8000D461E68FFF7A8
:108DA0006BFD0AA9C0B201F0C3FB28B1FFF77EFF3B
:108DB00030460DB0BDE8F08F94F8B8B0294658465B
:108DC000FFF75AFD4FF02C080BA9C0B208FB05F8BD
:108DD00001F0AEFB00284ED04FF0580A2C230AFBBE
:108DE0000BF703FB057704EB0709D9F8106016F0C1
:108DF000100655D1FFF752FF0A9B94F8B810069061
:108E000009930891FFF74AFF07904FF480701AFB0F
:108E10000B8201902A48CDE90366099B08990296C6
:108E2000009022443046FFF73DFD06460798FFF7C5
:108E300045FFFFF73BFF0698FFF740FF214BE25944
:108E40000A989A420CD1D9F80C20B9F808309B182E
:108E500006D28268934203D21B4B1B68B34226D0D2
:108E60004DB38268002106F095F9184A452118484B
:108E700006F058F919E00B9806F0A7F906460B988A
:108E800006F05DF9582394F8B82013FB02832344BD
:108E90005A1E033312F8011FB1429DD19A42F9D1F3
:108EA0001DB120460A9905F002FF0A4B1E680A9878
:108EB00006F045F97AE7084AD8E700BF0400002029
:108EC0009C3000203DB8F396080000208810010077
:108ED0009210010000000020801001007FB50D46B7
:108EE0000021044690F8B8202846CDE9021105F08B
:108EF000CFFE60B358235A431C4EA358B34203D14C
:108F0000204603AA05F06CFE582294F8B83002FB04
:108F10000343DB6AB34204D10121204602AA05F0D3
:108F20005FFEDDE90232934288BF0393039BAB608F
:108F3000039A2946204600F0F9FD0D4B1A68002AD5
:108F400003DD57210B4806F0EDF804B070BD104664
:108F500001A9FFF763FE019805F1080105F0EFFD97
:108F6000AB680198039306F0EAF8E1E73DB8F396A1
:108F700090280020BA1001007FB590F8B83006465E
:108F80000D468BB3012B1A4818BFFF2001A9C0B2B0
:108F900001F0CEFA50BB019805F0C6FDD6F8B4102A
:108FA0000446284605F0FAFE0444019806F006F946
:108FB0000646019806F009F9082201460DEB020069
:108FC00006F08EF92B7921468DF80830019833464A
:108FD00002AA06F0CAF8041E019818BF012406F080
:108FE000AEF8204604B070BD0D20CFE70124F8E7AD
:108FF000080000002DE9F84F884691469A46002661
:10900000DFF868B01A4C1B4D0B9B9E4201D3002029
:109010000FE00B9B40469F1BB7F5806F28BF4FF4B6
:109020008067124A3B4606EB0A0106F089F810B148
:109030000120BDE8F88F0A993B465A464846711808
:1090400006F093F80028F3D1C4F800563E44C4F863
:109050000456C4F80856C4F80C56C4F81056C4F8A0
:109060001456C4F81856C4F81C56CDE7D423002073
:10907000008001503546526E2DE9F04F4FF0000A46
:1090800004460E46574693B0BAF1010F84F8B8A0D3
:1090900006D9002F00F0F28100202C25582767E127
:1090A00004EB0A0292F8B950002D4AD14FF058094A
:1090B0004FF02C0B09FB0A42B04B03EBCA21B04B1B
:1090C000516203EBCA21116529465046FFF7D4FBD4
:1090D000202394F8B810804619FB01310BFB0511D1
:1090E000C0B2214401F024FA48B15346424645211A
:1090F000CDE90050A34806F015F805F03DFD4FF00E
:1091000001087DB12046FFF715FE054660B9002233
:109110002046114605F043FDC8B1572194F8B82008
:10912000994824E04546CFE74FF48072572197488D
:1091300005F0F8FF94F8B830012D234483F8B0808F
:10914000E5D194F8B83001335FFA83FA9CE7204602
:1091500005F037FE68B108A805F091FD01462046EC
:1091600000F0C4FA60B1572194F8B820884805F09F
:10917000D9FF012294F8B830234483F8B020E0E707
:1091800008A805F085FD80F0010108AA2046C9B2B3
:1091900005F005FD02460028BFD108A805F078FDBE
:1091A000054600284CD194F8B8305BBB204608A98E
:1091B000FFF794FE94F8B8009DF82730221882F843
:1091C000B030033B012B08D800F0F4FA28B1FF229D
:1091D00094F8B830234483F8B0209DF8273094F8F1
:1091E000B800023B022B1ED800F0C8FAD8B1FF220B
:1091F00094F8B830234483F8B0204521654805F041
:1092000091FFFEE794F8B020042A04BF012284F8FD
:10921000B020012BCAD094F8B130042BC6D1012361
:1092200084F8B130C2E794F8B830234493F8B030F2
:10923000FF2BE2D00021204608AA05F0B0FC98E7F9
:109240009DF82730012B74D1582194F8B830DFF8FD
:109250004881059208F8032001FB03434F4AD96A6D
:10926000D86C914247D1998E042305AA194405F080
:1092700067FF014608B34FF0050994F8B83023445E
:1092800083F8B09094F8B83073B1E21892F8B02037
:10929000012A3FF456AF042A0DD094F8B020042AD6
:1092A00002D1012284F8B020234493F8B030023B6D
:1092B000022B3FF646AF2F4643E794F8B800FFF77E
:1092C000DBFA0CA9C0B201F033F90028D3D10C9A13
:1092D000059953688B4229D892681A44914225D83F
:1092E000B3F5004F02D0B3F5003F04D1012294F84A
:1092F000B83008F8032094F8B80003F02DF9831E65
:10930000022B8146B9D8FFF7C9FC012180462046CF
:10931000FFF73CFD82464046FFF7D0FC204B1B6820
:109320009A45AAD01F4B1B689A45A4D14FF001095A
:10933000A3E7FFF7B3FC012180462046FFF726FD97
:1093400081464046FFF7BAFC154B1B68994518BF8C
:10935000052294F8B83008BF9DF82720234483F8ED
:10936000B0208FE7231893F8B920EAB10130C0B2DA
:10937000012884F8B800F5D980E000BFD41300209C
:10938000D4030020E910010078110100361101001A
:10939000A4110100CE1101009C3100203DB8F396CC
:1093A000080000200000002093F8B08008F0FB08BF
:1093B000B8F1010818BF4FF001084146FFF75CFA09
:1093C00003A9C0B201F0B4F8002840F08C8001235A
:1093D00005FB08F894F8B810039A17FB0181009375
:1093E000214440230CA805F0C6FA804600287CD111
:1093F00000230DF10A0204A90CA805F00AFB0028BD
:109400003CDB03987ED1BDF80A300C2B78D104994F
:1094100005AA05F095FE00287DD19DF81430012B9A
:109420007CD8E21892F8B0207B43023A022A8CBF23
:109430000022012205FB02332344197D9DF81820E8
:109440009142D5D80AD3597D9DF819209142CFD8A1
:1094500004D3DA8ABDF81A309A42C9D294F8B830E7
:109460000398234493F8B020012A3AD0023A012A03
:1094700002D8012283F8B02005F061FE0022894D58
:10948000894F012A84F8B8204BD90023874DDFF893
:109490002082884F0C93012B84F8B83040F29980D9
:1094A0000C9B022B01D005F067FB94F8B930002B20
:1094B00040F0DB80582505FB034284F8B830106A81
:1094C00005F03DFA307194F8B83005FB03431B6A90
:1094D0005B68B36094F8B83003FB05453560734BA7
:1094E00093E00422C6E70398C6E7039805F027FE39
:1094F000B8F1030FC2D140F20113A4F8B030BDE7B8
:109500004FF00308039805F01AFEB8F1000FEFD1F1
:1095100094F8B8002AE74FF00108F3E74FF0070886
:10952000F0E7A11891F8B93043BB08A805F0A7FBF4
:1095300091F8B030042B8DF8273006D8012B22D8B3
:109540000FD0FF2381F8B0300BE0052BF9D1104686
:1095500000F030F928B1FF2294F8B830234483F8A2
:10956000B02094F8B830234493F8B030FF2B05D1E5
:109570004521284605F0D6FD05F0FEFA94F8B820FE
:109580000132D2B27DE7204608A9FFF7A7FC94F884
:10959000B800231893F8B030DA1E012A0FD800F073
:1095A00009F978B994F8B80000F0E8F850B994F8DF
:1095B000B830FB5C002BD4D0012000F095FE022BCC
:1095C000F5D1EFE7FF2294F8B830234483F8B020B8
:1095D000EDE7234493F8B9208DF814209DF814107A
:1095E00001F0FF0239B10C9B01330C9394F8B830B1
:1095F0000133DBB24FE793F8B030012B07D01146AF
:10960000204605F0CCFA10B1294B1D681AE094F8F9
:10961000B830012BE7D0FFF741FB002182462046FE
:10962000FFF7B4FB81465046FFF748FB2B6899458E
:1096300006D1D8F80030994502D03B689945D2D17F
:10964000D8F800501022002108A805F049FE58263D
:109650000023012B84F8B8300FD9FFF727FB2846E9
:1096600013B0BDE8F08F012324E794F8BA30002B43
:10967000F9D0022384F8B83031E7E21892F8B92023
:109680005AB906FB0343D86C05F059FD94F8B8307D
:1096900006FB0343186A05F052FD94F8B830013315
:1096A000DBB2D6E7CE1101009C310020080000207B
:1096B000040000200000002070B50B4E0446BC22C0
:1096C0000021304605F00CFEFFF7E8FA214605467A
:1096D0003046FFF7D1FC04462846FFF7EFFAFFF7C4
:1096E000E5FA204670BD00BFD427002073B50D46B3
:1096F000064600F05BF90446E86090B3022837D1D3
:1097000096F8B83083B3012B1B4818BFFF2001A97E
:10971000C0B200F00DFF68BB2A463146019800F048
:10972000DFF80446D0B9019806F06FFC012301462A
:109730000DF10302019805F003FD0446B0B90122C2
:1097400001980DF1030106F074FC10B101238DF8AE
:1097500003309DF8033003F00F03EB71019805F01F
:10976000EEFC204602B070BD0D20D0E70124F5E7E5
:109770000724F6E70124F4E70800000013B588B1D8
:10978000012811D10A48C0B201A900F0D1FE68B980
:10979000019806F0E5FC0446019805F0D0FC20464F
:1097A00002B010BD0D20EFE7FF20EDE70124F6E742
:1097B000080000001FB5D8B101281BD11048C0B265
:1097C00001A900F0B5FEC8B9019802A902F06EFE29
:1097D000044688B99DF80B30032B03D1019806F09D
:1097E0008DFC0446019805F0AAFC204604B010BD8B
:1097F0000D20E5E7FF20E3E70124F3E70124F4E788
:10980000080000002DE9F74306460C4690461D4629
:109810000BB900272FE0184605F03AFA0028F8D1D6
:10982000694696F8B800FFF7F9F9009838B90124AD
:10983000009805F084FC204603B0BDE8F08301A940
:1098400005F07DF90028F2D1009805F078FC30464B
:10985000019905F094FA582296F8B83002FB036398
:109860005B6A5F686B79012B23D1002CD1D12B6807
:10987000834298BF0027214696F8B800FEF7FCFF08
:109880006946C0B200F054FE0028D0D120234246E1
:109890003946009805F054FC04460028C7D1002D35
:1098A000C6D0D8F800400D4BE41A18BF4FF0FF3473
:1098B000BEE7022BADD12B68012B05D98342A8D876
:1098C000B4FA84F46409A4E7A3D1002CD3D0012C0A
:1098D0009FD12C79023C18BF01249AE73DB8F3963A
:1098E0002DE9F04F0C460746014685B094F8B800C4
:1098F0001646FFF77BF9051E52DB3846D4F8B44014
:1099000005F012F95FFA84F94FF0000A4FF0010BED
:109910004FF0FF346B1E09FB03089DB9BAF1010F2C
:1099200003DD4521204805F0FDFB631C06D0FF2C1C
:109930002ADC40F2011301343460B380284605B0BC
:10994000BDE8F08F6B1E00934146012338460DF1B0
:109950000F0205F0F5FB031E019323DB01223846BD
:109960000DF10F0106F065FB019B40B15B4501D095
:109970000AF1010A9B46009DA8EB0908CDE7B4F166
:10998000FF3F08BF2C46F5E70223A4F580747371EE
:10999000631004F001040133013433603471CDE706
:1099A0000725CBE70125C9E7DA11010010B590F8CA
:1099B000B84088B0002C4ED0012C2D4818BFFF2095
:1099C00004A906F0A8FB9DF81020012A45D0294BD8
:1099D0002949032A08BF0B469DF813202748029205
:1099E0009DF81220492101929DF811200092244AED
:1099F00005F098FB012C8CBFFF20022006A906F081
:109A00008AFB9DF81820012A29D01A4B1A49032AEB
:109A100008BF0B469DF81B20492102929DF81A2091
:109A2000164801929DF819200092164A05F07AFB1B
:109A30009DF81030012B14D19DF81230032B10D15A
:109A40009DF81830012B0CD00F48492105F06AFB16
:109A5000022008B010BD0D20B2E70C4BBCE70B4B49
:109A6000D8E70B48492105F05DFB0020F1E700BF76
:109A700008000000FD110100061201001A12010089
:109A80000C1201005B1201006B12010001120100B7
:109A90008A12010070B54B6814461E4A03F0FF237A
:109AA000934206460D4686B02FD10B68012B2CD170
:109AB000204604A902F0FAFC9DF81020012A26D0C5
:109AC000154B1649032A08BF0B469DF81320492160
:109AD00002929DF81220124801929DF811200092E6
:109AE000104A05F01FFB9DF81030032B0DD12146C5
:109AF000304605F0DCF8204606F000FB2046A96859
:109B000005F02BF8204602F0B1FC06B070BD064B04
:109B1000DBE700BF00010004FD1101000612010097
:109B20001A1201005B120100011201002DE9F04F31
:109B300004461646582789B00D468548492105F048
:109B4000F1FA3146204605F01AF994F8B830834608
:109B500007FB03435B6A28465E6805F099F810B37B
:109B6000D4F8B40004F0DBFF94F8B83007FB0343EB
:109B70009F6A0023013F3344834201D2013FFAE749
:109B8000BB4510D35721734805F0CCFA07FB06F309
:109B900057210BFB0662704805F0C4FA0123EB71F4
:109BA00009B0BDE8F08F94F8B83006A9D3B1012B05
:109BB00012D0FF2000F0BCFCFF2007A900F0B8FC89
:109BC00029462046079AFFF765FF6B79012B58D18C
:109BD0005F46DFF888A14EE06148C0B200F0A8FC03
:109BE0000220EAE70D20F9E72A68C2F101035B448D
:109BF0009F423FD8582194F8B830012A01FB034313
:109C00005B6A196853F8370003EBC70353F8083C45
:109C1000A0EB0109A3EB0103049311D1079B03936C
:109C2000EB68022B08D04146204605F040F82A4652
:109C30004146204605F07FF82046039905F037F8A5
:109C400032464946404605F030F8049B42464146BC
:109C50002046CDE90096FFF7CDF929462046FFF7CB
:109C60008BF92B6801332B6020B1DAF80030013317
:109C7000CAF80030013FDDF81880002FB4D101236D
:109C80002B60022301276B71BB45DDF8189006D2CB
:109C9000484605F054FA079805F051FA80E72B681A
:109CA0009F4252D3582394F8B820DDF81CA003FB40
:109CB0000242516AFB0051F83700126D04900868A7
:109CC000083BC9580390D0581368A0EB03082B79C0
:109CD000012B38D1039B3246C91A4846059104F03E
:109CE000E4FF059943464A460091204651460196B5
:109CF000FFF780F929462046FFF73EF902232B7132
:109D000018B1164A13680133136032464146504673
:109D100004F0CBFFDDE9032349469B1A2046524657
:109D2000CDE90086FFF766F929462046FFF724F9BA
:109D30002B6801332B6001232B7130B1074A136864
:109D40000133136001E0022BDFD001379CE700BF35
:109D5000A1120100CA120100F9120100902800208E
:109D6000080000000A4619B1024B00211B68184781
:109D7000704700BF0C000020BFF36F8F72B6002346
:109D80004FF0FF30094A03F120010133102B42F854
:109D90002100F8D100234FF0FF30044A03F16001A5
:109DA0000133102B42F82100F8D1704700E100E0A8
:109DB000002318460649D1F89020C2F307229342A7
:109DC00000DB7047C1F89830C1F8A0000133F6E716
:109DD00000ED00E02DE9F8434FF0FF3501274FF08B
:109DE0000008204BDFF880905F60C3F84853C3F849
:109DF000085303F580535F60C3F84853C3F8085312
:109E000059F8044B002644F30730C4F8085300F017
:109E100021FF80226760C4F84C61D4F84C31C4F84B
:109E20001061D4F81031C4F844613146D4F844319B
:109E3000A018C4F8006505F053FA8022314604F5F5
:109E4000C07005F04DFAB8F1000F08D0074BC3F809
:109E500008554FF05023C3F80853BDE8F8834FF07E
:109E60000108CDE700400150880A01000070015050
:109E7000014B1B68184700BF1000002007B50B46B8
:109E8000002102460091034800F00CF803B05DF891
:109E900004FB00BF719E0000014B1860704700BFBB
:109EA000100000202DE9F04F82464FF000098DB0E0
:109EB0001D46531E01910393039B58785C1C252873
:109EC00019D100204FF0FF381E46444603460236A3
:109ED000029031780396392955D81F2914D80029C2
:109EE00000F0EF8101992520D04701993078D047C3
:109EF00009F10209E0E7002800F0E3810199D04769
:109F000009F101090394D7E7A1F12002192AE9D840
:109F100001A757F822F000BF819F0000E59E0000D6
:109F2000E59E0000819F0000E59E000001A000006A
:109F3000E59E0000E59E0000E59E0000E59E000015
:109F40004DA00000819F0000E59E000061A0000080
:109F50000DA00000E59E00001BA000003BA000003B
:109F60003BA000003BA000003BA000003BA0000085
:109F70003BA000003BA000003BA000003BA0000075
:109F800008460136A5E7582900F0EB80A1F16302ED
:109F9000D7B2172FA6D8172AA4D801A757F822F0AE
:109FA00009A2000087A00000E59E0000E59E0000D9
:109FB000E59E000067A0000087A00000E59E00006D
:109FC000E59E000067A00000E59E0000E59E000001
:109FD000E59E00003DA10000E59E0000E59E00001A
:109FE000DDA10000E59E000087A00000E59E0000C6
:109FF000E59E00003DA10000E59E000067A0000076
:10A0000025200199D04709F1010955E7029A4FF03F
:10A01000000802F0FE020292B3E7002C0DDAB8F15C
:10A02000000F0DDA029A002A00F043810A2224EA86
:10A03000E47402FB0414303CA3E7B8F1000FF5DB35
:10A040000A2202FB0812A2F130089AE7B8F1000FC9
:10A0500055F8042B80F22F81002A80F22E81544281
:10A06000022202928DE7682903D1682B06D148238A
:10A0700087E76C2902D16C2B00F02181002B7FF443
:10A0800031AF0B467DE77A2B06D1752955F8046B65
:10A0900014D14FF0000B0CE06C2BF6D04C2BF4D10C
:10A0A000073525F00703752903F10805D3E9006B8F
:10A0B00006D120283BD1854F013C09E04FEAE67BE1
:10A0C000BBF1000FF5DA7642814F6BEB4B0B013C95
:10A0D0000DF12D03059300230493304659460A22BF
:10A0E0000023FEF7D3F9059BB446303203F8012D67
:10A0F0005A460593049BBCF10A0F8B4672F100028D
:10A1000003F1FF3106460491E7D2C3F1010B30336E
:10A110000DEB0306B8F1000FA6F104066DDA029B01
:10A12000D9077DD4A8EB0B03A4EB0B0413E02B2879
:10A130000ABF684F684F04F1FF34C9E770290FD197
:10A1400055F8042B0023FAB96FF004034FF0050B08
:10A15000614F624E053C029A920770D4A04666E0B9
:10A1600078216C2B03D1002355F8042B08E04C2BED
:10A17000F9D1073525F007031D465B6855F8082B14
:10A18000232825D1880621D5554F023C002601F011
:10A190006001A1F1390B0DF12D0E02F00F0109291B
:10A1A00088BF594430310EF8011D102A4FEA1211B0
:10A1B00041EA03714FEA131C73F1000306F1FF300B
:10A1C00008D2C6F1010B06F13003A1E7454FDCE7E9
:10A1D000414FDBE706460A466346DEE755F8046B67
:10A1E000304605F05BF8B8F1000F834602DB4045CE
:10A1F000A8BFC3464FF00008374FA8EB0B03002B56
:10A2000092DDA4EB0804A6E755F8043B4FF0010BE0
:10A210008DF81830304F4FF0FF33013C06AE9AE70F
:10A22000A046EAE7029320200199D047029BB8F1AB
:10A230000108F7D524EAE472013C9144A41AB84617
:10A2400006E0049302920199D047029A049B90463B
:10A25000424612F8010B0028F3D11A46013A15D5EF
:10A26000002BACBFC7EB03077F425B46013B15D514
:10A27000BBF1000FA8BF5F4426464F44013E14D5F2
:10A28000002CA8BF3F1907EB080915E604930292BA
:10A2900030200199D047049B029ADFE7029301998D
:10A2A00016F8010BD047029BE0E701992020D04728
:10A2B000E4E70122D5E6904663E6144661E64C23C6
:10A2C0005FE648460DB0BDE8F08F00BF8713010080
:10A2D000851301008913010073150100911301001A
:10A2E0008B1301008E130100044608B5EFF31183B0
:10A2F000202383F31288BFF36F8F02F00BF8204600
:10A3000000F0EEFB024804F01EFE04F0ABFFFCE799
:10A31000971301002DE9F047058B04462807904666
:10A3200011D4022905F0070540F0CC80204604F046
:10A3300021FE78B10138218B042811D8DFE800F024
:10A34000C2106D85950001290CBF45F0100545F040
:10A350002005258388F31188BFF36F8FBDE8F08750
:10A3600001F0070AAA4500F0A5800027B9463E463D
:10A37000A368002B00F0BC8041F00801218388F322
:10A380001188BFF36F8FA168002900F0BA800D68B3
:10A39000002900F0B680334652462046D1F80480AA
:10A3A000C047002D76D02B6829461D46F0E701F006
:10A3B00007035A1F012A1BD8002221F00701062B90
:10A3C000276889B2C4E9002209D13B4603E0628BC9
:10A3D000013262831B68002BF9D141F00201204653
:10A3E000218304F0C7FD00287AD041F0200176E0F7
:10A3F000042B0AD121F0070189B22046218304F001
:10A40000B9FD10B141F020012183218B01F0070A31
:10A41000AA454FD00027B946AAE7236921F00701D2
:10A4200041F00601062DD3F8009021832DD1B9F11A
:10A43000000F3FD041F00801218388F31188BFF35A
:10A440006F8F20463949C84729E021F00701236969
:10A4500041F0040189B2042DD3F804902183E6D0A1
:10A4600000274FF0040A3E4682E721F007012369E6
:10A4700041F0050189B2052DD3F808902183D6D08B
:10A4800000274FF0050A3E4672E700274FF0060A04
:10A490003E466DE72B4687E7B9F1000FD1D1EFF3C8
:10A4A0001188202383F31288BFF36F8F238B23F04F
:10A4B00008032383258BEA062ED525F0100323837A
:10A4C00005F007056669218B002EBFF670AF0023EB
:10A4D0002768C4E9003321F0070141F0010121831D
:10A4E000218B4FF0000901F0070AAA457FF440AF25
:10A4F000002F9CD041F00801218388F31188BFF31D
:10A500006F8F002FC8D03D683946334652462046EB
:10A5100004F05CFD2F46F4E7AB067FF51BAF25F09A
:10A520002003238305F0070500E700BFF9EF0000D3
:10A5300070B5114B0D461C68DCB1104B1968002337
:10A540008B4202DB6FF0010070BD224612F8106BE7
:10A55000864202D014460133F2E7E06810B96FF08A
:10A560001200F1E705F060FF0028F8D000202C6011
:10A57000EAE76FF00C00E7E714000020900A010002
:10A5800070B588B005460C46C0B269461646FFF75E
:10A59000CFFF00281BDB0098C8B1436822680293F4
:10A5A00083680195CDE903360023CDE906230593A1
:10A5B000C56804F0C4FD6DB12846084901AA05F03C
:10A5C000A4FA079808B9059B236008B070BD6FF026
:10A5D0001500FAE76FF01200F7E700BFD9F10000AD
:10A5E00008B5054804F0AFFC044804F0ACFCBDE835
:10A5F0000840034804F0A7BCC0130100F813010091
:10A600002B140100014803F0EFBF00BF140C010040
:10A6100038B5044618B90F4B0F485B689847616816
:10A62000B1F5683F10D0B1F5680F0DD00B4DA942C0
:10A630000AD011F46861206807D00146084805F087
:10A6400049FF00232360656038BD142204F048FEF2
:10A65000F9E700BF4C010020591401002C5F5CA9F0
:10A66000942D002008B500B34368B3F5683F0CD1C2
:10A6700001220368D3E8EF1F002903D1C3E8E02FCC
:10A680000028F7D10DD1002008BD094A93420AD015
:10A6900000684FF0FF324FF0FF3303F08DF90028D0
:10A6A000F1D00448F0E70448EEE76FF4E040EBE750
:10A6B0002C5F5CA9E98FFFFFEA8FFFFF08B5B8B1F7
:10A6C0004368B3F5683F0CD100220368D3E8EF1F5D
:10A6D000012903D1C3E8E02F0028F7D10BD10020D6
:10A6E00008BD074A934208D0006803F0DDF9F6E799
:10A6F0006FF4E040F4E70348F2E70348F0E700BFF7
:10A700002C5F5CA9E98FFFFFEA8FFFFF10B50446BD
:10A7100018B91D4B1D485B6898476368B3F5683FDF
:10A720002FD0B3F5680F2CD0194A934219D1236862
:10A7300003BB4FF0FF324FF0FF332146154803F0C3
:10A740000DF908B923681BB90F4B13485B6898478C
:10A7500014220021206804F0C3FD4FF46863636095
:10A7600008E0B3F5683F0DD83A2B03D040F6BA6243
:10A770009342DED1206805F0E5FE636843F03A03BA
:10A78000636010BD054AF3E74C0100205914010035
:10A790002C5F5CA9942D00207F1401003A00003A40
:10A7A00008B5064940231422054805F085FEBDE89A
:10A7B00008400449044803F089BF00BF94280020E2
:10A7C000942D00201C0C0100300C010030BFFFF75D
:10A7D000FDBF00BF074A936893F90E10002907DBFD
:10A7E000526993421FBF044A536843F08053536039
:10A7F000704700BF942E002000ED00E0154B9A6AD0
:10A8000012F0007F9A6A14BF1E201D2012F0807F74
:10A810009A6A18BF1F2012F4801F9A6A18BF02207C
:10A8200012F4002F9A6A18BF212012F4802F9A6A1E
:10A8300018BF222012F4003F9A6A18BF232012F496
:10A84000803F9A6A18BF24206FEA02426FEA1242E0
:10A850009A62704700ED00E010B5194B0246986A05
:10A860009C6A10F4805F14BF1720162014F4006F48
:10A870009C6A18BF1820A40509D5986B986A000433
:10A8800004D51AB19A6A22F400429A6219200C4B3C
:10A890009A6A12F4806F9A6A18BF1A20D2050CD4F3
:10A8A0009B6A13F4005F18BF1C20054A936A43F4A7
:10A8B0007F43936200230B7010BD1B20F5E700BFA0
:10A8C00000ED00E010B51C4B0246986A9C6A10F03F
:10A8D000100F14BF1120102014F0080F9C6A18BF2D
:10A8E0001220A40709D5586B986A000604D51AB13E
:10A8F0009A6A22F080029A6213200F4B9A6A12F031
:10A90000010F9A6A18BF142012F0200F9A6A18BF1C
:10A910001520D40658BF9B6A074B9A6A920642BF1D
:10A920005A6A22F400525A629A6A42F0FF029A620C
:10A9300000230B7010BD00BF00ED00E070B5444B6C
:10A9400006465B6800258AB0C3F3080385F31188C7
:10A95000BFF36F8F02F07F40B0F17F4F11D102F053
:10A960000C0008280DD010074CBF0E460125002210
:10A97000033B8DF80720032B05D8DFE803F01E5CAE
:10A9800060592E46F3E700249DF807309BB920223A
:10A99000314602A804F099FC099B002D53D0C3F363
:10A9A000080222B96FEA53236FEA43230993204632
:10A9B00002A904F037FC0AB070BD254BDA6A910792
:10A9C000E1D4DA6A002ADEDBDA6A5200DBD55A69A2
:10A9D000B16942F480725A61BFF34F8FBFF36F8F3A
:10A9E0005A6931F8021C22F480725A61BFF34F8F0A
:10A9F000BFF36F8F4DF60272914209D09A6AD2B2BC
:10AA000042B101200DF10701FFF75CFF0446BBE7EF
:10AA10003468B9E79A6A12F47F4F05D001200DF12E
:10AA20000701FFF719FFF1E79B6AB3F5803FAAD34F
:10AA3000FFF7E4FEEAE700200DF10701E4E700205C
:10AA40000DF10701EDE723F4FF7323F00103ADE7F8
:10AA500000ED00E0044B5A6942F010025A615A6955
:10AA600042F480625A61704700ED00E0EFF3088025
:10AA7000EFF3098101B57246FFF760FF01BD00BF2A
:10AA8000002080F31488BFF36F8F002080F30A88C2
:10AA900080F30B8801F028FE00200E490860BFF308
:10AAA0004F8F0D4880F3088800F02CF8202080F3A9
:10AAB00011880A484FF40061401880F30988EFF3C9
:10AAC00014800221084380F31488BFF36F8F00F0D5
:10AAD000F9F8000094ED00E0F8420020B8310020C1
:10AAE000BFF34F8F0549064BCA6802F4E062134377
:10AAF000CB60BFF34F8F00BFFDE700BF00ED00E06C
:10AB00000400FA0572B6002383F313884FF0FF3078
:10AB10000C4A03F120010133102B42F82100F8D137
:10AB200000234FF0FF30074A03F160010133102B7F
:10AB300042F82100F8D162B6BFF34F8FBFF36F8F99
:10AB4000704700BF00E100E0084B9B6883420BD1D7
:10AB5000EFF3058343B1064B5A6842F080525A60C6
:10AB60005A6A22F400425A6205F0AABD942E0020CF
:10AB700000ED00E06FF00A01084A93689967084900
:10AB800058674B6843F080534B60002383F3118870
:10AB9000BFF36F8F9368986F704700BF942E0020AB
:10ABA00000ED00E0EFF31183202383F31288BFF35D
:10ABB0006F8F4FF00061064A53699360054A5160F8
:10ABC00000215A6F596782F31188BFF36F8F704766
:10ABD000942E002000ED00E00E498A684FF030000E
:10ABE0001044EFF3098C80E8F01F74467046FFF7BD
:10ABF000D9FFA64607498A6802F1300090E8F01FA5
:10AC00008CF3098802F1000004B504F020FBBDE8D4
:10AC100004407047942E00201EF0040F0CBFEFF389
:10AC20000880EFF30980816911F8021C0229FFD026
:10AC300001B504F0FDFA01BD40B2002807DB012395
:10AC40004109034A00F01F00834042F82130704759
:10AC500000E100E040B200280CDB01220649430974
:10AC600000F01F008240203341F82320BFF34F8FB4
:10AC7000BFF36F8F704700BF00E100E0054B420952
:10AC800053F82220012300F01F0003FA00F01040C7
:10AC9000704700BF00E100E040B2002801F101016F
:10ACA000ACBF00F16040064B4FEA4111C9B2ABBFE7
:10ACB00000F5614000F00F0080F800131954704750
:10ACC00014ED00E00B4A08B50B4B22F07F029A60AE
:10ACD000BFF34F8FBFF36F8FD3F8882022F4700239
:10ACE000C3F8882002F07EFD03F0DCFA00F046F89D
:10ACF00002F0B8FD0082000000ED00E042F8203CC8
:10AD0000009B0B4942F81C3C019B21F0010142F8D9
:10AD1000183C029B42F8081C42F8143C4FF0807328
:10AD200042F8043C0023203A02654367704700BFA5
:10AD300061EF00000B4B0E4698601546436E83F39F
:10AD40000B882C4686F309884FF00000064B984785
:10AD500020464FF000014FF000024FF00003034C7B
:10AD6000204700BF942E002057F2000061EF000042
:10AD70001022014B1A61704700ED00E000232021F2
:10AD80000348C2180133412B82F80013F9D17047F0
:10AD900000E100E008B5EFF30583064A103B02EB43
:10ADA000C30152F8330049688847BDE80840FFF7FF
:10ADB00011BD00BF40080100014B1860704700BF83
:10ADC000380000200122024B0020C3F840257047C4
:10ADD0000090035020B1034B800143F0010318475A
:10ADE000704700BF700A0100084B70B5C31A0D46CA
:10ADF00007499B10044659434022064804F085FA4F
:10AE00002B4601462046BDE870401847C42D00205F
:10AE1000B76DDBB6B4070100402373B50B4C00934C
:10AE2000041B0B460D460A49A41061430646094A15
:10AE3000094804F095FA011E05DA30462B4602B0A7
:10AE4000BDE87040184702B070BD00BFC42D00209F
:10AE5000B76DDBB6C9F30000B407010010B5EFF31E
:10AE60001184202383F31288BFF36F8F074A13687E
:10AE700023F00201DB07116002D4012005F0FCF988
:10AE800084F31188BFF36F8F10BD00BF142E002014
:10AE900070B50022012104460520FFF7FDFE0F4892
:10AEA00001F01AFD0E4B984215D101F025FD2669DF
:10AEB0000C49304604F0ADF800280BDB0125356461
:10AEC0002469084904F11C0004F0A3F8002801DB00
:10AED0000020E56470BD6FF00400FBE7E1AF000007
:10AEE0000000AD0B400C01001FB500220123CDE98D
:10AEF00002236B46084ACDF800D0CDF804D004F008
:10AF00005CFA002805DB4FF480420023684602F01B
:10AF10002BFE05B05DF804FBE7F300000C22104B9C
:10AF2000014602FB0033002030B4D3E90E5298638F
:10AF3000EFF31180202484F31288BFF36F8F1C6C11
:10AF400004F0C00444F002041C6480F31188BFF3D1
:10AF50006F8F1DB12B4630BC0248184730BC70477C
:10AF6000C42D0020B407010010B4EFF31182202398
:10AF700083F31288BFF36F8F1748016841F0020412
:10AF80000460C80707D482F31188BFF36F8F0120D4
:10AF900010BC01F0C5BC4FF05021D1F80C04D1F821
:10AFA0000C14C907EFD5EFF3118083F31288BFF3B8
:10AFB0006F8F0A490B6C03F0C00343F002030B646C
:10AFC00080F31188BFF36F8F82F31188BFF36F8F07
:10AFD000002010BCFFF7A2BF142E0020C42D0020BB
:10AFE00010B1012804D07047034B1B6C5B0701D1E3
:10AFF000FFF794BF704700BFC42D00202DE9F0413A
:10B00000012207463649D1E8EF3FC1E8E02F00288A
:10B01000F9D133B9334934484B60CB608A6004F0CE
:10B020000BF87B1E012B2BD8012F07D14FF050239B
:10B03000D3F81C3403F00303022B21D005F095FA5A
:10B040000546F8B9294B1B78E3B14FF05023022293
:10B050000646C3F808234FF05024DFF89480D4F854
:10B060001824D4F81834D20315D503F00303022BA7
:10B0700001D0012F0FD16DB386F31188BFF36F8F0D
:10B08000BDE8F081EFF31186202383F31288BFF32C
:10B090006F8F0125DFE7C5B1304604F0F0F8D4F832
:10B0A0001835DBB2012BDAD1D4F80421002AD6D02E
:10B0B0000022C4F80421D4F804210222C4F818257F
:10B0C0002022C8F88021A360C9E70021212003F0D5
:10B0D0003FF8E4E74FF050230222C3F80423CFE700
:10B0E000C02D0020B02D0020E02D0020B231002026
:10B0F00000E100E008B5074805F096F938B10648C8
:10B10000FFF75AFE0448FEF7C7FE002008BD6FF0A7
:10B110001200FBE7F00701001DB100000A2838B556
:10B120000446074D04D1AB680D2128465B6898475B
:10B13000AB6803485B68E1B29847204638BD00BF62
:10B14000F0070100004870470C0D0100024B0B6036
:10B1500001231360704700BF382E0020004870475D
:10B16000280D010010B501220648114605F0F1F93D
:10B1700005F0E9F8044C206005F0E2F8606000207A
:10B1800010BD00BF402E0020382E002070B50C46A8
:10B19000154605F0D5F829460646204604F05BFC26
:10B1A00008B3B4FBF6F306FB1343E3B9B5FBF6F3C0
:10B1B00006FB1353BBB9AE4201D9002070BD4FF05E
:10B1C000FF324FF0FF33094802F0CEFC05F0B8F82B
:10B1D0000646204601F0C4FFAD1B3444F9D10348B4
:10B1E00002F09EFCE9E76FF01500E7E7402E002033
:10B1F000F8B50E461946304617461C4604F02BFC9F
:10B2000008B344EA060515F003051CD1A4B14FF0BC
:10B21000FF324FF0FF330D4802F0A6FC24F0030488
:10B22000A54206EB050009D1094AD2F80034DB0734
:10B23000FBD5064802F074FC0020F8BD795901F0F6
:10B24000ADFF0435ECE76FF01500F6E7402E002067
:10B2500000900350C3780F2B14D9C96B0B480B0E09
:10B2600013708B0200EA911003F47C030906034378
:10B2700001F0FE4110680B43054901400B430020DB
:10B28000136070476FF08500704700BF00FF030038
:10B29000FF00008038B545682B69B3B110352846EA
:10B2A00001F03AFE044680B90146284601F002FE4C
:10B2B000084B98420BD122462846074901F0E2FD8F
:10B2C000224605210D20FFF7E7FC002038BD6FF076
:10B2D0000400FBE70000AD0BDDB20000430970B5D0
:10B2E00007D10B4B596821B101250C68094E8540E7
:10B2F00001B970BD8A682A4002D030464B68984731
:10B300001CB1236821461C46F2E72346FAE700BF3A
:10B31000502E0020C80701002DE9F04340F2063509
:10B320004668D00648BF0320337B02EA050558BFB4
:10B33000C2F3401087B001F01F07B5F5837F1446B4
:10B3400047EA43178DF8030041D00FD8062D18D0D7
:10B3500007D8B5B1022D3CD06FF0150007B0BDE89D
:10B36000F083B5F5807FF7D101250AE040F2022293
:10B37000954230D0B5F5407F2FD0B5F5007FEBD1A9
:10B38000022522032BD5012372688B40936032691A
:10B3900062BB07F01F037F0975D13D4A84F48031F9
:10B3A00002EB8302D2F80032C1F30041C4F34044FF
:10B3B00023F4E16344EA410423F007031C4344EA15
:10B3C000800444EA0524C2F800420020C6E70725AD
:10B3D000D7E70425D5E70525D3E70325D1E76303A0
:10B3E00041BF012372688B40D360D0E710363946E5
:10B3F00030460DF1020201F04BFD14F4403F80464F
:10B400000CD13946304604F091FF224B9845DCD1EF
:10B4100030469DF8021001F089FDD6E74FF0000993
:10B4200001AB3946304603AACDE90439CDE901998B
:10B43000CDF80C9001F000FC164B98428CD114F41E
:10B44000003315D09DF8033084F48034C4F30044F5
:10B450008DF80E3039464B46304603AA8DF80C5015
:10B460008DF80D4001F096FC0A4B9842CDD073E761
:10B47000CDE9043339460DF10303304603AA0393A3
:10B4800001F0DAFBF0E7803352F82330FFDE00BF33
:10B49000002584500000AD0BF0B5406801F01F049A
:10B4A000057B87B044EA45140569002D5FD0B2F5ED
:10B4B000001F00F1100506D12146284604F038FF90
:10B4C000002007B0F0BD0027B2F5800F01AE019754
:10B4D000776037D1B3F1007F14BF052304238DF8C3
:10B4E00004300023CDE904630393836823FA01F158
:10B4F00011F0010118D1B2F1A07F15D104F01F03A2
:10B50000620903F1800338D11D4A52F82330DB076A
:10B510000AD40DF1030632462146284601F0B8FC54
:10B52000184B984219D002962146284603AA01F0EA
:10B5300083FB154B98421DD101222146284601F07C
:10B5400001FDBDE7B3F1C06F05D0B3F1007F14BFBB
:10B5500001230223C3E70323C1E73146284601F054
:10B56000EBFC094B9842DED06FF00B00A9E76FF0BF
:10B570008500A6E76FF01500A3E751F82330FFDE42
:10B58000002584500400AD0B0000AD0B2DE9F04701
:10B5900040F2FF16594FDFF868C1DFF868E100EBB1
:10B5A0008101814202D10020BDE8F087046814F4D3
:10B5B000804FC4F3C325C4F3080340F08C80640CAF
:10B5C000B34208BF4FF0FF337D5D192C00F2868037
:10B5D000DFE804F00D13191C1F251C8484848436B5
:10B5E0006084848484848484848463787B7EC2F8C9
:10B5F0000C355C1C5BD10430D3E7C2F814355C1CFD
:10B60000F9D000245CE0C2F80835F2E7C2F8103542
:10B61000F5E75C1CC2F80835EDD0002404E05C1CA2
:10B62000C2F80C35E7D001245FEA531859D14FF026
:10B630000109DFF8CC8009FA03FAC8F80CA008E089
:10B64000C2F80835002DDAD15C1CD4D000240625C0
:10B65000A146D0F800A00AF40048B8F1000F1CBFC2
:10B660004FF00009012403F01F085B093FD10CEBE8
:10B670008808D8F80032CAF3412A03EA0E0343EAE5
:10B680008A0343EA052343EA090343EA4403C8F86B
:10B690000032B0E7C2F80C35D4E7C2F86035B3F138
:10B6A000FF3F0468A7D0C4F30044002CBBD05C0962
:10B6B0001AD10124DFF8488004FA03F9C8F8089089
:10B6C000A146C6E7C2F86435E9E7C2F86835E6E79F
:10B6D000C2F86C35E3E76FF0150065E76FF08500A1
:10B6E00062E70023DB60FFDE00239B60FBE70023B3
:10B6F00008F1800853F82830F5E700BFF314010083
:10B7000000258450F0F8FCFF2DE9F7434FF00008C6
:10B71000476805693C680646C4F800852860D7F884
:10B720000C904146484601AA04F07BFA00283CDB15
:10B73000019BD9F8002019791868FFF727FF002826
:10B7400033DB6B7A3169012B03D0032B2BD14FF004
:10B750001008AB7A032B26D195F80BC0BCF1000F73
:10B7600002D0BCF1010F1ED12A7A12B1022A1AD1DD
:10B770000E226B687068B3F5164F006800F0B28057
:10B7800034D8B3F5165F00F0B0801AD8B3F5966FD1
:10B7900000F0AD800CD8B3F5967F00F0AB80B3F528
:10B7A000167F00F0AA806FF0850003B0BDE8F0833B
:10B7B000B3F5166F00F0A480B3F5965FF3D15C4B40
:10B7C00043E0B3F5E14F00F09E8008D8B3F5615F28
:10B7D00000F09B80B3F5964FE5D1564B35E047F628
:10B7E000122E7345DFD14FF400032EE0B3F5613F15
:10B7F00000F08D8015D8B3F5963F00F08B800AD805
:10B800004DF6C02E734500F08780B3F5614FCAD165
:10B810004FF46B0319E0B3F5E13FC4D14FF0EB7384
:10B8200013E0B3F5612F7AD009D8DFF80CE1734546
:10B8300078D0B3F5E12FB6D14FF0E86305E0DFF83B
:10B84000FCE07345AFD14FF08053C0F824357368E6
:10B8500048EA0C081B6842EA0802C3F86C250B1D75
:10B86000D5E9010183E803007B68990712D505F14A
:10B87000180001F0DFF8324B984256D1287E04F1CF
:10B880000C0204F5907104F097FC01202B7E984087
:10B8900001F01CF80823C4F800353B7A53B9C4F80A
:10B8A0001031D4F810316B69C4F834350123C4F871
:10B8B000383523607B6800209A075CBF4FF48073A3
:10B8C000C4F804337B68DB0644BF4FF48003C4F83C
:10B8D00004332B69C4F844350123C4F84805A36038
:10B8E000E36062E74FF41D03AFE7164BADE74FF49B
:10B8F0009E23AAE74FF4A033A7E74FF41C33A4E735
:10B900004FF41D23A1E7104B9FE7104B9DE74FF02D
:10B910006C739AE70E4B98E74FF4650395E74FF089
:10B92000706392E74FF080638FE76FF004003CE7AD
:10B9300000B0130000A04E0090D0030040420F0062
:10B940000000AD0B0050270000C0750000F03A0069
:10B9500000903A012DE9F04104460D46076904F0D4
:10B9600004FE4FF02008B0B92C4B1B789BB1642625
:10B97000606804F084F9F0B9012004F01BFC013E7A
:10B98000F6D10021212002F0E3FBF0E786F31188D5
:10B99000BFF36F8FF5E7EFF31186314688F3128816
:10B9A000BFF36F8F606804F06AF980B986F311887D
:10B9B000BFF36F8FEFE7EFF31186314688F31288FC
:10B9C000BFF36F8F606804F05AF90028DED03B693E
:10B9D0001D70626838691368C3F844050120C3F814
:10B9E00048050020C3F82001D3F82051C3F85801BE
:10B9F0005268D3F85801D20608D508206268126848
:10BA0000C2F800054FF48002C3F8042301229A60B3
:10BA100081F31188BFF36F8FBDE8F081B231002050
:10BA20002DE9FF4105690646D0F80480A86C2B6D0E
:10BA3000002835D1002B53D0B8F830406A6C9C42B6
:10BA400028BF1C46EF6CEB6C53B1296D41B107F078
:10BA50006041B1F1005F03D0082C28BF08246F6E4D
:10BA600000926A6CAC651AB1AA6C002A18BF224613
:10BA7000CDE901271BB12B6D002B18BF23460022F7
:10BA800069464046039301F041FD184B984229D086
:10BA90006FF00401304604B0BDE8F04104F025BA6F
:10BAA000696CEF6C0A46B8F83040ABB1834228BFEE
:10BAB00003469C4228BF1C460029C4D001F06043C5
:10BAC000B3F1005FBFD0082C28BF0824286E22469F
:10BAD00003F0FBFB2A6EB6E7844228BF0446EBE77F
:10BAE0001946D7E704B0BDE8F08100BF0000AD0BF8
:10BAF0002DE9F04F984643688DB001938B880F462F
:10BB0000990405469146046900F10E814FF0FF3219
:10BB10004FF0FF3304F1100002F026F86760D5F80B
:10BB200004B0D5F810A0DBF8083003939AF85D3024
:10BB30001BB1DAF800309F427AD0B7F804E01EF467
:10BB4000006F40F01E811EF0090F40F01781CEF308
:10BB50004513082B40F012813B680293029AA04BD8
:10BB60009A4240F20B8104AE0BF10C0CBCE80F00C2
:10BB70000FC69CE80F0086E80F00DDE902329A420A
:10BB800028BF1A46974B9A4215D2974B9A4200F219
:10BB9000D480964B9A4200F2D280954B9A4200F2A2
:10BBA000D080944B9A4200F2CE809348934B9449B4
:10BBB000824288BF0B461EF0020F09930EF0040369
:10BBC00000F0C380002B14BF032302238DF828301C
:10BBD000CEF300138DF82930DBF800301EF0020F91
:10BBE000D3F8082587484FF00103CEF340014FEA10
:10BBF000521640F0AE80002E40F0ED809340C360BE
:10BC00009AF85D302BB1584601F044FC00238AF8C5
:10BC10005D302B4658467C4A04A901F007FC7B4B5B
:10BC2000984240F09B800123CAF800708AF85D308A
:10BC3000012384F85C30019B996B4A1C03D003F10B
:10BC40003C0000F01DF9B9F1000F40F09D80C4F8F0
:10BC500034900023A36304F1480204F1380104F195
:10BC6000340004F076F86064B8F1000F40F095807D
:10BC7000C4F83C800023236404F1500204F1400125
:10BC800004F13C0004F065F8002601213246E0642E
:10BC90002663204604F084F82846FFF7C1FE3246AA
:10BCA0003346A06B834240F0818000231946266C06
:10BCB000B14240F08280934238BF134627464FF48A
:10BCC000FA524FF0000802FB03F657F8203B4FF4FE
:10BCD000004C1B684146B6FBF3F640F2E730C8362D
:10BCE0004FF47A720023E6FB0C01FCF7CFFB02460F
:10BCF0000B46384601F038FF024618B9266B16F19C
:10BD0000740F61D10198C4F8588001F0C3FB6FF043
:10BD10007301284684F85D8004F0E7F8384601F0A6
:10BD200049FF6FF073061BE0A369002B7FF4EEAEB2
:10BD300063689F427FF4EAAEF1E6354B3BE7354B53
:10BD400039E7354B37E7354B35E7003B18BF012363
:10BD50003CE7002E41D19340836051E76FF0040629
:10BD600023689B8813F4005304D1636004F110002E
:10BD700001F0D6FE30460DB0BDE8F08F6FF015062D
:10BD8000EEE76FF08506EBE7D9F800306363002B30
:10BD90003FF45FAFD9F804305CE7D8F80030E363D4
:10BDA000002B3FF467AFD8F8043064E7616B01EB18
:10BDB000C301496801330A4474E7E06B00EBC1003A
:10BDC00040680131034473E7002EC9D00146286959
:10BDD00003F0E6FFC4E7C960FFDE00239B60FBE7DA
:10BDE00047E8010000127A00FF083D007F841E0032
:10BDF0003F420F001FA107008FD0030048E8010059
:10BE000090D00300002584500DFF00000000AD0B12
:10BE100000093D0080841E0040420F0020A1070061
:10BE20000123F0B587B08DF80230022300248DF88D
:10BE300004306B4403930F4601AB0DF103010493EF
:10BE400005460291059401F077F80C4B064698429E
:10BE50000FD13946284603AA00F0EEFEB0420BD0BF
:10BE600028469DF8031001F061F86FF0040007B058
:10BE7000F0BD6FF01200FAE72046F8E70000AD0BC6
:10BE80002DE9F0410D46064604F054FA002207461B
:10BE90002946304601F056F86B0905F01F0429D1F8
:10BEA000174B03EB8404D4F80022164B134043F0E5
:10BEB0000C03C4F8003204F08EF880463368DB5976
:10BEC0007BB100273046294604F032FAD4F800222C
:10BED0000C4B3846134043F00403C4F80032BDE86D
:10BEE000F08104F078F8A0EB08000628E6D96FF09E
:10BEF0007307E7E70023803453F82430FFDE00BFE8
:10BF000000258450F0F8FCFF0123834070B5DC432A
:10BF10000B4AD2E8EF1F01EA0405C2E8E65F002EF3
:10BF2000F7D14FF4803282400648C0F80823BFF3AF
:10BF30005F8FBFF36F8F0B4214BF0120002070BDD5
:10BF4000602E00200050015070B40E4922F07F4650
:10BF5000D1E90034D01AC31844F10004C1E9003417
:10BF6000A6F50013B3F5400F09D2074B1B681A0A58
:10BF70001B069C19054B42F10005C3E9004570BC46
:10BF800002F06ABA20020020642E0020280200205D
:10BF9000D9B101230D4A8340D2E8EFCF4CEA030C1C
:10BFA000C2E8E1CF0029F7D14FF48033084A83403B
:10BFB000C2F80433074BD3E8AF3FC340DB0742BFAF
:10BFC0004FF40012044BC3F800217047602E00208C
:10BFD000005001505C2E002000E100E00D4B18687D
:10BFE000010A0006BFF35F8F0B4BD3F80435181816
:10BFF00041F10001B3F5801F0AD2084BD3E90023B9
:10C00000904271EB030303D210F1807041F1000103
:10C01000704700BF642E002000500150280200200D
:10C020002DE9F04F85B016461F4604469DF840A006
:10C03000FFF76AFF0190FFF7D1FFB04271EB0703F2
:10C0400052D23B4B301A67EB0101984271F100016B
:10C050004DD2384B03EB0413D3E902239F4208BFB0
:10C06000964258D04FF48038334908FA04F82046F5
:10C0700026F07F4BC1F8488303F0A1FF4FF003097E
:10C08000584604F15005AD00ADB205F1502504F558
:10C09000A87305F580350293029A20F07F4341F89A
:10C0A0002230C1F84483D1F80435244AC01A033839
:10C0B00020F07F4090422ED9286868B1D1F804352D
:10C0C000A3EB0B0020F07F40B0F5000F039322D9C3
:10C0D000204603F074FF039BBAF1000F07D109EB70
:10C0E000030009F10109D7E7BAF1000F09D06FF099
:10C0F000150520460199FFF74BFF284605B0BDE81E
:10C10000F08F01230E4AA340D2E8EF0F1843C2E894
:10C11000E10F0029F8D107490E982301C8500F9B61
:10C1200001EB04120025C2E902675360E1E700BF9A
:10C13000010080001002002000500150FDFF7F0030
:10C140005C2E00207FB500254FF0FF304FF0FF310F
:10C15000194C1A4B0226C4F80833C4F84833184B5C
:10C16000C4F80855C3E902014FF480334FF40012BC
:10C17000C4F80433134B0121C4F804631520C3F839
:10C1800080212A46FEF788FD1520FEF755FD012384
:10C190000D4AA360236013600C4B0D4A00932846A0
:10C1A0000023CDE90155FFF73BFF3046FEF726FFA0
:10C1B000284604B070BD00BF0050015003000F00BE
:10C1C0001002002000E100E0602E002049BF0000C6
:10C1D000FFFF7F002DE9F7432E4BD3F80423900790
:10C1E0000BD5D3F8042142B10022C3F804212A4A16
:10C1F000D3F80431136801331360264AD2F80433AC
:10C20000D90326D5254BD3E8EF1F21F00100C3E861
:10C21000E40F002CF7D1CB0702D4D2F84031C3B1E0
:10C2200000251C4CC4F84051D4F84031FFF7D6FE2D
:10C23000EFF31182202383F31288BFF36F8F184B23
:10C24000D3E90267B042B94106D282F31188BFF345
:10C250006F8F03B0BDE8F0834FF0FF38D3E90010D3
:10C260004FF0FF391D60C3E902894FF48033C4F8F1
:10C270004833C4F84051D4F8403182F31188BFF3F9
:10C280006F8F0029E5D0009032463B46284688470C
:10C29000DFE700BF00500150642E00205C2E00201C
:10C2A0001002002030B5431C124C85B005D08442EA
:10C2B000A8BF0446012CB8BF0124FFF78FFE0E4B28
:10C2C0000C4DD3E90013401AB0F5000F0FD222181D
:10C2D000AA4228BF2A46002052180849CDE9010089
:10C2E000009143F10003FFF79BFE05B030BD2A46E5
:10C2F000F1E700BFFFFF7F002002002049BF0000E0
:10C3000008B5FFF76BFE024B1B68C01A08BD00BFE3
:10C3100020020020012310B5074C15206360FEF7B2
:10C3200099FC4FF40012054BC4F80833C4F84833A5
:10C33000034BC3F8802110BD0050015003000F00D3
:10C3400000E100E040EA0103C3F30E0330B58BB90E
:10C3500040F21515094CC90BC0F3C730994201D101
:10C36000002030BDC218D2B202F5C07244F822508B
:10C370000133F3E76FF01500F3E700BF0030005022
:10C38000054B1B68DA6AB2F5807F01D8DB69184774
:10C390006FF00D00704700BFFC420020014B1B688E
:10C3A0001B6A1847FC420020014B1B685B6A184758
:10C3B000FC42002010B4034C2468E469A44610BC7D
:10C3C000604700BFF84200202DE9F043234885B0C4
:10C3D00003F005FE00250446204B214ED3F838809B
:10C3E000DFF88090A84503D8002005B0BDE8F083B1
:10C3F000636A96E807001F6801AB83E807000C2218
:10C400001946384602F051FF88B987B1636A21693D
:10C410001B681A6991420AD19A69A169914206D8AA
:10C42000E169914203D962695B699A430CD0276A3A
:10C4300077B10D4802F087FD002383F31188BFF325
:10C440006F8F0423184602DFE36801351C44C9E7F7
:10C45000484602F078FD636A1F60F5E7008400003B
:10C46000500A0100411501001815010030B581681E
:10C4700085B0103921F00704054602F0A6FE10220F
:10C480000146684602F02CFF10226846064902F079
:10C490001CFF10236A462146284602F066FE00383B
:10C4A00018BF012005B030BD180F010030B50D4692
:10C4B000816887B0102302AA1039044602F040FEBA
:10C4C000002802DA012007B030BD1022204602A960
:10C4D00003F0AFFD00283AD110221E4902A802F055
:10C4E000E4FE00280CBF012302232B70204603F03A
:10C4F0008CFD012301460DF10702204602F020FECB
:10C500000028DFDB9DF80730204603F00F021B09EF
:10C510006A702B7101220DF1070103F08AFD10B939
:10C520006B78042B03D901236B7000232B71A26855
:10C530002046183A22F00702083AA91C03F08CFDA5
:10C540000028BFD12046E91C03F0DFFDBBE7032331
:10C55000CBE700BF180F0100F0B585B0054669466E
:10C5600000284DD0012807D0FF2003F0D4FD00287B
:10C5700048D0FF2005B0F0BD324803F0CCFD0028C4
:10C58000F7D1022002A903F0C6FD01283CD12A46BA
:10C5900049212D4802F0C6FD2C4B029300238DF853
:10C5A0000C3000229DF800609DF80870284C314640
:10C5B000207803F030FD70B33946607803F02BFD2E
:10C5C00048B3A378042B03D09DF80310994222D1DD
:10C5D000E378042B03D09DF80B1099421BD12379EB
:10C5E000042B14D16279022A21D11A4B1A482A4607
:10C5F000492102F097FD6079831E022BBAD9B8E772
:10C600000D20BAE7FF20BDE70028CAD0B1E79DF8AA
:10C6100002109942E6D00132032A04F10604C6D181
:10C620000E482A46492102F07DFD0120A2E7032A97
:10C6300005D00B4B0B49042A08BF0B46D6E70A4B23
:10C64000D4E700BF080000009715010003010303B1
:10C650002C16010079150100E215010006160100F3
:10C660007E150100901501007415010008B5EFF367
:10C670001083012B0C4A07D1126ABFF34F8F511C54
:10C680004A424A41104608BD03F072FD00B172B63D
:10C69000126ABFF34F8F531C5A425A4103F068FD90
:10C6A0000028EFD062B6EDE70080FF0008B5EFF399
:10C6B0001083012B0B4A06D1D269BFF34F8F02F0D2
:10C6C0000102104608BD03F053FD00B172B6D269F5
:10C6D000BFF34F8F02F0010203F04AFD0028F0D0B3
:10C6E00062B6EEE70080FF0010B503F041FD30B107
:10C6F0004FF050230022C3F81421C3F8182103F08F
:10C7000046FD28B101224D4BC3F8382AC3F87825DD
:10C710004FF47F02D2F83031D2F83421BFF34F8F7B
:10C72000C3F30B03092B05D1012A1EBF0122434B82
:10C73000C3F8782503F02BFD18B10E22404BC3F847
:10C74000E42E03F015FD30B100223C4BC3F80C275A
:10C750000122C3F810270022D30003F57F03D3F88A
:10C760000013BFF34F8F013108D0D3F8001301320B
:10C77000D3F80433B2F5807F0B60EDD1EFF3108472
:10C78000FFF794FF00284DD0BFF34F8F2D4BD3F808
:10C790000024012AFBD1C3F80425D3F80024012A80
:10C7A000FBD1012C03D003F0E3FC00B172B6FFF71C
:10C7B0007DFF58B1244AD36923F00103D361BFF34D
:10C7C0004F8F204AD2F80034012BFBD1FFF74EFFE8
:10C7D00068B11D4A136A23F0FF0343F0200313627C
:10C7E000BFF34F8F174AD2F80034012BFBD1012C35
:10C7F00003D003F0BDFC00B162B60022114BC3F8B8
:10C800000425D3F80024012AFBD1BFF34F8F0F4931
:10C810000F4BCA6802F4E0621343CB60BFF34F8F43
:10C8200000BFFDE7FFF722FF0028ADD1074AD2F88D
:10C830008C3043F44063C2F88C3010BD004000508F
:10C8400000A00350009003500080FF0000ED00E0C6
:10C850000400FA0530B50468ACB1B4FA84F30122DF
:10C86000C3F11F03DBB29A4024EA0202D0E8EF5F73
:10C87000A54204D1C0E8EC2FBCF1000FF6D1EAD1FB
:10C8800002480B7030BD0248FCE700BF0000AD0B52
:10C890000200AD0B10B50368CB40DB0710D40123B9
:10C8A0008B40026843EA0201D0E8EF4F944204D182
:10C8B000C0E8EC1FBCF1000FF6D1F2D1014810BD69
:10C8C0000148FCE70000AD0B0400AD0B014BC3F8C1
:10C8D0000405704700700150044B1A7922B90122F7
:10C8E00018601A710248704702487047682E00208D
:10C8F0000000AD0B0C00AD0B08B5084B1B6833B145
:10C900000520FEF7BBF910B90520FEF795F94FF0A9
:10C9100050230122C3F8182508BD00BF682E00204F
:10C9200010B510B1012847D010BD4FF05023D3F8F7
:10C930001814D3F81824C90322D502F00303022BDC
:10C9400005D0012B02D0002003F03DFC01234FF065
:10C9500050220220C2F8183508224FF482730021B9
:10C9600003F1502319601C68012402F15022146065
:10C97000164A126822B34FF05023C3F80403D3E7DA
:10C98000D3F81424D207E1D5D3F81C2402F0030213
:10C99000013A012AD7D80D4A12681AB10222C3F807
:10C9A0000423C1E7D3F80421002AFBD00022C3F8F6
:10C9B0000421D3F80431B7E700224FF48073CEE7A7
:10C9C0001A68002AFCD019601B68ADE7682E0020A9
:10C9D0004FF0502310B5D3F8002152B10020C3F816
:10C9E0000001D3F800210122C3F80823104B1B6873
:10C9F00098474FF05023D3F8042182B10022C3F8A6
:10CA00000421D3F80421D3F81824D3F818240221E0
:10CA100002F00302012A03D1C3F818159A6010BD71
:10CA2000C3F80813024B0120BDE810401B681847EB
:10CA3000682E002001460148FFF70CBFDC000020F3
:10CA4000036803F01F025B090260024818BF002060
:10CA5000704700BF0025845070B50D4C00F10803ED
:10CA600034F813300546DA050E4607D5C3F34323E1
:10CA700004EBC302526854F833309847A3682BB1D3
:10CA800031462846E268BDE87040184770BD00BFD7
:10CA9000E0000020024611F0010004D003490B6AB7
:10CAA00013600B6203B90020704700BF002584505B
:10CAB00010B4124AC0B2083032F81030D9051BD574
:10CAC000C3F3432123F4F85322F81030002002F17D
:10CAD0000E0434F8023F13F4807F03D0C3F34323E2
:10CAE000994209D001302028F3D1002342F8313097
:10CAF000034810BCFFF7CEBE10BC7047E00000201A
:10CB000038010020F0B505460020012604460746FE
:10CB10008C420BD1114BD3F87C2132B10022C3F8E7
:10CB20007C21D3F87C3140F00040F0BDE3B29B00A3
:10CB300003F580729B0806FA03F31D420BD002F145
:10CB4000A04202F55042D2F800C0BCF1000F02D062
:10CB50001760126818430134DAE700BF00D00050B4
:10CB6000064BC0B2083033F81000830643BF400BB9
:10CB7000800000F580704FF4BE707047E000002028
:10CB8000CBB2024608460D49083331F813309906F6
:10CB900011D599070FD4012110685B0B9940C0F89B
:10CBA0000813126802EB8303D3F8102522F0030266
:10CBB000C3F810257047002103F0A9BBE000002056
:10CBC000F7B5194ECDB2083536F815300746DB07F4
:10CBD0000C4626D5FFF7D4FF36F815309A0608D54F
:10CBE0005A0B3B6803EB82030022C3F81025C3F8FD
:10CBF00010252046FFF75CFF002301A826F815301A
:10CC00000194FFF71DFF019B00EB8300D0F8002289
:10CC1000064B134043F00203C0F80032044803B04F
:10CC2000F0BD0448FBE700BFE0000020F0F8FCFF87
:10CC30000000AD0B0400AD0B2DE9FF411368074662
:10CC40000C461646FBB1DFF83C81CDB2083538F80A
:10CC5000152002F02202222A22D000222046CDE90D
:10CC600000228DF80E208DF80F200DF10E010DF130
:10CC70000F0203F003FB38F8153023F0020343F0F2
:10CC8000010328F8153073684BB31A785868DFF839
:10CC9000F4C0E3B208333CF813108D0702D5B0B1ED
:10CCA00039481FE021F02001C904C90C2CF81310E9
:10CCB00068B1032AF4D870683D68406890F800E0D5
:10CCC00005EB8E058AB9C5F81025C5F810253CF886
:10CCD000131021F01C0141EA82022CF81320B368E2
:10CCE0002BBB2A4804B0BDE8F081D5F8108541EA95
:10CCF0004E3128F00308C5F810853D6841F0200149
:10CD000005EB8E05D5F810052CF8131020F44730EC
:10CD100020F44070C5F810052002D5F8107500F415
:10CD2000F85040EA02403843C5F81005CFE72046E6
:10CD3000D3E90067FFF7BCFE002ED2D0114DD5E934
:10CD40000023964203D19F4201D1002209E01048FE
:10CD50000DF10F01FFF77EFD0C4B9842C2D19DF8FB
:10CD60000F20E4B205EBC20308345F6035F81430DD
:10CD700045F8326043EA422343F4807325F81430C7
:10CD8000AFE700BFE00000200400AD0B0000AD0BDA
:10CD9000380100202DE9FF4107460C461E4612B31C
:10CDA000DFF8D480CDB2083538F81530980701D4B3
:10CDB000990621D413F01C0F02D05378012B1BD0FD
:10CDC00001238DF80F3000232046CDE900230DF11B
:10CDD0000F01931C013203F051FA38F8153043F07B
:10CDE000030328F81530002E44D0234DE1B208315A
:10CDF00035F81120930703D4204804B0BDE8F08132
:10CE0000002096F800E03B6822F02002D20403EBF9
:10CE10008E03D20CC3F8100525F81120C3F81005B5
:10CE200096F801C04FEA8E08BCF1000F22D0386896
:10CE3000B6784044D0F810354FEA0C4C23F49813E0
:10CE400023F4F853C0F81035230203F4F8530CF41C
:10CE5000403C3605D0F8107543EA0C0306F4801602
:10CE6000334342EA4E323B4342F02002C0F81035D1
:10CE700025F811200248C0E7E00000200400AD0BB7
:10CE80000000AD0B014BC3E902127047E000002027
:10CE9000054BC9B2083133F81130990643BF5B0B1B
:10CEA0000248137002487047E00000200000AD0BFC
:10CEB0000400AD0B70B5154D064695F860401CBBDF
:10CEC0002146402205F1100002F00AFA214630689E
:10CED0002E6D8E420ED10023C0F87C31D0F87C310B
:10CEE00040F30730FDF7A8FE0123094885F86030BC
:10CEF000AB6570BDCBB29B0003F580727C2B04BF89
:10CF0000845083580131E4E70248F2E7E000002052
:10CF10000000AD0B0C00AD0B034B93F86000003824
:10CF200018BF0120704700BFE00000200148FFF754
:10CF3000B1BC00BF340100200148FFF78BBC00BF2B
:10CF40003401002073B503680C46D3F8041300299C
:10CF5000A4BF4FF00041C3F804131E49E3B20833E5
:10CF600031F8133099061AD513F0020617D15B0B6E
:10CF700005689C0004F580716E5069580168214471
:10CF8000D1F8104544F00104C1F810452AB101223E
:10CF9000016802FA03F3C1F8043302B070BDC3F3B1
:10CFA0008203042B11D0052B11D001A80194FFF7A7
:10CFB00047FD019A0369D34003F00103991C204601
:10CFC00002B0BDE8704003F0A2B90321F7E70221E7
:10CFD000F5E700BFE00000202DE9F347534B544F25
:10CFE000D3F80403396DC0B240F00040FFF78AFD6A
:10CFF000051E18DA00236846F96D00934FF001080A
:10D00000FFF748FD97F85C30DA0757D4396D4FF0D9
:10D010000040FFF777FD6846F96DFFF73BFD0028FC
:10D02000F0D125F000450124002D66D102B0BDE805
:10D03000F08794FAA4F4B4FA84F4E00804F1080345
:10D0400037F8139004F007021DF8003008FA02F2D6
:10D0500023EA02030DF8003001A80194FFF7F0FC69
:10D06000019B4FEA9901803350F82360C9F3820A8B
:10D070004B07D146C6F3014624D520465146FFF75B
:10D08000EBFC01A80194FFF7DBFC019BF6B28033B7
:10D0900050F82330C3F301439E4207D100212046BC
:10D0A00003F035F93146204603F031F901A8019427
:10D0B000FFF7C6FC019B08FA03F30362009C002CF7
:10D0C000B7D1A3E7022E0CD10321204603F01FF9AC
:10D0D0000AF00503012BE9D149462046FFF7BCFCC5
:10D0E000E4E70221204603F012F9BAF1030FF3D06E
:10D0F000032EDBD1BAF1020FEDE795FAA5F3B3FAEF
:10D1000083F304FA03F29B0003F1A04303F55043B9
:10D11000D3F81005D3F81015C0F30420C1F3014172
:10D1200025EA0205FFF798FC7EE700BF00D000501B
:10D13000E00000200022034BC3F88425C3F8042537
:10D14000704700BF00900350044AD2F80834DB0750
:10D15000FBD50160BFF35F8F704700BF00900350A5
:10D1600008B5C0F30B0383B90222094BC3F8842529
:10D17000C3F804254FF0FF320260D3F80024D20731
:10D18000FBD5FFF7D7FF034808BD0348FCE700BF06
:10D19000009003500000AD0B0A00AD0B012208B552
:10D1A000054BC3F88425C3F80425FFF7CDFFBDE880
:10D1B0000840FFF7BFBF00BF00900350430904D1F0
:10D1C0000123034A83409360704700239B60FFDE86
:10D1D000002584500C4B984213D00AD80B4B984230
:10D1E0000FD00B4B98420CD00A4BC31A58425841EF
:10D1F0007047094B984204D0084B984201D0084B25
:10D20000F3E70120704700BF40420F0090D00300B9
:10D2100020A1070048E8010000093D0000127A0043
:10D2200080841E00431C14D000F01F0340090BD162
:10D23000084A02EB8302D2F80012074B0B4043F07E
:10D240000203C2F8003270470022803352F82330C4
:10D25000FFDE704700258450F0F8FCFF430904D13D
:10D260000123034A8340D36070470023DB60FFDE65
:10D270000025845038B51446421C054616D00129B5
:10D2800002D1A3B1FFF79AFF05F01F036D0911D179
:10D290000B4A41EA840402EB8303D3F80002094AF3
:10D2A0000240144344EA4101C3F8001238BDFFF7BD
:10D2B000D5FFE9E70022803352F82330FFDE00BFBC
:10D2C00000258450F0F8FCFF2DE9F843504B4D69E0
:10D2D00006469D420C4690F8049000F0848077D872
:10D2E0004C4B9D4200F082804B4B9D4200F0818070
:10D2F0004A4B9D420CBF4FF000754FF080452422F1
:10D30000DFF81C81E07E02FB0983997F60F3000156
:10D3100099773379217C02FB03839A7F61F3410281
:10D320009A77E77EEFB9237E3A46012B94BF00231C
:10D33000012301212068FFF79DFF3B463A4601216A
:10D340006068FFF797FF3B463946A27EA068FFF76B
:10D3500091FF237C3A460121E06883F00103FFF747
:10D3600089FF242303FB0983E2681A62217C9A7FE8
:10D3700061F341029A77277FA07C217E637E326829
:10D3800047B9D4E900C7A468C2F808C5C2F80C754B
:10D39000C2F81045003B18BF01230229C2F8C0059E
:10D3A000C2F824552BD003292CD0012901D143F0F8
:10D3B0000203C2F8543524223379534358F803301A
:10D3C0001BB33068BDE8F84340F30730FDF734BCC9
:10D3D000144B9D4210D0144B9D420CBF4FF00045A2
:10D3E0004FF080458BE74FF0805588E74FF0806520
:10D3F00085E74FF0006582E74FF000557FE743F087
:10D400000403D6E743F00603D3E7BDE8F88300BF83
:10D4100040420F0090D0030020A1070048E801001F
:10D42000702E002080841E0000127A002DE9F8433F
:10D430000746242597F80480124C05FB08F504EBF9
:10D4400005091E4699F81C30C3B999B14869FFF720
:10D45000C1FEA8B138466251C9F80460FFF734FF35
:10D46000242303FB08440023637701230648237722
:10D47000BDE8F8836251C9F80460F1E70348F7E7B3
:10D480000348F5E7702E00200000AD0B0C00AD0B3B
:10D490000400AD0B2DE9F041044606790068194DF2
:10D4A00040F30730FDF7D6FB24237343EB5853B109
:10D4B0002368154A06EBC601C3F80823206805EB6C
:10D4C000810102F096FF2368242404FB0654D3F85C
:10D4D0000805D3F80C75D3F81085A37FDB070AD4B1
:10D4E000FFF7A0FE4046FFF79DFE3846FFF79AFE85
:10D4F000206AFFF797FE242303FB065500232B77B2
:10D50000BDE8F081702E00205201080024232DE98F
:10D51000F0430779534D7B439046EA180E46517FFE
:10D52000814685B0002940F09B80EB5823B118F06C
:10D53000140F04BF01235377242496E80F0004FB43
:10D54000075404F10C0C8CE80F00206A421C04D034
:10D55000A37F9B071AD5FFF731FE3368D9F8004047
:10D5600023B103F06043B3F1005F06D1B36883B128
:10D5700003F06043B3F1005F0BD02423002203FBD0
:10D58000075339485A7705B0BDE8F083FFF766FEC8
:10D59000E3E718F0010318BF0123C4F8503518F071
:10D5A000020318BF0123EC46C4F8403596E80F008B
:10D5B0008CE80F00039BC4F84405C4F84815C4F870
:10D5C0003425C4F838350023C4F81831D4F818319C
:10D5D0000723C4F8003524237B4318F0080F05EB1C
:10D5E00003021DD10121E858216158B9D4F818313E
:10D5F000002BFBD062464021204602F0BCFE2423D3
:10D600007B43EA18EB5813BB106A461C13D107EB97
:10D61000C707204605EB870102F0EBFE1348B2E78F
:10D62000EB58A3B9106A411CF8D0937F9A070BD529
:10D63000FFF714FEF2E7937F9B0702D5FFF70EFE7C
:10D64000E5E7FFF7BBFDE2E7FFF7B8FDE6E74023BC
:10D6500018F0040F14BFC4F80833C4F80433DDE72E
:10D66000034890E7702E00200A00AD0B0000AD0BC0
:10D670000B00AD0B10B540210F4A104802F07BFEA5
:10D68000C8B10F4C206A421C04D0A37F9B070FD562
:10D69000FFF7E4FD637F1BB10949084802F0A9FECA
:10D6A000002323720748D4E90031BDE81040184731
:10D6B000FFF784FDEEE710BD7C2E002000B0005087
:10D6C000702E0020782E002038B5EFF3118520232E
:10D6D00083F31288BFF36F8F064B9C6802F0B7FE8E
:10D6E00085F31188BFF36F8F2046BDE83840FDF702
:10D6F0002BBA00BF942E002038B5094B53F82040B8
:10D70000013053F82050A54200D838BD636823B1DA
:10D71000204602F09FFE0834F5E723689847FAE7B1
:10D720005C0E0100012270B5294B032086B01A70EF
:10D73000FFF7E2FFFCF754FF0420FFF7DDFF254C65
:10D74000254D2646AE4204F1300410D300F042FCD1
:10D75000204C224EAC4226D300F050FCFAF7FEFFDC
:10D760001F4A137B23F00103137306B070BD54F8F6
:10D770000C3C059354F8103C049354F8143C039368
:10D7800054F8183C029354F81C3C019354F8203C84
:10D79000009354E90A2354E90C0100F027FA54F8E5
:10D7A000303C5E65CDE7D4E90A23B3F1FF3F08BF03
:10D7B000B2F1FF3F05D052EA0301206803D102F025
:10D7C000DAFE3034C6E73146183000F0CBFDF8E71A
:10D7D000B2310020480A0100480A01008306010016
:10D7E000B002002008B50348034A0021121A02F0D3
:10D7F00049FE08BD10020020B431002000230122A0
:10D8000070B586B0CDE904230F220193CDE9023231
:10D8100014234FF4A0720E4D0E4E03FB00550E491B
:10D8200006EBC016044602FB00110C4B3046009577
:10D8300000F0DCF9737B2C7423F004037373084B42
:10D84000013403EBC423EE606B6006B070BD00BF13
:10D85000942E002030020020B83900201F0501005E
:10D86000B8310020BFB50020FFF746FF2A4B03F573
:10D87000006282F3088883F30A880024E023274D9E
:10D88000274E85F82230EC772C766C76AC7685F8CE
:10D8900020406B6A234F43F4E0236B6285F82340FA
:10D8A000FDF7D8F8FDF764FA4FF0FF3340F20112AC
:10D8B000AB62EB621C4B1D4D9A81B360C3E9194406
:10D8C0001C6702F0B0FD0120FFF716FF0220FFF7F2
:10D8D00013FF00F0B3FB164B756105930123154947
:10D8E0004FF40062CDE9034328463B46CDE90144AD
:10D8F000009400F07BF906466A7B284622F0040279
:10D900006A7302F074FE2046FFF778FF3A4631460C
:10D910002846FDF70FFA00BFB831002000ED00E007
:10D92000942E002025D7000030030020B0020020F4
:10D930003E160100F83A0020002038B5054C064D8F
:10D94000AC4200D338BD204602F0A0FD0028F9DB30
:10D950001C34F5E7BA010020BA01002073B50C466B
:10D96000EFF31181202585F31288BFF36F8FC5680F
:10D970005DB125602B68C36083690133836100203A
:10D9800081F31188BFF36F8F11E052EA030603D1D0
:10D990006FF00B002560F3E7CDE900230246083065
:10D9A00000F064FA18B9034B9B685B69236002B00E
:10D9B00070BD00BF942E00202DE9F34104461746A8
:10D9C0001E46EFF31188202383F31288BFF36F8F75
:10D9D000C368334A7BB180689168884219D057EA9E
:10D9E000060318D188F31188BFF36F8F6FF00F0013
:10D9F00002B0BDE8F081916891F90E100133E36047
:10DA000093682161A36088F31188BFF36F8F0020B2
:10DA1000EEE72169F2E791F90E1090F90E306FF000
:10DA20007E029942A8BF19469142B8BF11468B4267
:10DA30002DDD02F07FFD054622464146CDE9007608
:10DA4000184800F013FA0028E1D0EFF311862023E4
:10DA500083F31288BFF36F8FA068D0B12368216968
:10DA60009C420AD04BB193F90E309942A8BF194697
:10DA70006FF07E039942B8BF194602F05BFD40B1DA
:10DA80003146084800F062FA6FF00A00B0E700255E
:10DA9000D2E7002DF4D186F31188BFF36F8FF3E73F
:10DAA000942E0020B331002038B58368044663B358
:10DAB000194A926893422BD1C368012B03D9013BC9
:10DAC000C360002038BDEFF31185202383F3128853
:10DAD000BFF36F8F0169806802F02CFD204602F0D1
:10DAE000D4FDA06058B190F90E2022610022826717
:10DAF00002F07DFD2946094800F028FAE1E7E060E0
:10DB000085F31188BFF36F8FDBE76FF01500D9E75E
:10DB10004FF0FF30D6E700BF942E0020B331002035
:10DB200038B50446EFF31185202383F31288BFF341
:10DB30006F8F02F0AAFD48B10022826702F057FD04
:10DB40002946BDE83840074800F000BAD4E902325F
:10DB50009A4218BF0133A36085F31188BFF36F8F1A
:10DB600038BD00BFB331002013B5EFF3118120247D
:10DB700084F31288BFF36F8F846844B1013C8460E2
:10DB800081F31188BFF36F8F002002B010BD52EAFD
:10DB9000030406D181F31188BFF36F8F6FF00F007C
:10DBA000F3E7CDE900230246014800F05FF9ECE716
:10DBB000B331002070B50446EFF31185202383F3C1
:10DBC0001288BFF36F8F6FF00A06204602F05DFDEA
:10DBD00018B1866702F00BFDF7E7A0602946BDE8A3
:10DBE0007040014800F0B2B9B33100202DE9FF4187
:10DBF0000E9E00F1580506730426C0E9165500254F
:10DC0000044646730D9EC0E906558673D61D0C9AD0
:10DC100026F00706C0E919168560C573C56602922D
:10DC20000B9A01EB060801920A9A00924246FDF710
:10DC300065F8054B65659B6803B11B6F404623671C
:10DC400004B0BDE8F08100BF942E002038B50D4D22
:10DC50002B4653F8184F9C4200D004B9EC68AB68CF
:10DC600038B95A7BD20604D1A26912B9DA897F2A5F
:10DC700005D89C4202D0204600F0BCFA23466B61D6
:10DC800038BD00BF942E002008B590F90D20014644
:10DC9000002A437B04DA03F07F03437302F06DFC38
:10DCA000044B9868431A58425841BDE80840FFF7B2
:10DCB000CDBF00BF942E002070B490F90D30427B90
:10DCC000002B29DBD30627D183692BBB134962F0D4
:10DCD0007F0242730A4652F8184F944218BF2346F7
:10DCE000CC6923B9C0E900242060C8610CE090F938
:10DCF0000E5093F90E60B5420AD0AE4208DD5A6864
:10DD0000C0E9003210605860002070BCFFF79EBF71
:10DD10009C42E7D01B68E4E770BC7047942E00205B
:10DD2000002A2DE9F0410E460CBF10210821427B4C
:10DD3000044611420FD141EA0203D20918D14373BC
:10DD400008291BD00120FFF781FFBFF35F8F637BA2
:10DD500023F060036373264B9B68A34241D1EFF32A
:10DD60000583002B3DD13046BDE8F041FCF702BFF2
:10DD700003F07F03437302F000FCE1E7A36813B1F3
:10DD8000204602F002FC04F1180002F0BBFC4FF048
:10DD9000000804F15807A56DBD4200D0A5B9144D87
:10DDA000AB689C42CED1EFF30583002BCAD0012093
:10DDB000FFF74CFF40F201120E4B9A810022AB603C
:10DDC000C3E919221A67C0E7284602F0DEFB05F115
:10DDD000180002F097FC2846C5F87880FFF76CFF22
:10DDE000D9E786F31188BFF36F8FBDE8F08100BFDC
:10DDF000942E00203003002070B590F90D200146CC
:10DE0000002A437B04DA03F07F03437302F0B5FB7F
:10DE1000154A4B7B104663F07F034B7350F8183F55
:10DE2000D469834208BF002323B9C1E900042160FB
:10DE3000D1610CE091F90E5093F90E60B5420ED00D
:10DE4000AE420CDD5868C1E900300160596090684D
:10DE5000BDE87040431A58425841FFF7F7BE9C4254
:10DE6000E3D01B68E0E700BF942E0020F8B5124B0A
:10DE70000C46DDE9067611469868104A1060EFF30B
:10DE80001182202282F31288BFF36F8F9D6828468B
:10DE900002F085FBB6F1FF3F08BFB7F1FF3F06D0A8
:10DEA0003A463346064905F1180000F05BFA204671
:10DEB000BDE8F840FCF75EBE942E0020B42E002092
:10DEC00083060100F8B50446EFF31186202383F39F
:10DED0001288BFF36F8F437B49B2DA0619D1856987
:10DEE000BDB903F07F03437302F047FB437B164A3F
:10DEF00063F07F0343731346817353F8180F9842FE
:10DF000018BF0546D0695DB9C4E900300460D4612A
:10DF100011E00020A17386F31188BFF36F8FF8BD65
:10DF200095F90E70B9420BD08F4209DD6B68C4E9D8
:10DF300000531C606C600120FFF788FE0120EAE7B7
:10DF4000A842E1D02D68DEE7942E002049B9EFF316
:10DF5000058030B9054B5A699B689A4201D0FCF79D
:10DF600009BE81F31188BFF36F8F7047942E002094
:10DF700010B5EFF31184202282F31288BFF36F8F64
:10DF8000427B510704D484F31188BFF36F8F10BD17
:10DF900022F004024273FFF78FFE2146BDE81040D5
:10DFA0000148FFF7D3BF00BFB3310020034648B993
:10DFB000EFF3058232B9064A51699268914201D065
:10DFC000FCF7D8BD83F31188BFF36F8F704700BF94
:10DFD000942E0020EFF31181202383F31288BFF3E6
:10DFE0006F8F054B9A68D37B013BD37381F3118804
:10DFF000BFF36F8F704700BF942E002038B5EFF34A
:10E000001185202484F31288BFF36F8F0A4B002000
:10E010009A68D37B0133D373FFF718FE85F3118819
:10E02000BFF36F8FEFF3118084F31288BFF36F8F0C
:10E03000BDE83840FFF7BABF942E0020024B03F131
:10E040001802C3E906227047942E0020F8B5EFF3BA
:10E050001185202383F31288BFF36F8F19498868D5
:10E06000437B03F07F03437302F087FA08468B6813
:10E070005A7B62F07F025A7350F8182FCC698242A3
:10E0800008BF002222B9C3E900042360CB610CE081
:10E0900093F90E6092F90E70BE420ED0B7420CDDBD
:10E0A0005168C3E900210B6053600120FFF7CEFDEA
:10E0B0002846BDE8F840FCF75DBDA242E3D01268F7
:10E0C000E0E700BF942E002050EA01032DE9F04163
:10E0D00005460E4603D1FFF7B9FF00202BE0831C55
:10E0E00071F1FF3329DB02F022FB2C18EFF31188CA
:10E0F000202383F31288BFF36F8F124F124BB8683F
:10E100001860FFF7C1FDB86810492A463346183039
:10E1100000F028F9BA684046537B43F0100353736C
:10E12000FCF728FD02F003FB201A63EB0303012830
:10E1300073F10003D1DBBDE8F0816FF00104241A14
:10E14000D4E700BF942E0020B42E002083060100E7
:10E15000B1F1FF3F08BFB0F1FF3F08B506D10A4B50
:10E16000986802F053FA4FF0FF3008BDFFF7ACFF9C
:10E170004FF47A7147F6FF730022C0FB0132D80BCF
:10E1800040EA4240F1E700BF942E0020014B98681E
:10E19000704700BF942E00200122044BC01A044B8C
:10E1A000C0105843034B1A54704700BFB0030020FF
:10E1B000ABAAAAAAB3310020C3897F2B12D80A4B7D
:10E1C0001B6863B1094B90F90E201B689A4209DB6A
:10E1D000437BDB0606D1064BC31A18BF012303F0AD
:10E1E000010070470023FAE7BC2E0020B82E002063
:10E1F0003002002070B50E4B0E4C1E7C054606EB1F
:10E20000460304EBC304204602F07CFA00220A4BCA
:10E2100028469A55FFF7D0FF48B1084B2046BDE885
:10E2200070401A680649013AD31700F09BB870BDD8
:10E23000942E0020B0030020B3310020BC2E00201B
:10E2400099E1000038B5EFF31185202383F312889C
:10E25000BFF36F8F104B114A9C681068A04206D123
:10E26000FFF7C8FF85F31188BFF36F8F38BD00211A
:10E270001B7C11600A4AD35C002BF3D02046FFF7C9
:10E280009BFF0028EED0637BDB0602D12046FFF720
:10E29000B3FD2046E4E700BF942E0020B42E0020FA
:10E2A000B331002008B50648064A0749121A02F0A1
:10E2B000EBF8BDE80840054A0549064802F0E4B815
:10E2C000000000200C0200204C160100000000009D
:10E2D0004C16010000000020034B1B680BB9FEF731
:10E2E0000FB80020704700BFC02E002030B570B1BD
:10E2F0000B4B5B6898420AD0036843B1D3E9042111
:10E30000D0E90445121941EB0501C3E90421D0E924
:10E31000003213605A600023C0E9003330BD00BFF3
:10E320004401002010B50E4B1C689C4204D1FFF73D
:10E33000D3FF6FF0004010BDFFF7CEFF002CF8D0E8
:10E34000D4E904321B1A62EBE072B3F1004F72F1B0
:10E350000001EEDA002AACBF18460020EBE700BF50
:10E3600044010020B3F1FF3F08BFB2F1FF3FF8B511
:10E3700004461D4616465ED08160EFF311872023C8
:10E3800083F31288BFF36F8F013275F1FF3324DA04
:10E390006FF001032D49D1E900209B1A4FF0FF32A5
:10E3A00062EB00009E1B60EB0500012E70F1000384
:10E3B00001DA01260020C4E90460254ED6F800C029
:10E3C0007568B44508BF4FF0000CBCF1000F0DD1CB
:10E3D000C4E900652C6074601CE0FFF77DFF013626
:10E3E00045F10005361845EBE070E4E7DCE9042070
:10E3F000D4E90431934271EB000E1DDAD21ADCF835
:10E40000043060EB0100CCE90420C4E900C31C60C7
:10E41000CCF804403368B34209D09C4207D10D4B7D
:10E420001C6824B9FFF77EFF2146FDF73BFF87F309
:10E430001188BFF36F8FF8BD9B1A61EB0001AC45EB
:10E44000C4E90431C4D0DCF800C0BEE7C803002032
:10E4500044010020C02E00202DE9F84FEFF3118C6D
:10E46000202383F31288BFF36F8FDFF8B0A0DFF8AB
:10E47000B0900024C9F80000DAF8000000255045EB
:10E4800008BF0020274FE046D7E90021D9F8003027
:10E4900078B3D0E9046C4FEAE37EB3427EEB0C0B19
:10E4A00005DAF61A6CEB0E04C0E9046421E0B21838
:10E4B00041EBE671C0E90445C7E90021FFF716FF0B
:10E4C00088F31188BFF36F8F83689847EFF3118843
:10E4D000202383F31288BFF36F8FD9F80030DAF866
:10E4E00000009B1B5045C446C9F80030CBD1D7E98A
:10E4F000002100249A1841EBE373C7E90023C9F80F
:10E500000040FFF70FFF2146FDF7CCFE88F311888E
:10E51000BFF36F8FBDE8F84FFFF794BE44010020B2
:10E52000C02E0020C803002010B5EFF31184202373
:10E5300083F31288BFF36F8FFFF7CEFE0346054AC1
:10E54000D2E90001181841EBE37184F31188BFF39D
:10E550006F8F10BDC803002010B50A4C23681BB193
:10E5600001232360002010BD00F0ECF80028F7D054
:10E570000138062803D8044B53F8200010BD034887
:10E5800010BD00BFC42E0020740E0100FE8FFFFFDF
:10E59000BFF34F8F0549064BCA6802F4E06213438C
:10E5A000CB60BFF34F8F00BFFDE700BF00ED00E081
:10E5B0000400FA0530B44FF0FE320025074B084C3A
:10E5C00008494968C3F80024C3F80424C3F80824A0
:10E5D000C3F80C24C4F8005530BC08470010845020
:10E5E000000084504C010020024BD0E90012C3E926
:10E5F000001270474C01002010B5044650B163680A
:10E6000013F0685F05D0064A934202D0002362608F
:10E61000236010BD034B04485B689847EFE700BFD9
:10E620002C5F5CA94C010020900E0100C8B143682A
:10E630000D4A934213D013F0685F0ED0012350E8C7
:10E64000002F194640E8001C9CF0000FF7D1012A6A
:10E65000F5D0BFF35F8F002070470448704704482F
:10E6600070476FF4E04070472C5F5CA9E98FFFFFB3
:10E67000EA8FFFFF034680B1426809498A420AD007
:10E6800012F0685F05D0BFF35F8F002210461A605A
:10E69000704704487047044870476FF4E040704783
:10E6A0002C5F5CA9E98FFFFFEA8FFFFF10B50446DE
:10E6B00020B10023034A2360626010BD0248FFF7C7
:10E6C00079FFF6E73A00003AB80E010070B5194C30
:10E6D000D0F804C00668C4F804C0D0F808C0C06808
:10E6E000C4F808C0E06026600868134B134D18603A
:10E6F0004868D5F818215860886812F0685F9860FB
:10E70000C8680969D860196112D000230C4A05F560
:10E710008A70C5F81431C5F8B831C5F81821C5F8A4
:10E72000BC21B047236805F5DC70BDE87040184790
:10E7300070BD00BF6801002054010020DC2E0020C5
:10E740002C5F5CA938B500F02FF820B1032400F04D
:10E7500063F8204638BD00F031F898B900F0ACF805
:10E7600098B90F4DD5F828391B0EF02B08D1D5F8E4
:10E77000242A0C4B9A420AD0072400F017F8E6E747
:10E780000624FAE70424204638BD0024F5E70120DA
:10E7900000F092F804460028F7D1C5F80C0AD8E733
:10E7A000001084500000E0200020704700207047D7
:10E7B000014BC3F8040A70470010845010B511488B
:10E7C00000F048F800B110BD0F4800F043F80028F1
:10E7D000F9D10E4C204600F03DF80028F3D10C4B47
:10E7E0000C481C6000F036F801460028EBD100F020
:10E7F0002DF8044608B1204610BD00F03FF8204631
:10E80000FAE700BFA8010020A4010020A001002019
:10E81000980100209C01002008B5084800F024F869
:10E82000074800F021F8074800F01EF8064800F0FD
:10E830001BF8BDE8084000F00BB800BFA80100209D
:10E84000A4010020A00100209C01002000207047AE
:10E85000704700BF08B5034B02681B6810689847F3
:10E86000002008BD6801002008B5034B02685B6802
:10E8700010689847002008BD6801002070B5094C59
:10E88000094D2069AB68984718B1084B08485B6888
:10E8900098470021074AEB6811602069BDE8704085
:10E8A000184700BF54010020680100204C010020DF
:10E8B000DC0E0100D82E0020F8B51A4D1A4E044681
:10E8C000B26828699047E8B9184F3B684CB1A3B1CA
:10E8D000012B19D0013B3B602869F3689847002061
:10E8E000F8BD43B90121124AC2F800151149D1F807
:10E8F0001029002AFBD101333B60F368286998474F
:10E900000020F8BD0C48F8BD0A4AD2F81039002B97
:10E91000FBD1074A6FF07E40C2F80035FFF748FF91
:10E920003B68D7E75401002068010020D82E002062
:10E930000000845000108450E98FFFFF70470020D2
:10E94000704730B5836804468B42154685B00ED9B2
:10E950006368C068194401AA01F0D3F828B9626855
:10E96000019B9B1A2B60029B6B6005B030BD6FF062
:10E970002100FAE770472DE9F7430E4617469946FE
:10E98000044628B94FF0FF38404603B0BDE8F08395
:10E990000029F7D0002AF5D0CB680D8938461D44F0
:10E9A000042329460DEB030200F0CAFB8046002831
:10E9B000E8D146F60812BDF804107389914225D1BA
:10E9C000BDF806109942DDD1042338460DEB030251
:10E9D000294400F0B5FB0028D4D146F60713BDF852
:10E9E00004209A42CED1C4E900679DF82830A4F8EB
:10E9F0000890A3727389BDF806202B44E3607389E5
:10EA000013442B44043563612561BDE7002BE4D03A
:10EA1000B8E72DE9F3410E4617461D46044620B9D6
:10EA20004FF0FF3002B0BDE8F0810368002BF7D053
:10EA30004368002BF4D04FF6FF78D4E904239A42C0
:10EA400016D223685B8923B1E368934204BF043381
:10EA500023610423216960680DEB030200F070FB61
:10EA60000028DDD1A37A2BB1D4E903329A4201D335
:10EA70000120D7E72389BDF80610434501F10402C0
:10EA800003D0BDF804C09C450BD115B1BDF80430CE
:10EA90002B80236904333360398023691344236155
:10EAA000C0E7236913442361C7E748B103683BB15A
:10EAB00043682BB1C068884294BF00200120704792
:10EAC0004FF0FF30704773B50C46064611460223DF
:10EAD000204601AA00F0C3F90546E8B9019A1F2AA9
:10EAE0000ED9A2F12001304620222368194400F0FB
:10EAF000ECFB2368019A13442360284602B070BDE2
:10EB00000146C2F12002304600F0EAFB019A21687A
:10EB1000C2F120003044EAE76FF00205EDE74FF460
:10EB2000407358433030704710B5044600F046FB40
:10EB30004FF44072A368303B02FB103010BD70B53B
:10EB40000D46044601F061FA2A46A0F108010423AB
:10EB50002046BDE8704000F0F3BA13B504460191B9
:10EB600001F053FA0423A0F108010DEB0302204643
:10EB700001F08EFA02B010BDFFF7FEBFFFF7FCBF39
:10EB8000FFF7FABFFFF7F8BFFFF7F6BFFFF7F4BFD5
:10EB9000FFF7F2BFFFF7F0BFFFF7EEBF7047F8B522
:10EBA0001346164658220F4690F8B810044601FB4B
:10EBB00002020021FAF726FE94F8B85008B1012DA0
:10EBC0000DD1582303FB054501213346204605F1AD
:10EBD0002C02FAF717FE10B1002F08BF0020F8BD75
:10EBE0002DE9F341044690F8B8000D461646F9F7B2
:10EBF00043FE6946C0B2FBF79BFC88BB2C224FF05A
:10EC00005808554394F8B830009808FB0353234440
:10EC10001F89DB681F44042339460DEB030200F013
:10EC20008FFAE8B994F8B830BDF8042008FB035512
:10EC300046F608132C449A426489009816D1BDF810
:10EC400006309C420CD10423E1190DEB030200F0C5
:10EC500077FA28B946F60713BDF804209A4208D07F
:10EC6000009800F06CFA02B0BDE8F081002CF1D001
:10EC7000F6E7BDF80610214439443160F0E701237E
:10EC8000036003F1012343600023C0E902337047AE
:10EC90004379012B07D10368012B04D10079431E6E
:10ECA0005842584170470020704700F073BA2DE970
:10ECB000F84F90F8B8600F46044600213046F9F747
:10ECC000DBFD054601213046F9F7D6FD3B789D4234
:10ECD0002DD098422DD101262C224FF058095643B1
:10ECE00094F8B830D4F8B40009FB036323449D6A58
:10ECF000FFF715FF4FF0000A8046013D94F8B83049
:10ED0000384609FB036323445B6A03EBC50253F8EF
:10ED10003510D2F804B01B685A46C91ADA44FFF716
:10ED2000C4FFC24505F1FF35E8D3BDE8F88F0026E2
:10ED3000D2E70120F9E773B5154690F8B8600C46A4
:10ED4000012E69468CBFFF20022001F0E4F9E97929
:10ED5000012903D03246204601F0F1F99DF8033035
:10ED6000012B02D1204601F0C9F9A9682046FFF71E
:10ED7000F4FE2046FDF77AFB002002B070BD582259
:10ED800090F8B83002FB0300436A00205A6803463B
:10ED900013448B4200F10100FAD3704710B5437958
:10EDA0000279012B06BF00230C460B0202F1FF3251
:10EDB00001FB0233026818BF4C00013A04FB023029
:10EDC00010BD0120704770B50368CD1A002D02DC1C
:10EDD0006FF05F0070BD93F900601C78002E0ADBB5
:10EDE0005C1C04601B7813600368C91A13688B42AB
:10EDF000EED80020EEE704F07F04013C032C2BD872
:10EE0000DFE804F0020A1421012DE1D05B781360E1
:10EE1000036802330360E7E7022DD9DDB3F8013060
:10EE20005BBA9BB2136003680333F3E7032DCFDDB6
:10EE30009C785D782402DB7844EA05442343136020
:10EE400003680433E6E7042DC2DDD3F801301BBAB2
:10EE5000136003680533DDE76FF06300BAE770B451
:10EE600004680E1B002E07DD26789E4208D101346F
:10EE7000046070BCFFF7A7BF6FF05F0070BC704705
:10EE80006FF06100FAE738B503230446FFF7E7FFA8
:10EE900018B9136813B96FF0670038BD013B1360F0
:10EEA00023681A78002AF6D101332360F5E72DE9AB
:10EEB000F34190461F4601AA302305460E46FFF750
:10EEC000CEFF0446F0B92B68F61A002E34DD424618
:10EED0001B78284642F8043B2E68019B1E443146AD
:10EEE0000623FFF7BCFF044660B92B68D8F804205E
:10EEF000C8F808309918B142296007D10C2138466A
:10EF0000FAF730FF204602B0BDE8F0819B5C3A463C
:10EF100042F8043B2B683146013328462B60FFF74B
:10EF200052FF60B92B687A68BB601344B34218BFC4
:10EF30006FF065042B60E5E76FF05F04E2E70446DD
:10EF4000E0E7002070470FB407B504A951F8040B9F
:10EF50000191FAF793FF03B05DF804EB04B070473A
:10EF6000044608B5084611461A46A047FFF70EF9B1
:10EF7000FBF7EAFD038B13F0070305D10368002BB1
:10EF80000CBF002003207047022B05D1408BB0FA44
:10EF900080F0400980007047012B05D10368002BE9
:10EFA0000CBF0020052070470020704710B50C46AC
:10EFB00000B111B96FF0150010BD081D00F093F8F5
:10EFC0000028F9D1A368032BF6D9F3E72DE9F04126
:10EFD0000D4607461946281D90461E4600F094F837
:10EFE000044638B13346424629463846A446BDE871
:10EFF000F0416047BDE8F08110B4EFF311822024A6
:10F0000084F31288BFF36F8F416110BC0121FBF7BD
:10F0100081B938B50C46054658B151B10B6843B1BA
:10F020004B6833B11C22002100F05AF900202C61FA
:10F0300038BD6FF01500FBE770B505460E46FFF7CB
:10F04000B5FF041E14DBEFF31182202383F3128833
:10F05000BFF36F8F4FF6FF716B8B2C8B8B4204F0DD
:10F06000070407D182F31188BFF36F8F6FF00A0492
:10F07000204670BD022C0CD101336B8382F31188C2
:10F08000BFF36F8F0023224631462846FFF79EFFCD
:10F09000EEE7062C14D8DFE804F004131313041A67
:10F0A0000400002333606B683BB9C5E90066ACB966
:10F0B00002212846FBF72EF9DAE71E606E60F6E7BC
:10F0C00082F31188BFF36F8F6FF00404D0E782F3EF
:10F0D0001188BFF36F8F6FF08504C9E782F3118841
:10F0E000BFF36F8FC4E7034658B1426802F00302D2
:10F0F000012A03D0032A04D1026812B100209860CB
:10F1000070476FF0150070474268034602F0030233
:10F11000032A4FF00002816014BF104600685A6055
:10F12000704770470FB407B504A951F8040B01915B
:10F13000FAF7A4FE03B05DF804EB04B07047704723
:10F14000002930B4044618460BDBA5680844A842E1
:10F1500007D8E0686468214484682468A44630BC09
:10F1600060476FF0150030BC7047002930B404468A
:10F1700018460BDBA5680844A84207D8E068646815
:10F18000214484686468A44630BC60476FF0150071
:10F1900030BC70470029034610B410460ADB9C6857
:10F1A0000844A04206D8D8685B681944836810BC3C
:10F1B0009B6818476FF0150010BC704708B5C06811
:10F1C0008368DB689847006808BD08B5C068836835
:10F1D000DB689847007908BD70B54C680368A342A6
:10F1E00001D2012070BD8A682244934201D30020DD
:10F1F000F8E74E69D1E90325B54203D36FF00B035D
:10F200008B61F4E71B1B42F835304368086902EB59
:10F21000C00253600B6901330B61E2E7002008B5BF
:10F22000FBF762F8012801D1EFF30583FEF74CBA32
:10F2300001460068FFF7F6BF08B5FBF7C7FABDE85F
:10F240000840FBF7C7BA00210120FFF7EBBF436E70
:10F2500083F30B88704761B662B680F31188BFF301
:10F260006F8F704772B6002383F31188BFF36F8FDF
:10F27000BFF34F8F30BF62B6BFF36F8F704772B668
:10F28000002383F31188BFF36F8FBFF34F8F20BF2D
:10F2900080F31188BFF36F8F62B67047034600207A
:10F2A0001A5C02B970470130FAE710B55AB101395A
:10F2B000841810F8012B11F8013FA04201D09A42A6
:10F2C000F7D0D01A10BD1046FCE710B5431E0A4413
:10F2D000914200D110BD11F8014B03F8014FF7E73F
:10F2E0000346C9B20244934200D1704703F8011BA0
:10F2F000F9E74FF0FF3070470C220369C9B201FBF8
:10F300000233186C00F00700704770B5C9B203698A
:10F31000EFF31185202484F31288BFF36F8F0C263E
:10F3200006FB0134246C14F0C00408D0A24206D0BD
:10F3300085F31188BFF36F8F4FF0FF3070BD01224E
:10F3400071430B441A6485F31188BFF36F8F4368D0
:10F350000B445B6898470020F0E78022FFF7D5BF99
:10F36000F8B5069F0469C9B2EFF31186202585F32D
:10F370001288BFF36F8F0C2569430C44256C05F090
:10F38000070CBCF1010F0BD1276486F31188BFF382
:10F390006F8FC4E90E2343685B5898470020F8BD7F
:10F3A00005F0C005AF4286F31188BFF36F8F0CBF25
:10F3B0006FF077004FF0FF30F1E713B58024009431
:10F3C000FFF7CEFF02B010BD10B41C240069CBB211
:10F3D00003FB0400002110BC10470020FDF7A0BA79
:10F3E000002000F049BF1046FEF79ABB43681C336B
:10F3F0000B60012313607047FEF792BB4FF0FF32A2
:10F400004FF0FF33FEF7B0BBF0B54468076900204A
:10F410008BB000908DF804000120119E0790109889
:10F420008DF80010D107CDE9080602F08005CDF86F
:10F4300018D00DD53A7D1BBA0493D3071DD50422ED
:10F4400004A90DF10100FFF740FF079B0433079368
:10F45000002E0CBF0122022206ABCDE9032302934A
:10F4600002232146059351F8040B85B183681C687B
:10F47000002302AAA0470BB0F0BD03220DF1110139
:10F480000DF10100FFF721FF079B0333DFE78368DE
:10F490001C6804ABEDE7002373B50D1E466814BF6E
:10F4A00004210621CDE9003380220446FFF7ACFF9A
:10F4B00096F83430DB0609D540B93DB90346CDE9AD
:10F4C0000000802298212046FFF79EFF02B070BD09
:10F4D0001FB5012301930DF10F03009300230521B4
:10F4E0001A46FFF791FF08B99DF80F0005B05DF8C7
:10F4F00004FBF7B51E4643680D1E044617469B697C
:10F5000014DBAA199A4211D80069FFF777FF2B463E
:10F51000012203212046CDE90076FFF775FF05465D
:10F520002069FFF769FF284603B0F0BD6FF01505AD
:10F53000F9E7F7B54468054694F83430DA0744D55E
:10F54000076901F0F8F84FF47A76A0FB063206FB63
:10F550000122DB0B43EA42433A699B1A13D4E28D42
:10F56000268E9B1AB3420EDA4FF4004740F2E73082
:10F570000021F61A4FF47A720023E6FB0701F8F730
:10F5800085FFFEF7E5FD94F8343013F002031CD13B
:10F590008022AB212846CDE90033FFF735FFA8B91B
:10F5A00094F83430DB0710D540F2E7314FF40045D2
:10F5B0000E460146648E4FF47A72E5FB0461002327
:10F5C0003046F8F763FFFEF7C3FD002003B0F0BD3F
:10F5D0002DE9FF41064615461C4601270DF10F088F
:10F5E000002305211A463046CDE90087FFF70CFFBE
:10F5F00040B99DF80F30DB0704D528462146FEF7B9
:10F60000A7FDEDE704B0BDE8F0812DE9F74F054611
:10F610001F46436800690E1E92469B69B0F81E9013
:10F620004CDBF2199A4249D8FFF7E8FE0021284640
:10F63000FFF731FF0446B0BB83462FB901212846AE
:10F64000FFF729FF044632E0B945C84628BFB8464F
:10F6500006EB0803013B96FBF9F2B3FBF9F3934287
:10F6600018BF09FB12624FF0000318BFA9EB020894
:10F67000062180222846CDE900BBFFF7C5FE3346B0
:10F68000812202212846CDE900A8FFF7BDFE0446ED
:10F6900048B9012200232846A7EB0807C244464484
:10F6A000FFF796FFC9E701212846FFF7F4FE286916
:10F6B000FFF7A2FE204603B0BDE8F08F6FF01504FF
:10F6C000F8E72DE9F74F43680F1E05461646D3F8B5
:10F6D00018A077DBBB18534574D847EA0209C9F371
:10F6E0000B09B9F1000F6DD10069FFF787FE49469C
:10F6F0002846FFF7D0FE4FF0FF3B0446002E5AD1BC
:10F7000001212846FFF7C7FE002C08BF04462869E0
:10F71000FFF772FE204603B0BDE8F08F234680223B
:10F7200006212846CDE90044FFF76EFEB2450FD111
:10F7300023468022C7212846CDE90044FFF764FE16
:10F74000264640F2676200232846FFF741FFD5E7CF
:10F75000A0462A6902F115031D32597881B10BFACE
:10F7600001F037EA00000BD101208840B04207D8F1
:10F77000B8F1000F1AD098F80100884238BF9846B7
:10F7800002339342E9D1B8F1000F11D03B468122F8
:10F7900098F800102846CDE90099FFF735FE0123BF
:10F7A00098F8012093401F44F61ACAE79846E7E705
:10F7B0006FF01504C5E7002CB0D001212846FFF7F3
:10F7C0006AFEA4E76FF01504A4E72DE9F0430446B0
:10F7D00087B000694FF0FF32012100F0BAFE676880
:10F7E000386800F021FE28B96FF01205284607B0EE
:10F7F000BDE8F083F86858B92069FFF7FFFD20469F
:10F80000FFF797FE002808DA2069FFF7F5FDEBE720
:10F8100000F00AFE0028EFD1E6E72046FFF758FE89
:10F82000002806DDC50704D5002200232046FFF787
:10F83000CFFE2069FFF7E0FD2069FFF7DFFD4FF005
:10F840000308002302AE1A469F212046CDF804800B
:10F850000096FFF7D9FD05462069FFF7CDFD002D85
:10F86000C2D13046424607F12401FFF71EFD06468D
:10F87000002840F0CE8097F82C30206953B3FFF772
:10F88000BDFD2046FFF724FE051E1EDD97F82C3037
:10F89000802225EA0305062133462046CDE900668D
:10F8A0008DF81050FFF7B0FD03460028ACD10121C0
:10F8B00004AA0092204680220191FFF7A5FD0022B4
:10F8C000054600232046FFF783FE2069FFF794FDDD
:10F8D000002D89D10022CDE904226368276993F8BD
:10F8E000271007F115088DF813109E6A736893426C
:10F8F00080F28280012123F00043A3F12002C3F1B2
:10F90000200001FA02F221FA00F0024301FA03F3A7
:10F91000DB0843EA4275002108224046FFF7E0FC7D
:10F920004FF00109494609F10109424630465FFAA4
:10F9300089F900F016F9B9F1050F08F10208F1D1C3
:10F940009DF813300A2B89BF01234FF48073B26AEC
:10F95000C2F3031288BF9340FB8363689B699D4297
:10F960007FF442AF336813F4C02F27D0314603AA87
:10F9700004A8FBF76FFC054600BB9DF80C60731EE6
:10F98000DBB2FD2B1AD8B0073FF42EAF2069FFF78A
:10F9900035FDB10732D400238022B7212046CDE9BE
:10F9A0000033FFF731FD00287FF42EAF2269137D6D
:10F9B00043F0010313752069FFF71EFD6268D2E969
:10F9C00007134B4392699A427FF40EAF2069FFF709
:10F9D00015FD636893F83430DA073AD500238022A6
:10F9E000B9212046CDE90033FFF70EFD054698B159
:10F9F0002069FFF701FDF9E6013389E72B468022F4
:10FA000006212046CDE90055FFF7FEFC0028C2D0B4
:10FA1000FAE66FF01505E9E66368256993F8343076
:10FA2000DB070AD42846FFF7E7FC2069FFF7E6FC6E
:10FA30002046FFF77EFD0546DAE700F07CFE4FF436
:10FA40007A72A0FB020302FB0131C00B40EA414085
:10FA500028612069E7E738B505460C4600F06DFCE3
:10FA6000002D07DBA84205D9401B84428CBF002033
:10FA7000012038BD0020FCE770B50D461946284628
:10FA800016461C46FFF7E7FF38B124B12246294647
:10FA90003046FFF71AFC002070BD6FF01500FBE741
:10FAA000F7B51C460023164682682360A3600D4606
:10FAB0001369694601AA9847019B5A1E01921BB916
:10FAC0006FF0150003B0F0BD0098A2684768216888
:10FAD000676085B9B31AD0F800C0634528BF634694
:10FAE00003FB07111A442160A26002689A4206D8FB
:10FAF00008300090E0E76B1AB3FBF7F3EBE7002068
:10FB0000E0E713460022FFF7CBBF2DE9F0470024C2
:10FB1000836886B0884691461B6902AA01A9984766
:10FB2000A2462546029BAB4202D806B0BDE8F0874C
:10FB30000026019F07EBC5077B6804933A680AEB30
:10FB40000603B24202D89A460135EBE749460394D0
:10FB5000059303A8C0470028E7D0049B01361C4446
:10FB6000ECE74B1E5B0800EB8300C369C90758BF75
:10FB70001B0CC3F3072113F0FF031BBF0020117000
:10FB80006FF0150053707047436800205B681B6975
:10FB90000B607047436802EA01005B6821EA0201DA
:10FBA00098600020D9607047436800205B689960C6
:10FBB0007047436800205B68D960704743685A68A3
:10FBC000536821EA03000B4090600020D360704727
:10FBD00010B503695868F8B1884219D19C68086863
:10FBE000A142586000D19860002008602AB15A688C
:10FBF0000A609A68596002B99960002010E0814259
:10FC000006D10868206098688142EDD19C60EBE7DE
:10FC1000044600680028F2D1002AE8D16FF01500F0
:10FC200010BD30B543681360057A446804EBC50421
:10FC3000A34202D36FF0010030BD5C798C4201D049
:10FC40000833F0E70020F7E743681B68D3F8800427
:10FC5000C3F880047047436802691B68D3F8100139
:10FC600050B10020526912780A70C3F81001D3F81D
:10FC7000102101221A6070474FF0FF307047026870
:10FC80000346D2F8580140B95B689B0706D4D2F806
:10FC90002001003818BF01207047012070474268DA
:10FCA0001368D3F80413C90517D5D3F82011A1B1EF
:10FCB000EFF31181202080F31288BFF36F8FD3F808
:10FCC000200130B10020C3F82001D3F82001012029
:10FCD000D86081F31188BFF36F8F5268D20614D5B4
:10FCE000EFF31182202181F31288BFF36F8FD3F8D5
:10FCF000581111B10021C3F800154FF48001C3F869
:10FD0000081382F31188BFF36F8F704710B5044654
:10FD1000002201210920FAF7BFFF0920FAF78CFF22
:10FD20002046BDE81040FBF7EFBC10B504460022AA
:10FD300001210820FAF7B0FF0820FAF77DFF2046DE
:10FD4000BDE81040FBF7E0BC002201210B20FAF7D0
:10FD5000A3BF10B50B6813B91846136005E003681C
:10FD60005C681CB114600368186810BD0833036038
:10FD70000B68013B0B60EDE703460A461979012346
:10FD8000006803FA01F103691B68194218BF82F089
:10FD9000010212B18368DB68184783681B69FBE7BF
:10FDA00010B504460068D0B18368C3B149B10121E0
:10FDB0000830FFF7E1FF23681869BDE8104000F044
:10FDC0002EBB12B98388DB0409D4006900F027FB3D
:10FDD00020680021BDE810400830FFF7CDBF10BDFE
:10FDE00010B5012200210446FFF7DAFFA36933B9F9
:10FDF000636004F11000BDE81040FDF791BE10BD36
:10FE000010B5006903688B4206D190F85C4034B9A4
:10FE1000FFF7E6FF204610BD6FF01500FBE76FF01F
:10FE20000F00F8E72DE9F34144680569666B00218E
:10FE3000304601AAFFF7F5FE002825DB019B32685A
:10FE400019791868FBF7A2FB00281DDBA16B481C81
:10FE500011D10126E36A9847AC680834D5E902322B
:10FE600003EBC203A4F10802934210D82846FFF71F
:10FE7000B7FF002008E004F13C00FBF7D1FF10F1D0
:10FE8000130F01D0411DE4D102B0BDE8F08154F858
:10FE9000080C00F0C9FA28B354F8080C14F8041C34
:10FEA00034F8023CD0F810C0DA07DCF8007054BF18
:10FEB00043F4B01383F4D01323F4801206FA01FE46
:10FEC000DB07D0F808804CBF4EEA070727EA0E0789
:10FED000CCF80070D8F800309847002804F10804E6
:10FEE000BCDAD1E76FF01200CEE738B505690446F9
:10FEF000296305F12000FDF713FE002285F85C2040
:10FF000020691146BDE83840FFF74ABF38B502788E
:10FF10000346002A52D10C69A26D32B9606D6FF0B0
:10FF20007301BDE83840FFF7E0BFE06C40B1216DE0
:10FF300031B1DB6823B1834202D0616EFFF7C5F9AE
:10FF4000A36CA56D9BB19D4211D85B1BA3644BBBF9
:10FF5000636B04F1480208336363A36B04F1380157
:10FF6000013BA36304F13400FFF7F3FE6064236DEB
:10FF70009BB19D4211D85B1B2365CBB9E36B04F1A8
:10FF800050020833E363236C04F14001013B236416
:10FF900004F13C00FFF7DDFEE064606DBDE8384031
:10FFA000FBF73EBD636C002BE1D02B446364DEE7BE
:10FFB000E36C002BF1D02B44E364EEE738BD002264
:10FFC00000F150039B009BB203F1502303F58033F3
:10FFD0001A601B68704708B5FCF700F808BD0346B7
:10FFE0005A6B00233C309A4200D17047C1680133FC
:10FFF0000844F8E7FEF7B0BA08B5FAF703FBFAF7DA
:020000040001F9
:10000000CFFBBDE80840FEF7A7BA8068183820F09B
:10001000070010387047042809D0052803D1481E6E
:1000200018BF01207047431A5842584170470120B9
:10003000704738B515460C4661B15AB1FFF7C5F89F
:100040002146254411F8013B834203D1A942F9D14D
:10005000012038BD0020FCE738B50C4601231146CD
:1000600022460546FFF76CF800280FDB01222146E7
:100070002846FFF7DEFF38B92378012B14BF02238F
:1000800001230020237038BD0323FAE70120FAE79B
:100090002DE9F7431D4606460F469046FFF78EF8BA
:1000A0006C1E044440420440082C1AD83046FFF726
:1000B0008CF881462A4641466846FFF706F94946CC
:1000C000621B0DEB0500FFF70BF923466A46394624
:1000D0003046FFF74AF8003818BF012003B0BDE8EA
:1000E000F0834FF0FF30F9E707B501238DF80420C6
:1000F00001AAFFF7CDFF03B05DF804FB8168012280
:10010000183921F00701FFF7EFBF8268183A22F093
:100110000702FFF7A1BF13B50C46C0B201A9FAF759
:1001200007FA50B921460198FCF7C0F90446019836
:10013000FFF705F8204602B010BD0124FAE713B519
:1001400041EA021104468DF80710FFF75EFF012314
:1001500001460DF107022046FFF79AFF02B010BDDD
:1001600081680122183921F007010839FFF7BCBF67
:100170004FF47F03D3F83001D3F83431BFF34F8FFE
:10018000C0F30B00A0F109035842584170474FF4E7
:100190007F02D2F83031D2F83401BFF34F8FC3F36E
:1001A0000B03092B03D1431E5842584170470020CE
:1001B0007047004700F033B940F00040C1F88000BC
:1001C000C2F880007047F7B5044618B1012824D062
:1001D00003B0F0BD4FF050230222C3F808230122E0
:1001E0000646DA60C3F80401D3F80431012342F271
:1001F00010754FF050278DF80730DCB1012CE7D196
:10020000D7F80C3403F480338EBB002BE0D00120F0
:10021000FFF7D0FF013DF3D1DAE74FF05023002282
:10022000C3F808035860C3F80021D3F800310DF17A
:100230000706DBE7D7F8183403F480333EB9002B08
:10024000C6D00120FFF7B6FF013DF3D1C0E7D7F8D4
:10025000182402F003023270002BB9D09DF8070079
:100260000128B5D1FFF7A6FF013DC6D1B0E7D7F809
:100270000C2402F00102EEE7FFF7A5BFF7B5164622
:10028000DDE90847019001A81D46FCF7D9FB019B59
:10029000B6F1000C18BF4FF0010C00EB83000B1EF1
:1002A00018BF0123002D43EA4C0314BF4FF00C0C80
:1002B0004FF0000C002C43EA0C0314BF4FF4E06C29
:1002C0004FF0000C002F43EA0C0314BF4FF4403CE6
:1002D0004FF0000CD0F8002243EA0C0322EA03039B
:1002E00001B109780EB13678760019430DB12D7839
:1002F000AD0031430CB12478240229430FB13F787B
:100300003F040C433C43C0F8004203B0F0BD1FB5AE
:100310000DF10F03019300238DF80F101A461946B3
:100320000093FFF7ABFF05B05DF804FBFCF748BC9A
:10033000FCF726BC0846FCF713BC4FF4801070474E
:100340004FF4805070474FF48070704770B50126AD
:10035000A2F58074A40806FA04F4054614EA010024
:1003600008D0A85830B100213046A950AA581A68C0
:1003700022431A6070BD00232DE9F34104460D4667
:100380000193904601AB4FF4A672FFF7DFFF4FF4E5
:10039000827229462046FFF7D9FF4FF48C72074638
:1003A00029462046FFF7D2FF064630B1B8F1000FCC
:1003B0001DD017B13E46D4F83C354FF4887229461B
:1003C000204601ABFFF7C2FF30B1B8F1000F03D0F8
:1003D00016B90FB1D4F83C354FF490722946204637
:1003E00001ABFFF7B3FF019802B0BDE8F0814646CC
:1003F000E3E7012370B504460D46642643610022FD
:1004000002212046FFF7B7FF20B90120FFF7D2FEF7
:10041000013EF4D100236B77C4F8003570BD08B1FC
:10042000FAF7D8BC7047704740B1C368587810F0ED
:1004300001001EBF1878B0FA80F040097047EFF352
:100440001183202383F31288BFF36F8FFEE708B573
:10045000FFF7F5FF10B5D0E9003433B90020E268AA
:10046000537843F00103537010BD2046984700288D
:10047000F4D00028B8BF4042FF28A8BFFF20E3689F
:100480001870ECE7FEF72CBFFEF71FBF82684369C8
:10049000134313F003030CD1C3600169994201D8DF
:1004A00000207047C168013311604169C2600A448D
:1004B000F3E76FF01500704710B5C0E90432002370
:1004C000816083610446FFF7E1FF0028A8BFC4E90B
:1004D000004410BDF8B504460D46EFF31186202305
:1004E00083F31288BFF36F8FC7686FB900F0CDF840
:1004F00050B18767456100F07AF8314604F1080091
:10050000BDE8F840FDF722BDE3682B60A369E56014
:10051000013BA36186F31188BFF36F8FF8BD2024E0
:1005200008B5EFF3118384F31288BFF36F8FFEF7E2
:1005300099FEF6E790F90E308B4201D0FDF7C2BC70
:100540000020704703460020C3E90033C3E90200DE
:1005500070473AB18A4205D3C0E90212C0E90000EF
:10056000002070476FF015007047EFF305800038EA
:1005700018BF01207047FDF7FBBCD0E900321360C3
:100580005A600023C0E90033704708B5FFF7F5FF54
:10059000437B23F0020343730023836008BD38B517
:1005A00004460D46FDF770FB637B43F00203637363
:1005B000E5B1A5602B689D4209D16B68C4E9005381
:1005C0001C606C6012E06A689A42F6D01B68002BCF
:1005D000F3D094F90E2093F90E108A42F3D0914291
:1005E000F1DD5A68C4E9003214605C6038BD10B5B2
:1005F000EFF31184202383F31288BFF36F8FFDF78D
:100600005BFB84F31188BFF36F8F10BD10B50446F8
:10061000183000F077F8EFF31181202383F312886C
:10062000BFF36F8F627B12F0100204D081F3118848
:10063000BFF36F8F10BD2046BDE81040FDF770BBC3
:1006400038B50446EFF31185202383F31288BFF3F6
:100650006F8F437B13F0280F0BD183680BB1FFF72B
:1006600094FF637B51B903F0FB0320466373FDF7EE
:1006700023FB85F31188BFF36F8F38BD03F0EB03C5
:10068000F3E701211838FFF7DBBF38B5EFF3118529
:10069000202383F31288BFF36F8F0468A0420DD02C
:1006A00034B12046FFF771FF04F1180000F02AF87A
:1006B00085F31188BFF36F8F204638BD0024F7E71C
:1006C000EFF31181202282F31288BFF36F8F027B38
:1006D000D2070CD581F31188BFF36F8F002383F30A
:1006E0001188BFF36F8F0423184602DF7047437BE6
:1006F0001B0704D581F31188BFF36F8F7047012268
:10070000FDF70EBB10B5EFF31184202282F312889F
:10071000BFF36F8F03683BB1FDF7E8FD002084F362
:100720001188BFF36F8F10BD6FF01500F7E708B5A4
:10073000FDF7FAFE08BDFDF7F7BE0000847DFF7FE0
:1007400001000000C5AD00000000000091AE0000F7
:10075000B407010039D900000000000095B2000084
:10076000C8070100F5FF0000000000002BFD00009D
:10077000F00701000DFD0000DC070100F5B00000EE
:100780000000000045C1000000000000F9FF00006B
:100790000000000065B100000408010025FE000013
:1007A00018080100CBF700002C080100C9C30000A5
:1007B00000000000AC1401004C0C0100640C0100AE
:1007C000AC010020C42D0020E7140100300D010011
:1007D000480D0100B2010020502E0020FB14010042
:1007E0006C0D0100D40D0100B40100203C0000207C
:1007F00005150100A00D0100D40D0100B601002077
:1008000058000020D014010000000000140D010069
:10081000B0010020000000000F150100E00D0100F4
:10082000540E0100B801002074000020C314010020
:10083000800C0100F80C0100AE010020182E0020F1
:100840000000000047F200000000000047F2000036
:100850000000000047F200000000000047F2000026
:100860000000000047F20000D1C90000B301010000
:100870000000000047F200000000000047F2000006
:10088000F00701009FFC0000DC0701009FFC000056
:100890000000000047F2000075D60000B30101001F
:1008A0000000000047F20000D9CF0000B3010100B2
:1008B0000000000047F200000000000047F20000C6
:1008C0000000000047F200000000000047F20000B6
:1008D0000000000047F200000000000047F20000A6
:1008E0000000000047F2000000000000D5C1000039
:1008F0000000000047F200000000000047F2000086
:100900000000000047F200000000000047F2000075
:100910000000000047F200000000000047F2000065
:100920000000000047F200000000000047F2000055
:100930000000000047F200000000000047F2000045
:100940000000000047F200000000000047F2000035
:100950000000000047F200000000000047F2000025
:100960000000000047F200000000000047F2000015
:100970000000000047F200000000000047F2000005
:100980000000000047F200000000000047F20000F5
:100990000000000047F200000000000047F20000E5
:1009A0000000000047F200000000000047F20000D5
:1009B0000000000047F200000000000047F20000C5
:1009C0000000000047F200000000000047F20000B5
:1009D0000000000047F200000000000047F20000A5
:1009E0000000000047F200000000000047F2000095
:1009F0000000000047F200000000000047F2000085
:100A00000000000047F200000000000047F2000074
:100A10000000000047F200000000000047F2000064
:100A20000000000047F200000000000047F2000054
:100A30000000000047F200000000000047F2000044
:100A40000000000047F20000061001000300000053
:100A5000DEE61E28EAAC45B8025B0000DEE61E2892
:100A60004CBBCE8F025B00000000000000000000C5
:100A70000338FDD870470000010000002A13010070
:100A8000840A01005B0000000080005000900050CC
:100A900018000000000000000000000000800000BE
:100AA00004080100010000000000000000800000B8
:100AB00004080100020000000000000000000D001A
:100AC0002C0801000300000000800000004001002D
:100AD0000408010004000000008000000002000083
:100AE000040801000500000000820000003E010033
:100AF000040801000600000000820000003E010022
:100B0000040801000700000000C0010000400000D0
:100B1000040801000800000000000200004001007D
:100B200004080100090000000000020000020000AB
:100B3000040801000A00000000020200003E01005B
:100B4000040801000B00000000400300004000000A
:100B5000040801000C0000000080030000020000F7
:100B6000040801000D0000000080030000000C00DC
:100B7000040801000E000000008003000080000057
:100B8000040801000F0000000082030000FE0B00BB
:100B900004080100100000000082030000FE0B00AA
:100BA000040801001100000000820300007E000024
:100BB00004080100120000000000040000800B0087
:100BC00004080100130000000000040000800B0076
:100BD000040801001400000000000D000000730074
:100BE0002C0801001500000000800F00002000000C
:100BF000040801001600000000800F000020000023
:100C0000040801001700000000A00F0000600000B1
:100C100004080100000000001DF200003000002068
:100C20002800002020000020000000001800002004
:100C30000DA7000011A6000065A60000BDA60000DB
:100C400019AE0000E9AD00000000000069AF00002F
:100C50005DAE0000B7140100DBF30000E1F300001B
:100C6000BD140100E9AE00005BF30000BBF300001F
:100C700000000000F9F20000000000000000000089
:100C80001808010000127A0000010100C8070100E5
:100C900019000100000000000000800000080000B2
:100CA00000100000C2281710B80C0100000001005D
:100CB0000000010001000000E520F1FFFFFFFF033D
:100CC00044EB086B083B04BBEEFFFFFFFFFF00FF98
:100CD000FFFF00FF0C200F5210D800FF2372F50019
:100CE00082ED04CC4483484430B030B0F7C4D55CC6
:100CF00000BE29FFF0D0FFFFF3F400000BF6000068
:100D0000C3F6000045B10000EDF300000100000053
:100D1000FF00000079FA0000F1B100008DB1000081
:100D20005DB100004DB1000004000000FF000000B4
:100D3000FFFFFFFF002584500000000000000000BE
:100D400000D000500000000019B3000089FB000033
:100D500095FB0000A9FB0000B3FB0000BDFB0000F9
:100D600099B40000D1FB000000000000009000508A
:100D700002000000000000007C0D01000090005007
:100D8000880D010001000000900D0100040000002A
:100D9000010000000E000400000602000F0606001D
:100DA000008000500200000000000000B00D0100B3
:100DB00000800050BC0D010001000000C40D0100C6
:100DC000040000001D0000001B0004001C060200BF
:100DD0001A06060057FC000055B9000049FC000047
:100DE00000B000500000000000127A000000000077
:100DF0000000000000000000FFFFFFFF0000FF00F8
:100E000000000000000000010100000049FD00009A
:100E1000FF1F0000240E0100FFFFFFFF0000000085
:100E20000000000000B00050300E01000100000082
:100E3000380E0100030000000D1808000C180C000B
:100E40000B180A00C80701000A000100C8070100CA
:100E500019000100F1BA000001FE00004407010082
:100E600044070100840701008C070100B40701005A
:100E7000B4070100FF8FFFFFFF8FFFFFFE8FFFFF13
:100E8000FE8FFFFFFD8FFFFFFC8FFFFFFC8FFFFF3B
:100E90006D757465785F667265652063616C6C65FD
:100EA000642077697468204E554C4C2070617261E3
:100EB0006D6574657200000043616E277420696E71
:100EC000697469616C697A65206D757465782C2028
:100ED000776173204E554C4C0D0A0000436F756CC2
:100EE00064206E6F74206C6F636B20706F77657217
:100EF0002073617665206D757465780001000200CD
:100F000010001100200021002200230024003000E6
:100F1000310032003300FFFF77C295F360D2EF7FDC
:100F20003552500F2CB6798025633A205374617284
:100F300074696E6720626F6F746C6F616465720AAA
:100F40000025633A20556E61626C6520746F2066DF
:100F5000696E6420626F6F7461626C6520696D6197
:100F600067650A0025633A20426F6F746C6F616495
:100F7000657220636861696E6C6F6164206164648E
:100F800072657373206F66667365743A20307825D6
:100F9000780A0025633A204A756D70696E6720747F
:100FA0006F2074686520666972737420696D61676B
:100FB0006520736C6F740A0025633A2050726F7459
:100FC000656374206D6375626F6F7420666C617306
:100FD00068206661696C65642C2063616E63656C72
:100FE00020737461727475702E0A0025633A204E66
:100FF000657665722073686F756C64206765742010
:10100000686572650A006D6375626F6F74002563B1
:101010003A20696E76616C696420666C6173682041
:1010200049442025643B20657870656374656420BD
:1010300025640A002A8648CE3D030107002A864817
:10104000CE3D02010025633A20556E61626C652039
:10105000746F2064657465726D696E6520666C617D
:10106000736820736563746F72206F66207468659F
:1010700020696D61676520747261696C65720A0030
:101080007072696D617279007365636F6E6461720D
:10109000790025633A20496D61676520696E207487
:1010A000686520257320736C6F74206973206E6FE0
:1010B000742076616C6964210A0025633A202564F6
:1010C000207374617475732077726974652066612A
:1010D000696C7320706572666F726D696E672074DB
:1010E000686520737761700A0025633A204661695C
:1010F0006C656420746F206F70656E20666C617320
:101100006820617265612049442025642028696D4A
:1011100061676520256420736C6F74202564293A0B
:101120002025642C2063616E6E6F7420636F6E7473
:10113000696E75650A0025633A204661696C6564CD
:101140002072656164696E6720736563746F727382
:101150003B20424F4F545F4D41585F494D475F53CD
:101160004543544F52533D2564202D20746F6F200A
:10117000736D616C6C3F0A0025633A204661696CAF
:1011800065642072656164696E6720696D61676579
:1011900020686561646572733B20496D6167653DD8
:1011A00025750A0025633A204661696C65642072E2
:1011B000656164696E6720626F6F74207374617417
:1011C00075733B20496D6167653D25750A00256390
:1011D0003A2070616E6963210A0025633A204465F4
:1011E00074656374656420696E636F6E736973748C
:1011F000656E7420737461747573210A0062616492
:1012000000676F6F6400756E736574005072696D6E
:1012100061727920696D6167650025633A202573E5
:101220003A206D616769633D25732C207377617087
:101230005F747970653D307825782C20636F707904
:101240005F646F6E653D307825782C20696D61672D
:10125000655F6F6B3D307825780A005365636F6E6C
:101260006461727920696D6167650025633A204287
:101270006F6F7420736F757263653A207072696D59
:1012800061727920736C6F740A0025633A20426F93
:101290006F7420736F757263653A206E6F6E650AA6
:1012A0000025633A205374617274696E6720737706
:1012B0006170207573696E67206D6F766520616C53
:1012C000676F726974686D2E0A0025633A204E6F4D
:1012D0007420656E6F75676820667265652073702F
:1012E00061636520746F2072756E20737761702062
:1012F000757067726164650A0025633A20726571D2
:101300007569726564202564206279746573206252
:101310007574206F6E6C7920256420617265206180
:101320007661696C61626C650A003059301306079A
:101330002A8648CE3D020106082A8648CE3D030192
:1013400007034200042ACB403CE8FEED5BA449952C
:10135000A1A91DAEE8DBBE1937CD14FB2F245737EA
:10136000E5953988D994B9D65AEBD7CDD5308AD6F8
:10137000FE48B24A6A810EE5F07D8B6834CC3A6A49
:10138000FC538EFAC12D0020002B0030780030581D
:1013900000286E696C29004661696C656420746F71
:1013A000207265626F6F743A207370696E6E696E39
:1013B0006720656E646C6573736C792E2E2E0A003F
:1013C0002A2A2A20426F6F74696E67204D79204166
:1013D00070706C69636174696F6E2076322E312E85
:1013E000302D6465762D646166323934366130663D
:1013F0003037202A2A2A0A002A2A2A205573696EA1
:1014000067206E524620436F6E6E656374205344AE
:101410004B2076322E372E302D35636238353537F6
:101420003063613433202A2A2A0A002A2A2A2055C6
:1014300073696E67205A6570687972204F53207601
:10144000332E362E39392D313030626566633730B0
:10145000633734202A2A2A0A006D757465785F691B
:101460006E69742063616C6C6564207769746820B0
:101470004E554C4C20706172616D6574657200430D
:101480006F756C64206E6F7420616C6C6F63617437
:1014900065206D75746578206265666F7265206978
:1014A0006E697469616C697A696E6700636C6F63F9
:1014B0006B4035303030006866636C6B006C66637F
:1014C0006C6B006D783235723634333566403100DE
:1014D000666C6173682D636F6E74726F6C6C65728D
:1014E000403339303030006770696F4038343235FE
:1014F0003030000001020304050607756172744074
:1015000039303030007561727440383030300073DB
:1015100070694062303030004552524F523A204399
:10152000616E6E6F742066756C66696C6C204558D0
:10153000545F41504920726571756573742E0D0AB0
:10154000005741524E494E473A204F7074696F6EB2
:10155000616C204558545F41504920726571756532
:101560007374206E6F742066756C66696C6C65644C
:101570002E0D0A007065726D00746573740042551B
:10158000473B2063616E27742068617070656E0050
:101590007265766572740025633A205365636F6ED9
:1015A0006461727920696D616765206F6620696D7D
:1015B0006167652070616972202825642E29206981
:1015C0007320756E726561636861626C652E20546C
:1015D0007265617420697420617320656D7074791F
:1015E0000A0025633A20496D61676520696E64656C
:1015F000783A2025642C20537761702074797065C7
:101600003A2025730A0025633A20496D61676520F9
:10161000696E6465783A2025642C205377617020C8
:10162000747970653A206E6F6E650A0004010403D8
:1016300004020401040104030103030401046D61B5
:10164000696E000000800000FFFF000088EACD1FE7
:1016500055555515AAAAAA1AE1F2000043EF000059
:10166000940A0100D00100203A000000E4010020AB
:101670003A000000BC0100203A000000F801002000
:101680003A000000F3F200000000000000C2010078
:1016900000010300000000009F3100209E31002067
:1016A000000000000000000000C201000001030073
:1016B00000000000A1310020A03100200000000047
:1016C0000000000000000000440E010002000000C5
:1016D00084000020840000200000000001000000C1
:1016E0009400002094000020000000000100000091
:1016F00000000000000000000000000000000000EA
:1017000000000000000000000000000000000000D9
:1017100000000000180801000000000000000000A8
:10172000AA310020A2310020FFFF000000000000CD
:1017300000000000000000000000000000000000A9
:101740000000000000000000000000000000000099
:101750000000000000000000000000000000000089
:101760000000000000000000000000000000000079
:101770000000000000000000000000000800000061
:10178000FF00000000000000010000000000000059
:1017900044010020440100200000000091E5000009
:1017A000900100208801002080010020000000003E
:1017B00078010020ADE60000F9E500002DE600000C
:1017C00075E60000C82E00203A00003ACC2E00201A
:1017D0003A00003AD02E00203A00003AD42E0020E1
:1017E0003A00003AA0010020640100205C010020C2
:1017F00058010020540100200000000000000000FB
:10180000000000000000FFFFBC010020BC01002020
:1018100000000000000000000E000000D0010020C9
:10182000D001002000000000000000000E000000B9
:10183000E4010020E401002000000000000000009E
:101840000E000000F8010020F80100200000000058
:10185000000000000E00000015E015E0DEE61E2886
:1018600083845186025B0100008200005C7AA969D2
:101870007758C1782D735C05D7BC9652EEAF9F7236
:1018800079FF705F065C9335C989C54137D8164822
:101890002528D47024B5E3C97EBF88A2E3C189148A
:1018A000B1F88A49039A05A69EA0A03C025AD78F98
:1018B0003F23390FE0A60185E2E017815386666178
:1018C0004EFDA66DB61CF78F819B3379A2E8431CB1
:1018D000C5473725EFE5A4F676C10FDCB9238C2A7E
:1018E0004F5269861CCB6FC554CB7DF56F5F19D6FF
:1018F000BF2D22970A725B1A686D91F5181FFD952E
:0C190000A771227B1AE109D76AC3C9DA7B
:020000040002F8
:1002000060080120812A0200397202006D2A020072
:100210006D2A02006D2A02006D2A02006D2A02007A
:10022000000000000000000000000000192C020087
:100230006D2A020000000000D92B02006D2A020086
:10024000952D0200952D0200952D0200952D02009E
:10025000952D0200952D0200952D0200952D02008E
:10026000952D0200952D0200952D0200952D02007E
:10027000952D0200952D0200952D0200952D02006E
:10028000952D0200952D0200952D0200952D02005E
:10029000952D0200952D0200952D0200952D02004E
:1002A000952D0200952D0200952D0200952D02003E
:1002B000952D0200952D0200952D0200952D02002E
:1002C000952D0200952D0200952D0200952D02001E
:1002D000952D0200952D0200952D0200952D02000E
:1002E000952D0200952D0200952D0200952D0200FE
:1002F000952D0200952D0200952D0200952D0200EE
:10030000952D0200952D0200952D0200952D0200DD
:10031000952D0200952D0200952D0200952D0200CD
:10032000952D0200952D0200952D0200952D0200BD
:10033000952D0200952D0200952D0200952D0200AD
:10034000952D0200000000000000000000000000E9
:10035000000000000000000000000000000000009D
:10036000000000000000000000000000000000008D
:10037000000000000000000000000000000000007D
:10038000000000000000000000000000000000006D
:10039000000000000000000000000000000000005D
:1003A000000000000000000000000000000000004D
:1003B000000000000000000000000000000000003D
:1003C000000000000000000000000000000000002D
:1003D000000000000000000000000000000000001D
:1003E000000000000000000000000000000000000D
:1003F00000000000000000000000000000000000FD
:10040000DEE61E284CBBCE8F025B00008C00000095
:100410005C960000010000000002020000020200E1
:10042000FFFF02910000000000000000000000003B
:10043000000000000000000002000000DEE61E28B0
:10044000EAAC45B8025B0000280000000310000081
:100450000100000001000000FF000000010000009A
:1004600060080120DEE61E28EAAC45B8025B000009
:100470002800000002100000000000000100000041
:10048000FF000000010000006408012053B94AB9D0
:10049000002908BF00281CBF4FF0FF314FF0FF308C
:1004A00000F00CB8ADF1080C6DE904CE00F008F8CE
:1004B000DDF804E0DDE9022304B07047704700BFB7
:1004C0002DE9F04786468C460846089E1546744638
:1004D0001946002B40F0C1808542B2FA82F245D91C
:1004E0004AB1C2F1200300FA02FC954094402EFA72
:1004F00003F343EA0C0C4FEA154EA8B2230CBCFBE5
:10050000FEF80EFB18CC08FB00F943EA0C439945B2
:1005100028D9EB1808F1FF3704D2994502D9A8F180
:1005200002072B44A3EB0903A4B2B3FBFEFC0EFBB2
:100530001C330CFB00F044EA0344A04214D92C19EC
:100540000CF1FF3304D2A04202D9ACF102032C44D7
:10055000241A43EA07401EB1D4400023346073607C
:10056000BDE8F0874746DDE76346F1E792BB431BF2
:1005700001214FEA154EAFB2200CB3FBFEFC0EFB7F
:100580001C330CFB07F840EA0343984561D9EB188C
:100590000CF1FF3004D2984502D9ACF102002B4493
:1005A000A3EB0803A4B2B3FBFEFC0EFB1C330CFB55
:1005B00007F744EA0344A7424DD92C190CF1FF3345
:1005C00004D2A74202D9ACF102032C44E41B43EA53
:1005D0000040C0E7C2F120039540944020FA03F1A7
:1005E0002EFA03F34FEA154E9040AFB20343B1FB2E
:1005F000FEFC0EFB1C10190C0CFB07F841EA004135
:10060000884522D969180CF1FF3004D2884502D9F7
:10061000ACF102002944A1EB08019BB2B1FBFEFC46
:100620000EFB1C110CFB07F743EA01439F420ED956
:10063000EB180CF1FF3104D29F4202D9ACF1020158
:100640002B44DB1B41EA004193E76046E3E7614648
:10065000F7E76046A4E76346B8E7834206D916B9D0
:10066000002108467CE7C6E900E0F9E7B3FA83F722
:100670008FB9834201D3724508D8BEEB020460EB08
:10068000030301209C461EB9002169E73846FAE7BA
:10069000C6E9004CF8E7C7F1200CBB400EFA07F59D
:1006A00022FA0CF42EFA0CF1BA401C4320FA0CF397
:1006B000B8404FEA144901431FFA84FEB3FBF9F82E
:1006C00009FB18300B0C08FB0EFA43EA00439A456D
:1006D00040D9E31808F1FF3004D29A4502D9A8F1B5
:1006E00002002344A3EB0A0389B2B3FBF9F809FB28
:1006F000183308FB0EFE41EA03418E452CD96118E0
:1007000008F1FF3304D28E4502D9A8F10203214437
:1007100043EA0040A1EB0E01A0FB02984145CE4602
:10072000434602D306D14D4504D20138B9EB020E3F
:1007300068EB0403002EA7D0B5EB0E0261EB0301BA
:1007400001FA0CFC22FA07F3F9404CEA0303C6E96C
:10075000003199E74046C5E74346D9E7F0B5354B48
:10076000354A4921C3F800263448C3F8042685B029
:10077000C3F80826C3F80C26C3F81026C3F81426BD
:10078000C3F81826C3F81C2606F0CCFC06F0F2F8D5
:1007900000F084FA054601A800F08EFF04462846C2
:1007A00000F08CFA264B1B68A34205D04521254852
:1007B00006F0B8FC06F0E0F9039A4921224806F059
:1007C000B1FC4921214806F0ADFC4FF440314FF413
:1007D000004003F0B7FD044620B145211C4806F057
:1007E000A1FCFEE769469DF8080000F035F8009B83
:1007F000039D1D44019B1E8903F08CFDAF1901F080
:10080000E9FA01F0B9FA01F0D3FA84F30B8884F322
:100810000A88AB5983F3088884F31488BFF36F8F79
:10082000BFF36F8F7B68984745210A4806F07AFC32
:10083000FEE700BF008001503546526E288F02004F
:1008400070C50020418F0200648F0200938F020068
:10085000B88F0200EB8F0200024608B538B1054898
:100860000023452106F05EFC6FF0150008BD08600E
:10087000FCE700BF0E90020021B1012908D06FF003
:100880001500704748B10128054818BFFF20704780
:10089000022834BF0220FF2070470D20704700BFA0
:1008A000030000002DE9F04FDFF8F8A1FDB03CA8EF
:1008B000DDE9888916461C468A9FDAF8005003F065
:1008C0005FFDB8F1000F07D0B9F1000F04DD4A4613
:1008D00041463CA803F062FD4FF00008338972895D
:1008E000D6F80CB013449B44C3453AD80CA93CA895
:1008F00003F05AFD27B1202238460CA906F0E5FC8A
:1009000000232246009331464FF6FF7306A806F0F7
:1009100032F8804610BB20460B9E00F0A9F98642B3
:100920001CD84FF0FF37DFF880910DF1120304AAB5
:1009300005A906A806F06DF800280FDB40F0A88096
:10094000059906A806F0B1F810BB4FF6FF71BDF887
:100950001200564A32F8023B8B4217D1DAF80050A7
:100960009AE0879BABEB0809994528BF9946414619
:100970004B462046869A06F0E3FB0028EED14A4615
:1009800086993CA803F00AFDC844ADE79842E1D13E
:10099000BDF81230102B1ED1BDF81060202EDDD115
:1009A0003346204605991CAA06F0CAFB0028D5D17B
:1009B00000F074F9324680461CA90CA800F0FEF83D
:1009C0000646404600F07AF9394B1B68B342C5D160
:1009D0004FF00108A9E7012B32D1BDF81030202BD0
:1009E000BCD8204605991CAA06F0AAFB0746002899
:1009F000B4D19DF810B0BBF1200F02D94FF0FF37F2
:100A000093E7D9F800302B4E0393039B9F42F5DA0E
:100A10003CA803F0B5FC72683CA8126856F8081BA5
:100A200003F0BCFC14A93CA803F0BEFC5A461CA968
:100A300014A806F03AFC00283FF477AF0137E4E74A
:100A4000222B7FF472AF7B1C3FF46FAFD9F80030DC
:100A5000BB42D3DDBDF81030802B3FF67FAF204680
:100A600005991CAA06F06CFB00287FF477AF00F014
:100A700015F9FFB206462021BDF810301CAA0097D8
:100A80000CA800F019F80546304600F017F9B5E754
:100A9000B8F1000F3FF462AF00F008F928467DB0CE
:100AA000BDE8F08F6CC50020788A0200FC8E020041
:100AB00070C500207C8A02002DE9F04796B01646EA
:100AC0001D469DF87820384B074653F8321003EB4B
:100AD000C2035B6801911868DFF8D08001443023BD
:100AE00002AA01A8D8F8009006F0B9F9002851D15F
:100AF000DDE901431C44214606AB03AA01A806F028
:100B0000D6F9002846D1049A072A43D128490598E6
:100B100006F0CBFB00283DD1079A082A3AD1254997
:100B2000089806F0C2FBA8BB214602AA01A806F05D
:100B3000AAF978BBDDE901A30AEB0302944229D1AB
:100B4000412B27D135443023294603AA02A8029617
:100B500006F085F9E0B9DDE9023213449D4217D36E
:100B60002A4602A906A805F0AEFF88B92A4602A9BE
:100B70000EA805F0A8FF58B99AF80030042B07D149
:100B80002021384606AB0AF1010203F013FC38B10C
:100B9000D8F8009000F08AF8484616B0BDE8F08713
:100BA000054BD3F80090F5E77C8A02006CC5002065
:100BB0003D9002003490020070C5002070B5094BD2
:100BC00004461D680023934205D1074B1D6800F0C1
:100BD0006DF8284670BDE65CC85C8642F7D10133EB
:100BE000F1E700BF6CC5002070C500200B7868B12C
:100BF000012806D0FF2B14BF4FF0FF304FF4407098
:100C00007047054A934203D0022BF4E70D2BFAE715
:100C10004FF44070704700BF030000001FB50C4642
:100C2000A8B1012815D11048C0B2214601F080FCBE
:100C300050B92068102381686A46103906F080FA9E
:100C400048B1206806F07BFA4FF0FF300AE00D2033
:100C5000EBE7FF20E9E710226846044906F025FB90
:100C60000028EED104B010BD03000000188F020070
:100C700013B5044605F058FF6A460146204605F0C4
:100C800060FE30B10448452106F04CFA002002B065
:100C900010BD0098FBE700BF45900200024B1868AA
:100CA000421C1A60704700BF38C90020024A13680E
:100CB000013B1360704700BF38C90020034B1B681D
:100CC000834201D005F058BF704700BF38C90020EB
:100CD00003464FF4807213B5084693F8B81001929A
:100CE000C1B1012903D0FF2804D0012010E0104A2F
:100CF000904211D1582404FB013204FB0133526AA3
:100D000003F1280401A901F03BFC08B9019B236011
:100D100002B010BD0D28ECE70228E6D1582404FBF0
:100D2000013204FB0133126D03F15404EAE700BF02
:100D30000300000038B590F8B8300446F3B1012B39
:100D400006D0FF21FFF7C4FFD0B10125284638BDEA
:100D50000D49FFF7BDFF0028F7D102212046FFF71C
:100D6000B7FF054670B9582294F8B83002FB034328
:100D7000186A06F023FAC4F8B400E7E70D21E8E7A3
:100D8000FF21EBE70925E1E7030000002DE9F04F23
:100D90004A4B8DB0044690F8B8000D461E68FFF728
:100DA0006BFD0AA9C0B201F0C3FB28B1FFF77EFFBB
:100DB00030460DB0BDE8F08F94F8B8B029465846DB
:100DC000FFF75AFD4FF02C080BA9C0B208FB05F83D
:100DD00001F0AEFB00284ED04FF0580A2C230AFB3E
:100DE0000BF703FB057704EB0709D9F8106016F041
:100DF000100655D1FFF752FF0A9B94F8B8100690E1
:100E000009930891FFF74AFF07904FF480701AFB8F
:100E10000B8201902A48CDE90366099B0899029646
:100E2000009022443046FFF73DFD06460798FFF745
:100E300045FFFFF73BFF0698FFF740FF214BE259C4
:100E40000A989A420CD1D9F80C20B9F808309B18AE
:100E500006D28268934203D21B4B1B68B34226D052
:100E60004DB38268002106F095F9184A45211848CB
:100E700006F058F919E00B9806F0A7F906460B980A
:100E800006F05DF9582394F8B82013FB028323443D
:100E90005A1E033312F8011FB1429DD19A42F9D173
:100EA0001DB120460A9905F002FF0A4B1E680A98F8
:100EB00006F045F97AE7084AD8E700BF6CC500207C
:100EC00004F600203DB8F39670C50020889002001B
:100ED0009290020068C50020809002007FB50D4608
:100EE0000021044690F8B8202846CDE9021105F00B
:100EF000CFFE60B358235A431C4EA358B34203D1CC
:100F0000204603AA05F06CFE582294F8B83002FB84
:100F10000343DB6AB34204D10121204602AA05F053
:100F20005FFEDDE90232934288BF0393039BAB600F
:100F3000039A2946204600F0F9FD0D4B1A68002A55
:100F400003DD57210B4806F0EDF804B070BD1046E4
:100F500001A9FFF763FE019805F1080105F0EFFD17
:100F6000AB680198039306F0EAF8E1E73DB8F39621
:100F7000F8ED0020BA9002007FB590F8B830064630
:100F80000D468BB3012B1A4818BFFF2001A9C0B230
:100F900001F0CEFA50BB019805F0C6FDD6F8B410AA
:100FA0000446284605F0FAFE0444019806F006F9C6
:100FB0000646019806F009F9082201460DEB0200E9
:100FC00006F08EF92B7921468DF8083001983346CA
:100FD00002AA06F0CAF8041E019818BF012406F000
:100FE000AEF8204604B070BD0D20CFE70124F8E72D
:100FF000030000002DE9F84F884691469A460026E6
:10100000DFF868B01A4C1B4D0B9B9E4201D30020A9
:101010000FE00B9B40469F1BB7F5806F28BF4FF436
:101020008067124A3B4606EB0A0106F089F810B1C8
:101030000120BDE8F88F0A993B465A464846711888
:1010400006F093F80028F3D1C4F800563E44C4F8E3
:101050000456C4F80856C4F80C56C4F81056C4F820
:101060001456C4F81856C4F81C56CDE73CE90020C5
:10107000008001503546526E2DE9F04F4FF0000AC6
:1010800004460E46574693B0BAF1010F84F8B8A053
:1010900006D9002F00F0F28100202C25582767E1A7
:1010A00004EB0A0292F8B950002D4AD14FF05809CA
:1010B0004FF02C0B09FB0A42B04B03EBCA21B04B9B
:1010C000516203EBCA21116529465046FFF7D4FB54
:1010D000202394F8B810804619FB01310BFB051151
:1010E000C0B2214401F024FA48B15346424645219A
:1010F000CDE90050A34806F015F805F03DFD4FF08E
:1011000001087DB12046FFF715FE054660B90022B3
:101110002046114605F043FDC8B1572194F8B82088
:10112000994824E04546CFE74FF48072572197480D
:1011300005F0F8FF94F8B830012D234483F8B0800F
:10114000E5D194F8B83001335FFA83FA9CE7204682
:1011500005F037FE68B108A805F091FD014620466C
:1011600000F0C4FA60B1572194F8B820884805F01F
:10117000D9FF012294F8B830234483F8B020E0E787
:1011800008A805F085FD80F0010108AA2046C9B233
:1011900005F005FD02460028BFD108A805F078FD3E
:1011A000054600284CD194F8B8305BBB204608A90E
:1011B000FFF794FE94F8B8009DF82730221882F8C3
:1011C000B030033B012B08D800F0F4FA28B1FF221D
:1011D00094F8B830234483F8B0209DF8273094F871
:1011E000B800023B022B1ED800F0C8FAD8B1FF228B
:1011F00094F8B830234483F8B0204521654805F0C1
:1012000091FFFEE794F8B020042A04BF012284F87D
:10121000B020012BCAD094F8B130042BC6D10123E1
:1012200084F8B130C2E794F8B830234493F8B03072
:10123000FF2BE2D00021204608AA05F0B0FC98E779
:101240009DF82730012B74D1582194F8B830DFF87D
:101250004881059208F8032001FB03434F4AD96AED
:10126000D86C914247D1998E042305AA194405F000
:1012700067FF014608B34FF0050994F8B8302344DE
:1012800083F8B09094F8B83073B1E21892F8B020B7
:10129000012A3FF456AF042A0DD094F8B020042A56
:1012A00002D1012284F8B020234493F8B030023BED
:1012B000022B3FF646AF2F4643E794F8B800FFF7FE
:1012C000DBFA0CA9C0B201F033F90028D3D10C9A93
:1012D000059953688B4229D892681A44914225D8BF
:1012E000B3F5004F02D0B3F5003F04D1012294F8CA
:1012F000B83008F8032094F8B80003F02DF9831EE5
:10130000022B8146B9D8FFF7C9FC0121804620464F
:10131000FFF73CFD82464046FFF7D0FC204B1B68A0
:101320009A45AAD01F4B1B689A45A4D14FF00109DA
:10133000A3E7FFF7B3FC012180462046FFF726FD17
:1013400081464046FFF7BAFC154B1B68994518BF0C
:10135000052294F8B83008BF9DF82720234483F86D
:10136000B0208FE7231893F8B920EAB10130C0B25A
:10137000012884F8B800F5D980E000BF3CD90020EE
:101380003CC90020E99002007891020036910200E9
:10139000A4910200CE91020004F700203DB8F3961C
:1013A00070C5002068C5002093F8B08008F0FB08E5
:1013B000B8F1010818BF4FF001084146FFF75CFA89
:1013C00003A9C0B201F0B4F8002840F08C800123DA
:1013D00005FB08F894F8B810039A17FB01810093F5
:1013E000214440230CA805F0C6FA804600287CD191
:1013F00000230DF10A0204A90CA805F00AFB00283D
:101400003CDB03987ED1BDF80A300C2B78D10499CF
:1014100005AA05F095FE00287DD19DF81430012B1A
:101420007CD8E21892F8B0207B43023A022A8CBFA3
:101430000022012205FB02332344197D9DF8182068
:101440009142D5D80AD3597D9DF819209142CFD821
:1014500004D3DA8ABDF81A309A42C9D294F8B83067
:101460000398234493F8B020012A3AD0023A012A83
:1014700002D8012283F8B02005F061FE0022894DD8
:10148000894F012A84F8B8204BD90023874DDFF813
:101490002082884F0C93012B84F8B83040F2998059
:1014A0000C9B022B01D005F067FB94F8B930002BA0
:1014B00040F0DB80582505FB034284F8B830106A01
:1014C00005F03DFA307194F8B83005FB03431B6A10
:1014D0005B68B36094F8B83003FB05453560734B27
:1014E00093E00422C6E70398C6E7039805F027FEB9
:1014F000B8F1030FC2D140F20113A4F8B030BDE738
:101500004FF00308039805F01AFEB8F1000FEFD171
:1015100094F8B8002AE74FF00108F3E74FF0070806
:10152000F0E7A11891F8B93043BB08A805F0A7FB74
:1015300091F8B030042B8DF8273006D8012B22D833
:101540000FD0FF2381F8B0300BE0052BF9D1104606
:1015500000F030F928B1FF2294F8B830234483F822
:10156000B02094F8B830234493F8B030FF2B05D165
:101570004521284605F0D6FD05F0FEFA94F8B8207E
:101580000132D2B27DE7204608A9FFF7A7FC94F804
:10159000B800231893F8B030DA1E012A0FD800F0F3
:1015A00009F978B994F8B80000F0E8F850B994F85F
:1015B000B830FB5C002BD4D0012000F095FE022B4C
:1015C000F5D1EFE7FF2294F8B830234483F8B02038
:1015D000EDE7234493F8B9208DF814209DF81410FA
:1015E00001F0FF0239B10C9B01330C9394F8B83031
:1015F0000133DBB24FE793F8B030012B07D011462F
:10160000204605F0CCFA10B1294B1D681AE094F879
:10161000B830012BE7D0FFF741FB0021824620467E
:10162000FFF7B4FB81465046FFF748FB2B6899450E
:1016300006D1D8F80030994502D03B689945D2D1FF
:10164000D8F800501022002108A805F049FE5826BD
:101650000023012B84F8B8300FD9FFF727FB284669
:1016600013B0BDE8F08F012324E794F8BA30002BC3
:10167000F9D0022384F8B83031E7E21892F8B920A3
:101680005AB906FB0343D86C05F059FD94F8B830FD
:1016900006FB0343186A05F052FD94F8B830013395
:1016A000DBB2D6E7CE91020004F7002070C500201F
:1016B0006CC5002068C5002070B50B4E0446BC22E6
:1016C0000021304605F00CFEFFF7E8FA21460546FA
:1016D0003046FFF7D1FC04462846FFF7EFFAFFF744
:1016E000E5FA204670BD00BF3CED002073B50D4605
:1016F000064600F05BF90446E86090B3022837D153
:1017000096F8B83083B3012B1B4818BFFF2001A9FE
:10171000C0B200F00DFF68BB2A463146019800F0C8
:10172000DFF80446D0B9019806F06FFC01230146AA
:101730000DF10302019805F003FD0446B0B9012242
:1017400001980DF1030106F074FC10B101238DF82E
:1017500003309DF8033003F00F03EB71019805F09F
:10176000EEFC204602B070BD0D20D0E70124F5E765
:101770000724F6E70124F4E70300000013B588B15D
:10178000012811D10A48C0B201A900F0D1FE68B900
:10179000019806F0E5FC0446019805F0D0FC2046CF
:1017A00002B010BD0D20EFE7FF20EDE70124F6E7C2
:1017B000030000001FB5D8B101281BD11048C0B2EA
:1017C00001A900F0B5FEC8B9019802A902F06EFEA9
:1017D000044688B99DF80B30032B03D1019806F01D
:1017E0008DFC0446019805F0AAFC204604B010BD0B
:1017F0000D20E5E7FF20E3E70124F3E70124F4E708
:10180000030000002DE9F74306460C4690461D46AE
:101810000BB900272FE0184605F03AFA0028F8D156
:10182000694696F8B800FFF7F9F9009838B901242D
:10183000009805F084FC204603B0BDE8F08301A9C0
:1018400005F07DF90028F2D1009805F078FC3046CB
:10185000019905F094FA582296F8B83002FB036318
:101860005B6A5F686B79012B23D1002CD1D12B6887
:10187000834298BF0027214696F8B800FEF7FCFF88
:101880006946C0B200F054FE0028D0D12023424661
:101890003946009805F054FC04460028C7D1002DB5
:1018A000C6D0D8F800400D4BE41A18BF4FF0FF34F3
:1018B000BEE7022BADD12B68012B05D98342A8D8F6
:1018C000B4FA84F46409A4E7A3D1002CD3D0012C8A
:1018D0009FD12C79023C18BF01249AE73DB8F396BA
:1018E0002DE9F04F0C460746014685B094F8B80044
:1018F0001646FFF77BF9051E52DB3846D4F8B44094
:1019000005F012F95FFA84F94FF0000A4FF0010B6D
:101910004FF0FF346B1E09FB03089DB9BAF1010FAC
:1019200003DD4521204805F0FDFB631C06D0FF2C9C
:101930002ADC40F2011301343460B380284605B03C
:10194000BDE8F08F6B1E00934146012338460DF130
:101950000F0205F0F5FB031E019323DB012238463D
:101960000DF10F0106F065FB019B40B15B4501D015
:101970000AF1010A9B46009DA8EB0908CDE7B4F1E6
:10198000FF3F08BF2C46F5E70223A4F5807473716E
:10199000631004F001040133013433603471CDE786
:1019A0000725CBE70125C9E7DA91020010B590F8C9
:1019B000B84088B0002C4ED0012C2D4818BFFF2015
:1019C00004A906F0A8FB9DF81020012A45D0294B58
:1019D0002949032A08BF0B469DF813202748029285
:1019E0009DF81220492101929DF811200092244A6D
:1019F00005F098FB012C8CBFFF20022006A906F001
:101A00008AFB9DF81820012A29D01A4B1A49032A6B
:101A100008BF0B469DF81B20492102929DF81A2011
:101A2000164801929DF819200092164A05F07AFB9B
:101A30009DF81030012B14D19DF81230032B10D1DA
:101A40009DF81830012B0CD00F48492105F06AFB96
:101A5000022008B010BD0D20B2E70C4BBCE70B4BC9
:101A6000D8E70B48492105F05DFB0020F1E700BFF6
:101A700003000000FD910200069202001A9202008B
:101A80000C9202005B9202006B9202000192020033
:101A90008A92020070B54B6814461E4A03F0FF2379
:101AA000934206460D4686B02FD10B68012B2CD1F0
:101AB000204604A902F0FAFC9DF81020012A26D045
:101AC000154B1649032A08BF0B469DF813204921E0
:101AD00002929DF81220124801929DF81120009266
:101AE000104A05F01FFB9DF81030032B0DD1214645
:101AF000304605F0DCF8204606F000FB2046A968D9
:101B000005F02BF8204602F0B1FC06B070BD064B84
:101B1000DBE700BF00010004FD9102000692020015
:101B20001A9202005B920200019202002DE9F04F2E
:101B300004461646582789B00D468548492105F0C8
:101B4000F1FA3146204605F01AF994F8B830834688
:101B500007FB03435B6A28465E6805F099F810B3FB
:101B6000D4F8B40004F0DBFF94F8B83007FB03436B
:101B70009F6A0023013F3344834201D2013FFAE7C9
:101B8000BB4510D35721734805F0CCFA07FB06F389
:101B900057210BFB0662704805F0C4FA0123EB7174
:101BA00009B0BDE8F08F94F8B83006A9D3B1012B85
:101BB00012D0FF2000F0BCFCFF2007A900F0B8FC09
:101BC00029462046079AFFF765FF6B79012B58D10C
:101BD0005F46DFF888A14EE06148C0B200F0A8FC83
:101BE0000220EAE70D20F9E72A68C2F101035B440D
:101BF0009F423FD8582194F8B830012A01FB034393
:101C00005B6A196853F8370003EBC70353F8083CC5
:101C1000A0EB0109A3EB0103049311D1079B0393EC
:101C2000EB68022B08D04146204605F040F82A46D2
:101C30004146204605F07FF82046039905F037F825
:101C400032464946404605F030F8049B424641463C
